:100000000C94A6160C94D7160C94D7160C94D716ED
:100010000C94D7160C94D7160C94D7160C94D716AC
:100020000C94D7160C94D7160C94D7160C94D7169C
:100030000C94D7160C9475590C94D7160C94D716AB
:100040000C94D7160C944DB30C94D7160C94D71669
:100050000C94D7160C94D7160C94637D0C942B59E2
:100060000C94D7160C94074C0C94D7160C94D716F6
:100070000C94D7160C94D7160C94D7160C94D7164C
:100080000C94D7160C94D7160C94D7160C94D7163C
:100090000C94D7160C94D7160C94D7160C94D7162C
:1000A0000C94D7160C94D7160C94D7160C94D7161C
:1000B0000C94D7160C94D7160C94D7160C94D7160C
:1000C0000C94D7160C94D7160C94D7160C94D716FC
:1000D0000C94D7160C94D7160C94BA580C947B58E1
:1000E0000C94D716E131FE312F324C3261328A3214
:1000F000F7325D33063440384E3847386E38723840
:100100008C38E73CA138ED3814393B396439BA39B9
:10011000CB39DC39ED39FE390F3AE73CF23BE73CAD
:10012000FD3B6D3C733C933C10C113C102C106C141
:100130000CC14AC117C11BC121C125C129C12FC191
:1001400033C137C14AC13DC141C145C1ADC6B2C6C7
:10015000B7C6C1C6CBC644C7D5C6DDC6E5C6EFC661
:10016000F9C603C712C71CC744C726C730C73AC75A
:10017000084AD73B3BCE016E84BCBFFDC12F3D6C0E
:1001800074319ABD56833DDA3D00C77F11BED9E474
:10019000BB4C3E916BAAAABE000000803F05A84C54
:1001A000CDB2D44EB93836A9020C50B99186880820
:1001B0003CA6AAAA2ABE000000803F004E414E493C
:1001C0004E495459494E46CDCCCC3D0AD7233C1715
:1001D000B7D13877CC2B329595E6241FB14F0A0062
:1001E0000020410000C84200401C4620BCBE4CCA52
:1001F0001B0E5AAEC59D74434F4D4D554E4943415C
:1002000054494F4E0044525952554E004552524F98
:10021000525300494E464F004543484F0047322F46
:1002200047332062616420706172616D657465722C
:10023000730A00206F6620004D424C20473239205F
:10024000706F696E74200059206F7574206F66207E
:1002500072616E67652028312D35292E0A005820DD
:100260006F7574206F662072616E67652028312D6E
:1002700035292E0A004D6573682070726F62696EB1
:100280006720646F6E652E0A005374617274206D6E
:100290006573682070726F62696E67207769746831
:1002A0002022473239205331222066697273742E1E
:1002B0000A004732380A47323920533200537461FA
:1002C00074653A20004D65736820626564206C6532
:1002D00076656C696E6720686173206E6F2064615B
:1002E00074612E0A0053206F7574206F662072614E
:1002F0006E67652028302D35292E0A004D657368FC
:1003000020706F696E742063616E6E6F7420626519
:10031000207265736F6C7665640A00456E642066B2
:10032000696C65206C6973740A00426567696E20A8
:1003300066696C65206C6973740A00286E6F2066AC
:10034000696C6529005344207072696E74696E6728
:10035000206279746520004E6F74205344207072BF
:10036000696E74696E670A0043757272656E7420F7
:1003700066696C653A20005072696E742074696D0C
:10038000653A20006F6E2E0A006F66662E0A0047DF
:1003900032362044656275672000180213020C0291
:1003A0000502F7016F66660044454255473A004B27
:1003B000494C4C45442E20004D3131332053006FC1
:1003C0006B002C20002C2000544845524D414C5FBE
:1003D00050524F54454354494F4E004155544F528B
:1003E00045504F52545F53445F535441545553004A
:1003F000454D455247454E43595F50415253455232
:1004000000434153455F4C494748545F4252494776
:1004100048544E45535300544F47474C455F4C4951
:100420004748545300534F4654574152455F504F2D
:10043000574552004255494C445F50455243454E42
:1004400054004C4556454C494E475F444154410089
:100450005A5F50524F4245004155544F4C45564506
:100460004C005052494E545F4A4F420050524F4741
:1004700052455353004155544F5245504F52545FCB
:1004800054454D5000564F4C554D4554524943002C
:10049000454550524F4D0053455249414C5F584FCE
:1004A0004E5F584F4646004649524D574152455FB0
:1004B0004E414D453A4D61726C696E20312E312EA0
:1004C0003920284769746875622C206461766964F4
:1004D00072616D69726F2920534F555243455F43D6
:1004E0004F44455F55524C3A68747470733A2F2FDD
:1004F0006769746875622E636F6D2F4D61726C69E8
:100500006E4669726D776172652F4D61726C696EAE
:100510002050524F544F434F4C5F56455253494F12
:100520004E3A312E30204D414348494E455F545993
:1005300050453A416E796375626963206933204D95
:100540006567612045585452554445525F434F55A5
:100550004E543A3120555549443A636564653261D9
:1005600032662D343161322D343734382D396231D1
:10057000322D6335356336326633363766660A00A8
:100580002F2F2000205400205200416363656C65CA
:10059000726174696F6E3A2050005741524E494E55
:1005A0004721204C6F77205A204A65726B206D617D
:1005B00079206C65616420746F20756E77616E744C
:1005C0006564207061757365732E0A00546F6F2027
:1005D0006661722066726F6D207265666572656E07
:1005E000636520706F696E740A0020466C6F773AFD
:1005F00020000001363726032BFFFFFF3C3D382A41
:10060000FFFFFFFF2E303E12FFFFFFFFFFFFFF083F
:1006100009FF2C071A1C18FFFFFF08440A2C43246B
:10062000221E20643A0020693A0020703A00496E88
:1006300076616C69642065787472756465720A000D
:1006400043290A0061626C656420286D696E20741C
:10065000656D702000436F6C6420657874727564FA
:10066000657320617265200020643A0020693A00B9
:1006700020703A004E6F2063617365206C69676873
:10068000740A00454550524F4D204F4B0A00205AE6
:10069000004475616C20456E6473746F7020416412
:1006A0006A7573746D656E7420286D6D293A20002B
:1006B0003F4B2076616C7565206F7574206F6620E6
:1006C00072616E67652028302D3130292E0A004175
:1006D0006476616E6365204B3D00416374697665A5
:1006E0002045787472756465723A2000496E7661AF
:1006F0006C69642065787472756465720A00436180
:100700006E6E6F7420656E746572207375626469B5
:10071000723A20004739310A4731205A2D302E31A4
:100720000A473930005370656369616C204D656E0E
:10073000753A205A20446F776E20302E310A0047D8
:1007400039310A4731205A2D302E30320A4739309C
:10075000005370656369616C204D656E753A205A6F
:1007600020446F776E20302E30320A004739310A2C
:100770004731205A2B302E30320A4739300053701F
:10078000656369616C204D656E753A205A2055701D
:1007900020302E30320A004739310A4731205A2B97
:1007A000302E310A473930005370656369616C201F
:1007B0004D656E753A205A20557020302E310A0052
:1007C000473239205332005370656369616C204DA4
:1007D000656E753A204E657874204D6573682050BB
:1007E0006F696E740A0047323920533100537065C7
:1007F0006369616C204D656E753A20537461727443
:10080000204D657368204C6576656C696E670A00DB
:100810004D31343020533630005370656369616C5C
:10082000204D656E753A205072656865617420428E
:1008300065640A004D353032005370656369616C40
:10084000204D656E753A204C6F61642046572044F8
:10085000656661756C74730A004D353030005370F5
:10086000656369616C204D656E753A2053617665EC
:1008700020454550524F4D0A004D33303320452D11
:100880003120533630204336205531005370656394
:1008900069616C204D656E753A204175746F205406
:1008A000756E6520486F74626564205069640A0043
:1008B0004D31303620533230340A4D3330332045F9
:1008C000302053323130204336205531005370658B
:1008D0006369616C204D656E753A204175746F20B7
:1008E00054756E6520486F74656E64205049440AE3
:1008F000003C5370656369616C5F4D656E753E00C9
:100900003C5370656369616C5F4D656E753E002F89
:10091000002F002F002F2E2E0A002F2E2E002F2EFC
:100920002E003C5370656369616C5F4D656E753E6A
:100930000A003C5370656369616C204D656E753EBD
:10094000003C5370656369616C204D656E753E00B7
:100950003C4C6F61642046572044656661756C7439
:10096000733E003C4C6F61642046572044656661CD
:10097000756C74733E003C4175746F2054756E65E0
:1009800020486F74626564205049443E003C4175C4
:10099000746F2054756E6520486F746265642050D2
:1009A00049443E003C4175746F2054756E65204883
:1009B0006F74656E64205049443E003C4175746F0D
:1009C0002054756E6520486F74656E6420504944EC
:1009D0003E003C457869743E003C457869743E00B1
:1009E0003C5361766520454550524F4D3E003C5387
:1009F00061766520454550524F4D3E003C4E65782E
:100A000074204D65736820506F696E743E003C4ED3
:100A1000657874204D65736820506F696E743E0070
:100A20003C5374617274204D657368204C65766523
:100A30006C696E673E003C5374617274204D65733F
:100A400068204C6576656C696E673E003C50726547
:100A500068656174206265643E003C50726568653B
:100A60006174206265643E003C5A20446F776E20BA
:100A7000302E313E003C5A20446F776E20302E31AC
:100A80003E003C5A20446F776E20302E30323E00BC
:100A90003C5A20446F776E20302E30323E003C5A54
:100AA00020557020302E30323E003C5A20557020A8
:100AB000302E30323E003C5A20557020302E313ED0
:100AC000003C5A20557020302E313E0056313136D0
:100AD000004A333320004D3530300A4D3432302057
:100AE00053310A4731205A313020463234300A47D8
:100AF00031205830205930204636303030004A32CC
:100B000032004A3232004731205A352046323430E2
:100B10000A4731205831393020593230204636309A
:100B200030300A4731205A302046323430004731C5
:100B3000205A3520463234300A4731205831393076
:100B400020593139302046363030300A4731205A6A
:100B5000302046323430004731205A352046323476
:100B6000300A47312058313930205932302046364A
:100B70003030300A4731205A302046323430004776
:100B800039310A4731205A313020463234300A4751
:100B900039300A4732380A4732390A473120583249
:100BA00030205932302046363030300A4731205A12
:100BB000302046323430004A3032004A3132004769
:100BC00031205A3130004F4B004731205A3130002C
:100BD00047393000473120452569463530300047D8
:100BE0003120452D302E31462569004731204530D2
:100BF0002E31462569004731205A2569462569006E
:100C00004731205A2D302E31462569004731205A70
:100C1000302E31462569004731205925694625691E
:100C200000473120592D302E3146256900473120AB
:100C300059302E314625690047312058256946250F
:100C40006900473120582D302E3146256900473143
:100C50002058302E31462569004739310047323857
:100C600000473238205A004732382059004732387E
:100C70002058004132305620004731205A31300090
:100C80004A3034004A3231004A3230004B494C4C31
:100C900045442E20004A303400454E4400464E2044
:100CA000004A3032003939393A393939004D004873
:100CB000004137562000413656202D2D2D004A3058
:100CC000320041365620005A3A2000593A20005846
:100CD0003A20004135560041345620004133562019
:100CE000004132562000413156200041305620004C
:100CF0004D383400473930004731205A35302046CE
:100D00003234300047393100473930004731205AFA
:100D10003135204632343000473931004739300010
:100D20004731205A31204632343000473931004AA9
:100D30003136004A3138004739310A4731205A31BB
:100D40003020463234300A473930004A3134004AC4
:100D50003030004A3031004A31300024F4D4305071
:100D6000C38E20C2A24017828B7011127A910D811E
:100D70006CD90AA861E108C7586607615143061E8D
:100D80004B5D05C145A7041A411104093D98037143
:100D90003931034036DB0265339102D4305402808E
:100DA0002E1D02632CEE01752AC501B028A001108A
:100DB0002781018F2564012B244B01E0223401ACF3
:100DC000211F018D200D01801FFC00841EED009766
:100DD0001DDF00B81CD200E61BC600201BBC00644F
:100DE0001AB200B219A8000A19A0006A189900D115
:100DF00017910040178B00B516840031167E00B3A2
:100E00001579003A157300C7146F0058146A00EE84
:100E10001366008813630025135E00C7125B006C25
:100E200012570015125400C111510070114F0021CA
:100E3000114B00D61049008D1047004610440002A7
:100E4000104200C00F4000800F3E00420F3C0006E1
:100E50000F3B00CB0E3800930E37005C0E35002799
:100E60000E3400F30D3200C10D3100900D300060E2
:100E70000D2E00320D2D00050D2C00D90C2B00AECF
:100E80000C2900850C29005C0C2700350C27000E6E
:100E90000C2600E80B2400C40B2400A00B23007DCB
:100EA0000B23005A0B2100390B2100180B2000F8EE
:100EB0000A1F00D90A1E00BB0A1E009D0A1D0080E1
:100EC0000A1D00630A1C00470A1B002C0A1B0011A4
:100ED0000A1A00F7091A00DD091900C4091900AB44
:100EE000091900920917007B091800630917004CC3
:100EF00009160036091600200916000A091500F522
:100F0000081500E0081400CC081400B8081400A468
:100F1000081400900813007D0812006B0813005895
:100F200008120046081200340811002308110012AC
:100F300008110001081100F0071000E0071000D0B0
:100F4000071000C0071000B0070F00A107100091A4
:100F5000070E0083070F0074070F0065070E005788
:100F6000070E0049070E003B070D002E070E00205C
:100F7000070D0013070D0006070D00F9060C00ED24
:100F8000060D00E0060C00D4060C00C8060C00BCE0
:100F9000060C00B0060C00A4060B0099060C008D90
:100FA000060B0082060B0077060B006C060B006137
:100FB000060A0057060B004C060A0042060A0038D3
:100FC000060A002E060A0024060A001A060A001065
:100FD00006090007060A00FD050900F4050900EBF3
:100FE000050900E2050900D9050900D0050900C777
:100FF000050900BE050900B5050800AD050800A5F6
:101000000509009C050800940508008C050800846B
:101010000508007C050800740508006C05070065DC
:101020000508005D050700560508004E0507004746
:101030000507004005080038050700310507002AAC
:10104000050700230507001C050600160507000F0D
:101050000507000805060002050700FB040600F569
:10106000040700EE040600E8040600E2040700DBC3
:10107000040600D5040600CF040600C9040600C318
:10108000040600BD040600B7040600B1040500AC68
:10109000040600A6040600A00405009B04060095B3
:1010A000040500900406008A0405008504050080FC
:1010B0000406007A04050075040500700405006B41
:1010C00004050066040500610405005C0405005782
:1010D000040500520405004D0405004804050043C2
:1010E0000405003E0404003A040500350405003000
:1010F0000404002C04050027040400230405001E3A
:101100000404001A04040016040500110404000D70
:10111000040400090405000404040000040400FCA5
:10112000030400F8030400F4030400F0030400ECDB
:10113000030400E8030400E4030400E0030400DC0B
:10114000030400D8030400D4030400D0030400CC3B
:10115000030400C8030300C503030024F404D920DA
:101160001BC40C5C0E9804C4095F0265077101F48E
:1011700005F900FB04B30048048700C10369005867
:1011800003550003034500BE023A008402310053B8
:10119000022A002902250004022000E4011C00C8E4
:1011A000011900AF011700980114008401130071A8
:1011B0000110006101100051010E0043010D0036C5
:1011C000010B002B010B0020010B00150109000C85
:1011D00001090003010800FB000800F3000800EB10
:1011E000000700E4000600DE000600D8000600D27A
:1011F000000600CC000500C7000500C2000500BDC8
:10120000000400B9000400B5000400B1000400AD02
:10121000000400A9000400A5000300A20003009F31
:101220000004009B00030098000300950002009357
:10123000000300900003008D0002008B0003008873
:101240000002008600020084000300810002007F8B
:101250000002007D0002007B00020079000200779E
:1012600000010076000200740002007200010071AB
:101270000002006F0002006D0001006C0002006AB5
:1012800000010069000200670001006600010065BE
:1012900000010064000200620001006100010060C2
:1012A0000001005F0002005D0001005C0001005BC6
:1012B0000001005A000100590001005800010057C8
:1012C00000010056000100550001005400010053C8
:1012D00000000053000100520001005100010050C5
:1012E0000001004F0001004E0000004E0001004DC3
:1012F0000001004C0001004B0000004B0001004ABF
:1013000000010049000100480000004800010047BA
:1013100000010046000000460001004500000045B5
:1013200000010044000100430000004300010042AE
:1013300000000042000100410000004100010040A7
:101340000001003F0000003F0001003E0000003EA1
:101350000001003D0000003D0001003C0000003C99
:101360000000003C0001003B0000003B0001003A8F
:101370000000003A00010039000000390001003887
:10138000000000380000003800010037000000377E
:101390000001003600000036000000360001003574
:1013A000000000350000003500010034000000346A
:1013B000000000340001003300000033000000335F
:1013C0000001003200000032000000320001003154
:1013D000000000310000003100010030000000304A
:1013E000000000300001002F0000002F0000002F3F
:1013F0000000002F0001002E0000002E0000002E33
:101400000001002D0000002D0000002D0000002D27
:101410000001002C0000002C0000002C0000002C1B
:101420000001002B0000002B0000002B0000002B0F
:101430000001002A0000002A0000002A0000002A03
:1014400000010029000000290000002900000029F7
:1014500000000029000100280000002800000028EA
:1014600000000028000000280001002700000027DD
:1014700000000027000000270000002700010026D0
:1014800000000026000000260000002600000026C4
:1014900000010025000000250000002500000025B7
:1014A00000000025000000250001002400000024A9
:1014B000000000240000002400000024000100239C
:1014C0000000002300000023000000230000002390
:1014D0000000002300000023000100220000002281
:1014E0000000002200000022000000220000002274
:1014F0000001002100000021000000210000002167
:101500000000002100000021000000210001002057
:10151000000000200000002000000020000000204B
:101520000000002000000020000000200001001F3B
:101530000000001F0000001F0000001F0000001F2F
:101540000000001F0000001F0001001E0000001E20
:101550000000001E0000001E000000232C0000B848
:10156000220000561800003A0F0000B8080000B131
:10157000040000710200003E010000696E206D6FE2
:1015800076655F746F282920666565645F76616C97
:10159000756520666F722058593A002C2065793D98
:1015A0000029202D3E202865783D002C2073793DB0
:1015B0000020436F6E6E656374696E67207769748F
:1015C0006820766572746963616C206C696E652051
:1015D0002873783D002C2065793D0029202D3E2080
:1015E0002865783D002C2073793D0020436F6E6E96
:1015F000656374696E67207769746820686F7269C3
:101600007A6F6E74616C206C696E65202873783D0A
:10161000003F53706563696669656420582C5920E2
:10162000636F6F7264696E617465206F7574206F8B
:101630006620626F756E64732E0A003F285229651A
:10164000706561742076616C7565206E6F742070B2
:101650006C61757369626C653B206D757374206293
:1016600065206174206C6561737420312E0A003F1F
:101670002852296570656174206D757374206265E8
:1016800020737065636966696564207768656E209C
:101690006E6F74207573696E6720616E204C4344D1
:1016A0002E0A003F537065636966696564206E6F3A
:1016B0007A7A6C652074656D706572617475726597
:1016C000206E6F7420706C61757369626C652E0A90
:1016D000003F5370656369666965642066696C6183
:1016E0006D656E742073697A65206E6F7420706CFE
:1016F00061757369626C652E0A003F53706563699A
:1017000066696564207072696D65206C656E6774CA
:1017100068206E6F7420706C61757369626C652EE1
:101720000A003F5072696D65206C656E67746820B1
:101730006D75737420626520737065636966696591
:1017400064207768656E206E6F74207573696E67AC
:1017500020616E204C43442E0A003F53706563693C
:1017600066696564206E6F7A7A6C652073697A6544
:10177000206E6F7420706C61757369626C652E0ADF
:10178000003F5370656369666965642052657472D1
:10179000616374696F6E204D756C7469706C6965F6
:1017A00072206E6F7420706C61757369626C652E47
:1017B0000A003F52657472616374696F6E204D75E3
:1017C0006C7469706C696572206D757374206265E4
:1017D000207370656369666965642E0A003F537003
:1017E00065636966696564206C6179657220686506
:1017F00069676874206E6F7420706C6175736962BC
:101800006C652E0A003F53706563696669656420E4
:101810006265642074656D706572617475726520AF
:101820006E6F7420706C61757369626C652028340A
:10183000302D31343043292E0A0047323620636F71
:101840006D6D616E6420737461727465642E2057CF
:10185000616974696E6720666F722068656174657E
:10186000722873292E0A00024A3135004A313200AB
:101870004A3137002020506C616E6E657242756689
:1018800066657242797465733A2000204672656518
:10189000204D656D6F72793A2000436F6D70696CF1
:1018A00065643A204A616E20313020323031390A85
:1018B00000207C20417574686F723A20286461763C
:1018C000696472616D69726F2C20666F7220416E5F
:1018D000796375626963206933204D656761290A00
:1018E00000323031392D30312D313000204C6173D0
:1018F0007420557064617465643A2000312E312E75
:10190000390A004D61726C696E0020536F667477FE
:101910006172652052657365740A002057617463B3
:1019200068646F672052657365740A002042726FA5
:10193000776E206F75742052657365740A002045B8
:10194000787465726E616C2052657365740A00501C
:101950006F77657255700A0073746172740A004D76
:101960003234004D3233202573006175746F256960
:101970002E67006572726F722077726974696E6784
:1019800020746F2066696C650A00205A3A0020595D
:101990003A0020583A00656E6473746F7073206863
:1019A00069743A2000446F6E6520736176696E67D2
:1019B0002066696C652E0A004D32390020746F6F05
:1019C000206C6F6E6720657874727573696F6E2016
:1019D00070726576656E7465640A0020636F6C646E
:1019E00020657874727573696F6E207072657665A4
:1019F0006E7465640A006F70656E206661696C655F
:101A0000642C2046696C653A200043616E6E6F74E9
:101A1000206F70656E2073756264697220004A30B1
:101A200035004A3233004739310A4731205A2D31C7
:101A30003020463234300A47393000534420636145
:101A40007264206F6B0A006F70656E526F6F742046
:101A50006661696C65640A00766F6C756D652E69E8
:101A60006E6974206661696C65640A004572726F04
:101A7000723A00534420696E6974206661696C0A89
:101A8000006563686F3A00454550524F4D206461D0
:101A9000746173697A65206572726F722E0A00290B
:101AA0000A002062797465733B20637263200053DF
:101AB000657474696E67732053746F72656420284F
:101AC00000290A002062797465733B2063726320E9
:101AD000002073746F7265642073657474696E6737
:101AE0007320726574726965766564202800202809
:101AF00063616C63756C6174656429210A0020213F
:101B00003D2000454550524F4D20435243206D69C2
:101B1000736D61746368202D202873746F7265641F
:101B20002920002053697A653A2000496E6465785F
:101B30003A2000204D61726C696E3D563535290A98
:101B40000028454550524F4D3D00454550524F4DA0
:101B50002076657273696F6E206D69736D61746351
:101B60006820001000C90210012C01400122017000
:101B7000011801B0010E01F00104015002FA00B099
:101B800002F0003003E600D003DC009004D20070C5
:101B900005C800A006BE000008B400B009AA00D025
:101BA0000BA000600E960060118C000015820020D2
:101BB000197800C01D6E00A0226400B0275A009062
:101BC0002C500000314600E0343C001038320090C8
:101BD0003A2800603C1E00A03D1400803E0A002010
:101BE0003F00002CFFFFFFFFFF0001010101016228
:101BF00065640A002C2073797374656D2073746FAB
:101C00007070656421204865617465725F49443A6B
:101C100020004265642068656174696E67206661B2
:101C2000696C65640048656174696E672066616906
:101C30006C65640045312048656174696E67206693
:101C400061696C65640048656174696E67206661EE
:101C5000696C65640070012C0190012701B00122BC
:101C600001C0011D01F00118011002130130020E24
:101C7000016002090190020401C002FF000003FAA2
:101C8000004003F5008003F000D003EB002004E6E1
:101C9000007004E100E004DC004005D700C005D27C
:101CA000004006CD00D006C8008007C3003008BE43
:101CB00000F008B900C009B400B00AAF00B00BAA28
:101CC00000D00CA500000EA000500F9B00C0109685
:101CD000005012910000148C00C0158700B01782CC
:101CE00000B0197D00D01B7800001E730040206EEC
:101CF0000090226900F024640040275F0090295A78
:101D000000E02B5500102E500020304B00103246C2
:101D100000E033410090353C001037370070383216
:101D200000A0392D00B03A2800A03B2300603C1EE3
:101D300000103D1900903D1400103E0F00703E0A47
:101D400000C03E0500003F0000403FFBFF803FF623
:101D5000FFC03FF1FF453120544845524D414C20D2
:101D600052554E415741590042454420544845522E
:101D70004D414C2052554E415741590054686572AF
:101D80006D616C2052756E61776179004531204537
:101D900072723A204D415854454D50004572723A86
:101DA000204D415854454D5020424544004D415826
:101DB00054454D50207472696767657265640045CB
:101DC00031204572723A204D494E54454D500045E0
:101DD00072723A204D494E54454D502042454400C0
:101DE0004D494E54454D5020747269676765726560
:101DF00064004D383420582059205A204500202FA7
:101E0000002042403A0020403A00256973002569CD
:101E10006D20256973002569682025696D20256975
:101E20007300256964202569682025696D2025696E
:101E30007300256979202569642025696820256952
:101E40006D2025697300656E7175657565696E67CE
:101E50002022004B494C4C45442E20005072696EA4
:101E60007465722073746F7070656420647565208A
:101E7000746F206572726F72732E204669782074B9
:101E80006865206572726F7220616E64207573657B
:101E9000204D39393920746F207265737461727402
:101EA0002E202854656D70657261747572652069A5
:101EB000732072657365742E2053657420697420D5
:101EC00061667465722072657374617274696E679D
:101ED000290A004E6F20436865636B73756D207728
:101EE000697468206C696E65206E756D6265722C10
:101EF000204C617374204C696E653A20004E6F204F
:101F0000436865636B73756D2077697468206C69CD
:101F10006E65206E756D6265722C204C6173742045
:101F20004C696E653A2000636865636B73756D205C
:101F30006D69736D617463682C204C617374204CFF
:101F4000696E653A20004C696E65204E756D62655C
:101F500072206973206E6F74204C617374204C6919
:101F60006E65204E756D6265722B312C204C61734D
:101F700074204C696E653A20004D313130004D338C
:101F8000310053442072656164206572726F720A79
:101F900000446F6E65207072696E74696E672066AA
:101FA000696C650A0020496E76616C696420657809
:101FB00074727564657220000000A0C0000000000B
:101FC00000000000000057430000574300004D434D
:101FD000486F6D696E67206661696C656400206E8C
:101FE0006F7420656E74657265642E0A0046696CB4
:101FF000652064656C657465643A0044656C65745D
:10200000696F6E206661696C65642C2046696C6539
:102010003A200050726F7465637465642050696E75
:102020000A0046696C616D656E7420757365643A6B
:10203000200053746174733A20002C204C6F6E673B
:10204000657374206A6F623A2000546F74616C206B
:1020500074696D653A200053746174733A20002CE2
:10206000204661696C65643A20002C2046696E69DF
:10207000736865643A20005072696E74733A200088
:1020800053746174733A20004A3036004A30340089
:102090004A30370020573A004A3038004A30390079
:1020A00020573A00205A3A0020593A0020436F75D1
:1020B0006E7420583A0020453A00205A3A002059C0
:1020C0003A00583A003A004361703A00205A002022
:1020D0005900580020204D61783A2000205A0020F5
:1020E0005900580020204D696E3A20004F6E2000A4
:1020F0004F666600536F667420656E6473746F700C
:10210000733A20004B64200023646566696E652085
:1021100044454641554C545F004B6920002364659B
:1021200066696E652044454641554C545F004B70CE
:10213000200023646566696E652044454641554C20
:10214000545F00504944204175746F74756E65206A
:1021500066696E69736865642120507574207468BF
:1021600065206C617374204B702C204B6920616E6C
:1021700064204B6420636F6E7374616E74732066A9
:10218000726F6D2062656C6F7720696E746F20438B
:102190006F6E66696775726174696F6E2E680A008A
:1021A000504944204175746F74756E65206661698D
:1021B0006C6564212074696D656F75740A00453122
:1021C00020544845524D414C2052554E415741599B
:1021D0000042454420544845524D414C2052554EF2
:1021E0004157415900546865726D616C2052756E9B
:1021F000617761790045312048656174696E6720B7
:102200006661696C65640042656420686561746933
:102210006E67206661696C65640048656174696E0B
:1022200067206661696C656400504944204175749B
:102230006F74756E65206661696C656421205465F4
:102240006D706572617475726520746F6F20686956
:1022500067680A00204B643A2000204B693A20004E
:10226000204B703A20000A20436C6173736963202D
:10227000504944200A002054753A2000204B753AFA
:102280002000206D61783A2000206D696E3A2000B0
:1022900020643A200020626961733A20005049446A
:1022A000204175746F74756E65206661696C656434
:1022B0002120426164206578747275646572206EB5
:1022C000756D6265720A00504944204175746F74DF
:1022D000756E652073746172740A004F66660A0039
:1022E00046616465204865696768742000426564DA
:1022F000204C6576656C696E6720004661696C6587
:102300006420746F20656E61626C65204265642094
:102310004C6576656C696E670A004D65736820428E
:102320006564204C6576656C20646174613A0A00CE
:102330004D65736820706F696E742063616E6E6F97
:1023400074206265207265736F6C7665640A004D57
:1023500034323120696E636F72726563742070610C
:1023600072616D657465722075736167650A007CC2
:102370003C3E5E2B3D3F2F5B5D3B2C2A225C006286
:102380007573793A2070617573656420666F722089
:10239000696E7075740A00627573793A20706175A0
:1023A00073656420666F7220757365720A006275CA
:1023B00073793A2070726F63657373696E670A0090
:1023C0004A3135004B494C4C45442E20004B494C7A
:1023D0004C20636175736564206279204B494C4CD5
:1023E00020627574746F6E2F70696E0A004B494CD1
:1023F0004C45442E20004B494C4C2063617573655D
:102400006420627920746F6F206D75636820696E37
:102410006163746976652074696D65202D2063752C
:102420007272656E7420636F6D6D616E643A200028
:102430004A3131005072696E7465722068616C7443
:1024400065642E206B696C6C28292063616C6C6557
:1024500064210A000000A0C000000000000000008D
:102460005761726E696E673A20486F6D696E6720BA
:1024700042756D702044697669736F72203C20311B
:102480000A000202040000A0400000A0400000007A
:102490004000005C430000574300004D43FFFFFF36
:1024A000FFFDFCFAF8F6F4F2F0EEECEAE9E7E5E31A
:1024B000E1E0DEDCDAD9D7D5D4D2D0CFCDCBCAC8D3
:1024C000C7C5C3C2C0BFBDBCBAB9B7B6B4B3B2B05A
:1024D000AFADACAAA9A8A6A5A4A2A1A09E9D9C9AB6
:1024E00099989795949392908F8E8D8B8A898887EF
:1024F0008684838281807F7E7D7B7A79787776750A
:1025000074737271706F6E6D6C6B6A696867666503
:1025100064636261605F5E5D5C5B5A5958585756F0
:10252000555453525150504F4E4D4C4B4A4A4948C6
:10253000474646454443424241403F3E3E3D3C3B88
:102540003B3A39383837363535343332323130303A
:102550002F2E2E2D2C2B2B2A2929282727262525DF
:1025600024232322212120201F1E1E1D1C1C1B1B77
:102570001A19191818171616151514131312121103
:1025800011100F0F0E0E0D0D0C0C0B0A0A09090885
:1025900008070706060505040403030202010000FC
:1025A000545249474745524544006F70656E003AA2
:1025B00020007A325F6D696E007A5F6D696E007916
:1025C0005F6D696E00785F6D696E005265706F7245
:1025D00074696E6720656E6473746F7020737461C4
:1025E0007475730A000A4D656173757265642070B5
:1025F0006F696E74733A0A005A206F666673657469
:102600003A20004E756D20582C593A20352C350A49
:102610000000000001000000010000800055555539
:10262000000000400033333300AAAA2A0049922454
:102630000000002000C7711C0099991900D14517AE
:1026400000555515003BB11300244912001111111A
:1026500000000010000F0F0F00E3380E0043790D4B
:1026600000CCCC0C00C3300C00E8A20B0064210BA2
:1026700000AAAA0A00703D0A009DD80900427B0901
:102680000092240900DCD308008888080010420862
:102690000000000800F0C107008787070075500799
:1026A00000711C07003EEB0600A1BC060069900605
:1026B0000066660600703E06006118060017F40505
:1026C0000074D105005BB00500B290050062720590
:1026D000005555050078390500B81E0500050505AB
:1026E000004EEC040087D40400A1BD040090A704B0
:1026F0000049920400C17D0400EE690400C756043D
:1027000000444404005C3204000821040041100429
:1027100000000004003FF00300F8E0030026D203AD
:1027200000C3C30300CCB503003AA803000A9B030F
:1027300000388E0300C08103009F750300D0690339
:1027400000505E03001D53030034480300913D0315
:10275000003333030016290300381F0300971503C5
:1027600000300C0300030303000BFA020049F102DE
:1027700000BAE802005CE002002DD802002DD00271
:102780000059C80200B0C0020031B90200DAB1023B
:1027900000AAAA0200A0A30200BC9C0200FA9502B3
:1027A000005C8F0200DF88020082820200457C020A
:1027B000002776020027700200436A02007C640250
:1027C00000D05E02003F590200C853020000002101
:1027D00000240027002A002D0030003300010100F2
:1027E00000040107010A0100002200250028002B37
:1027F000002E003100340002010000050108010B29
:1028000001000020002300260029002C002F0032A8
:102810000000010000030106010901050505050787
:102820000508080808020202020A0A08080404044B
:102830000401010101010101010303030303030377
:1028400003040707070C0C0C0C0C0C0C0C02020206
:102850000206060606060606060B0B0B0B0B0B0BF9
:102860000B01021020200808102040102040800298
:1028700001020108040201010204081020408080C6
:10288000402010080402018004020180402010084A
:102890000402010804020101020408102040800122
:1028A0000204081020408000000A0B02090C0D0EE3
:1028B0000807030401000000000000000000000001
:1028C0000000000000000000000000000000000008
:1028D00000000012111000000000000000000000C5
:1028E00000000000000000000000000000556E6BBA
:1028F0006E6F776E20636F6D6D616E643A2022009B
:102900002066697273740A005A0059005800486FB3
:102910006D652000000048420000484200008040F1
:102920000000000048617264636F64656420446560
:102930006661756C742053657474696E6773204C9E
:102940006F616465640A00B80B0000D00700003CAA
:10295000000000102700000000FA430000FA4300C6
:1029600000C040000070420000A0420000A04200F1
:1029700000C8433333B94220286D6D290020204D13
:10298000393030204B004C696E65617220416476AD
:10299000616E63653A0A0020440020490020204D02
:1029A00033303420500020440020490020204D3393
:1029B00030312050005049442073657474696E674B
:1029C000733A0A00205A0020204D36363600456EF4
:1029D0006473746F702061646A7573746D656E746E
:1029E0003A0A00205A00205900202047323920534B
:1029F00033205800205A0020204D3432302053001C
:102A00004D65736820426564204C6576656C696E1F
:102A1000673A0A00205A0020590020204D323036F3
:102A2000205800486F6D65206F66667365743A0ABA
:102A300000204500205A0020590020580020540052
:102A400020530020204D32303520510020453C6D70
:102A500061785F655F6A65726B3E0020583C6D610E
:102A6000785F785F6A65726B3E20593C6D61785F74
:102A7000795F6A65726B3E205A3C6D61785F7A5F60
:102A80006A65726B3E00416476616E6365643A20EC
:102A9000513C6D696E5F7365676D656E745F7469D7
:102AA0006D655F75733E20533C6D696E5F6665654D
:102AB00064726174653E20543C6D696E5F7472612E
:102AC00076656C5F66656564726174653E0020546E
:102AD0000020520020204D323034205000416363EA
:102AE000656C65726174696F6E2028756E697473A8
:102AF0002F7332293A20503C7072696E745F6163A3
:102B000063656C3E20523C726574726163745F61F0
:102B10006363656C3E20543C74726176656C5F61E2
:102B20006363656C3E0A00204500205A002059006E
:102B300020204D3230312058004D6178696D756D1F
:102B400020416363656C65726174696F6E202875DE
:102B50006E6974732F7332293A0A00204500205A97
:102B60000020590020204D3230332058004D61782C
:102B7000696D756D20666565647261746573202882
:102B8000756E6974732F73293A0A00204500205A24
:102B90000020590020204D393220580053746570B0
:102BA000732070657220756E69743A0A0020204D9A
:102BB0003230302044300A0020204D323030204462
:102BC000002044697361626C65640A0046696C6147
:102BD0006D656E742073657474696E67733A002056
:102BE00020473231202020203B00526573656E64FF
:102BF0003A20006F6B0020746F6F206C6F6E67203F
:102C0000657874727573696F6E2070726576656E23
:102C10007465640A0020636F6C6420657874727553
:102C200073696F6E2070726576656E7465640A00F4
:102C30004572726F722077726974696E6720746F63
:102C400020454550524F4D210A0057726974696EF4
:102C50006720746F2066696C653A20006F70656E3E
:102C6000206661696C65642C2046696C653A2000B9
:102C70006F70656E206661696C65642C2046696CB6
:102C8000653A200046696C652073656C6563746500
:102C9000640A002053697A653A200046696C652011
:102CA0006F70656E65643A20002066696C653A2035
:102CB00000646F696E67006672657368004E6F77B7
:102CC0002000454E4420535542524F5554494E45DD
:102CD0000A002220706F73002220706172656E748A
:102CE0003A2200535542524F5554494E45204341D4
:102CF0004C4C207461726765743A22004B494C4C0D
:102D000045442E2000747279696E6720746F2063C9
:102D1000616C6C207375622D67636F6465206669F2
:102D20006C6573207769746820746F6F206D616EB5
:102D300079206C6576656C732E204D4158206C654A
:102D400076656C2069733A005AE33BE511241FBE97
:102D5000CFEFD1E2DEBFCDBF00E00CBF14E0A0E0BA
:102D6000B2E0ECE3F4EE01E00BBF02C007900D927D
:102D7000A831B107D9F728E1A8E1B4E001C01D925C
:102D8000AE3FB207E1F716E1C5EAD6E100E006C0C2
:102D900021970109802FFE010E9476F1C43AD107E4
:102DA00080E00807A9F70E94A7DD0C940DF20C94AF
:102DB00000002F923F924F925F926F927F928F927C
:102DC0009F92AF92BF92CF92DF92EF92FF920F93BA
:102DD0001F93CF93DF93CDB7DEB7CA58D1090FB693
:102DE000F894DEBF0FBECDBF21E020935A10809132
:102DF0004B188D3411F40C94D721843511F40C94B4
:102E0000972E873411F00C94E32E809149189091FD
:102E10004A188A31910509F4BEC79CF484309105A3
:102E20003CF482309105B4F597FF2DC00C94D3216A
:102E30008430910509F4D2C1059709F40EC20C94AF
:102E4000D3218A32910511F40C94CA204CF48C31B0
:102E5000910509F4A4C74D9709F4A6C70C94D32192
:102E60008B35910511F40C9455218C35910511F495
:102E70000C9459218A35910511F00C94D3211092AC
:102E80002B040C94E52E8091270281110C94EA2EDC
:102E90000C94E52E20912702222311F40C94E52EA8
:102EA00011E0029709F010E00E94899119821A82BC
:102EB0001B821C821D821E821F82188682E50E9450
:102EC000E14C882309F43AC10E94614C4B015C013A
:102ED00020E030E0A9010E94FDE9882309F444C103
:102EE000C0904004D0904104E0904204F09043042C
:102EF000CCAADDAAEEAAFFAAC0904404D090450453
:102F0000E0904604F0904704C8AED9AEEAAEFBAEFE
:102F1000C0900D18D0900E18E0900F18F090101877
:102F2000CCAEDDAEEEAEFFAEC0901118D090121850
:102F3000E0901318F09014182496CCAEDDAEEEAEEF
:102F4000FFAE24972CAD3DAD4EAD5FAD6CA97DA914
:102F50008EA99FA90E94FDE981110BC0A7019601CE
:102F600068AD79AD8AAD9BAD0E94FDE9882309F477
:102F7000FBC020E030E0A901C501B4010E94FDE9D9
:102F8000881F8827881F181739F0C12CD12C80E89A
:102F9000E82E8FEBF82E06C0C12CD12C00E8E02ED5
:102FA0000FE3F02E2C96CCAEDDAEEEAEFFAE2C973E
:102FB0002CA93DA94EA95FA96CAD7DAD8EAD9FAD8D
:102FC0000E9479EE28966CAF7DAF8EAF9FAF2897A9
:102FD00028AD39AD4AAD5BAD24966CAD7DAD8EADFF
:102FE0009FAD24970E9479EE6B017C0128962CAD51
:102FF0003DAD4EAD5FAD2897CA01B9010E9462EAAE
:103000002B013C01A7019601C701B6010E9462EAAB
:103010009B01AC01C301B2010E947AEE0E94E5F06F
:103020002B013C0120E030E040E05FE30E9462EAD7
:1030300060966CAF7DAF8EAF9FAF6097A501940196
:10304000C501B4010E9462EA4B015C0160962CAD9F
:103050003DAD4EAD5FAD6097CA01B9010E9462EA15
:103060009B01AC01C501B4010E9479EE0E94E5F01C
:103070002C962CAD3DAD4EAD5FAD2C970E9462EA13
:103080004B015C01C701B6019058A30192010E9457
:1030900056EFA50194010E9462EA6B017C012CAD00
:1030A0003DAD4EAD5FAD6CA97DA98EA99FA90E94D3
:1030B0007AEE20E030E040E05FE30E9462EA9B01AC
:1030C000AC01C701B6010E947AEE2CA93DA94EA918
:1030D0005FA90E9479EE69837A838B839C8324960F
:1030E0002CAD3DAD4EAD5FAD249768AD79AD8AADE9
:1030F0009BAD0E947AEE20E030E040E05FE30E946A
:1031000062EA6B017C01A301920128966CAD7DAD52
:103110008EAD9FAD28970E9456EFA50194010E94A5
:1031200062EA9B01AC01C701B6010E947AEE28ADAC
:1031300039AD4AAD5BAD0E9479EE12C089E40E94C0
:10314000E14C882331F00E94614C69837A838B8340
:103150009C838AE40E94E14C882331F00E94614CF8
:103160006D837E838F83988720E030E0A901698199
:103170007A818B819C810E94FDE981110EC020E043
:1031800030E0A9016D817E818F8198850E94FDE9E3
:10319000811103C0ECE6FAE10DC0412FBE016F5F63
:1031A0007F4F8DE098E10E943FAF0C94E52E0E9486
:1031B000A78AF80184918F010F5F1F4F8111F7CF0C
:1031C000EDE1F2E084918F010F5F1F4F882311F42E
:1031D0000C94E52E0E94A78AF801F4CF80E50E94A6
:1031E000E14C882379F08091250490912604009782
:1031F00049F04AE050E060E070E00E947CE86B013A
:103200007C0103C0C12CD12C760183E50E94E14CE6
:10321000882361F00E94614C20E030E04AE754E4EA
:103220000E9462EA0E94C3EF6B017C010E94386A2F
:103230000E941F59C60ED71EE81EF91E0E941F5974
:10324000DC01CB018C199D09AE09BF09B7FD02C095
:103250000C94E52E0E94EAAAF1CF809127028823E0
:1032600011F40C94E52E0E94899189E40E94E14CAE
:10327000882329F00E94614C2B013C0103C0412CA2
:10328000512C32018AE40E94E14C882329F00E94EB
:10329000614C4B015C0103C0812C912C540180E5F1
:1032A0000E94E14C882329F00E94614C6B017C0153
:1032B00003C0C12CD12C760181E50E94E14C88230A
:1032C00039F00E94614C6CAB7DAB8EAB9FAB04C000
:1032D0001CAA1DAA1EAA1FAA20915910C657DF4F6B
:1032E0002883CA58D0406091020270910302072ED1
:1032F000000C880B990B0E9403EA20914202309146
:10330000430240914402509145020E9462EA2AE041
:1033100037ED43E25CE30E9462EA68AB79AB8AABCB
:103320009BAB4091400450914104609142047091E4
:10333000430448AF59AF6AAF7BAF9A01AB01C301F9
:10334000B2010E947AEEA1966CAF7DAF8EAF9FAFB7
:10335000A1974090440450904504609046047090BA
:103360004704A3019201C501B4010E947AEEA5961B
:103370006CAF7DAF8EAF9FAFA59720910D183091A8
:103380000E1840910F1850911018C701B6010E94F5
:103390007AEEA9966CAF7DAF8EAF9FAFA9972091C3
:1033A00011183091121840911318509114186CA9EB
:1033B0007DA98EA99FA90E947AEEAD966CAF7DAFD4
:1033C0008EAF9FAFAD97C8ACD9ACEAACFBACC982AD
:1033D000DA82EB82FC824D825E826F8278860E9466
:1033E0001F599B01AC0128533F4F4F4F5F4FC358AC
:1033F000DF4F288339834A835B83CD57D040BDECB0
:103400008B2EBCEC9B2EA92CBDE3BB2E25961FAEAC
:10341000259729961FAE29972D961FAE2D97619659
:103420001FAE61970E94C6810E941F598B019C01AB
:10343000C358DF4FC880D980EA80FB80CD57D04089
:103440000C191D092E093F0937FD10C09B01AC0165
:1034500028533F4F4F4F5F4FC358DF4F2883398367
:103460004A835B83CD57D0400E94EAAAA50194010C
:103470002596BFAD25972996AFAD29972D96FFAD1F
:103480002D976196EFAD61976B2F7A2F8F2F9E2F1F
:103490000E947AEE6CAB78AF8CAF21969FAF2197EC
:1034A00020E030E040E85FE30E94A0F0181644F40A
:1034B0001CAA18AE30E83CAF4FE321964FAF2197DE
:1034C00060910D1870910E1880910F18909110183E
:1034D000E1966CAF7DAF8EAF9FAFE19780914004D6
:1034E00090914104A0914204B0914304E5968CAFC1
:1034F0009DAFAEAFBFAFE59721969FAD21979F934C
:10350000ACADAF93B8ADBF93ECA9EF93E196ACAC83
:10351000BDACCEACDFACE197A996ECACFDAC0EAD8A
:103520001FADA997A1962CAD3DAD4EAD5FADA19756
:10353000E5966CAD7DAD8EAD9FADE5970E9479B5FA
:103540000F900F900F900F9062966FAF62976396F7
:103550007FAF639764968FAF649765969FAF6597CB
:10356000C0901118D0901218E0901318F090141811
:10357000E996CCAEDDAEEEAEFFAEE9972091440405
:10358000309145044091460450914704ED962CAF8C
:103590003DAF4EAF5FAFED9721963FAD21973F9383
:1035A0004CAD4F9358AD5F936CA96F93E996ACAC5B
:1035B000BDACCEACDFACE997AD96ECACFDAC0EADDE
:1035C0001FADAD97A5962CAD3DAD4EAD5FADA597AA
:1035D000ED966CAD7DAD8EAD9FADED970E9479B54A
:1035E0000F900F900F900F9066966FAF669767964B
:1035F0007FAF679768968FAF689769969FAF699717
:1036000089819A81AB81BC81CF57DF4F88839983B1
:10361000AA83BB83C158D040CD80DE80EF80F88480
:10362000CB57DF4FC882D982EA82FB82C558D0408F
:103630006A961FAE6A9725967FAD259729966FAD3E
:1036400029972D969FAD2D9761968FAD6197272F66
:10365000362F492F582FBCA9A8ADFCAD2196EFAD50
:1036600021976B2F7A2F8F2F9E2F0E9479EE2FE6B6
:1036700032E143E05BE30E94FDE987FD29C1259625
:103680007FAD259729966FAD29972D969FAD2D97E4
:1036900061968FAD6197272F362F492F582FBCA9E0
:1036A000A8ADFCAD2196EFAD21976B2F7A2F8F2F10
:1036B0009E2F0E947AEE20E030E040E05FE30E941F
:1036C00062EA662E972E882E792E9F938F937F9392
:1036D0006F93E196ACACBDACCEACDFACE197A996F4
:1036E000ECACFDAC0EAD1FADA997A1962CAD3DADD8
:1036F0004EAD5FADA197E5966CAD7DAD8EAD9FAD46
:10370000E5970E9479B50F900F900F900F906B96F0
:103710006FAF6B976C967FAF6C976D968FAF6D9711
:10372000C757DF4F9883C958D0407F928F929F929E
:103730006F92E996ACACBDACCEACDFACE997AD9680
:10374000ECACFDAC0EAD1FADAD97A5962CAD3DAD6F
:103750004EAD5FADA597ED966CAD7DAD8EAD9FADD9
:10376000ED970E9479B50F900F900F900F90162F44
:10377000072FB82EA92E66962FAD669767963FAD98
:10378000679768964FAD689769965FAD6997CB5715
:10379000DF4F688179818A819B81C558D0400E9422
:1037A0007AEE20E030E040E05FE30E9462EA1B0135
:1037B0002C0162962FAD629763963FAD6397649636
:1037C0004FAD649765965FAD6597CF57DF4F6881C2
:1037D00079818A819B81C158D0400E947AEE20E095
:1037E00030E040E05FE30E9462EA9B01AC016B962F
:1037F0006FAD6B976C967FAD6C976D968FAD6D9737
:10380000C757DF4F9881C958D0400E9479EE6B01AD
:103810007C0120E030E0A9010E94A0F087FF04C0F5
:10382000F7FAF094F7F8F094A2019101612F702F4C
:103830008B2D9A2D0E9479EE1B012C0120E030E0A7
:10384000A9010E94A0F087FF04C057FA509457F8CE
:103850005094A2019101C701B6010E947AEE2DECAD
:103860003CEC4CEC5DE30E94FDE918168CF5669685
:103870001FAF669767960FAF67976896BFAE68975A
:103880006996AFAE69976B96DFAC6B976296DFAEC9
:1038900062976C96EFAC6C976396EFAE63976D96FC
:1038A000FFAC6D976496FFAE6497C757DF4F2881D2
:1038B000C958D04065962FAF65976CAA98AE8CAE6C
:1038C00021967FAE219731E06A963FAF6A97B3CEDB
:1038D0006A964FAD6A97411144C125967FAD2597F1
:1038E00029966FAD29972D969FAD2D9761968FAD37
:1038F0006197272F362F492F582FBCA9A8ADFCADB3
:103900002196EFAD21976B2F7A2F8F2F9E2F0E943C
:1039100079EE6B017C012DEC3CEC4CEC5DE30E94FC
:10392000A0F018160CF41DC1A7019601C701B6013D
:103930000E947AEE2596EFAD25972996BFAD29977F
:103940002D96AFAD2D976196FFAD61972E2F3B2F32
:103950004A2F5F2F0E947AEE662E972E882E792EA0
:1039600020E030E040E85FE30E94A0F087FFF9C06C
:103970007F928F929F926F92E196ACACBDACCEAC31
:10398000DFACE197A996ECACFDAC0EAD1FADA997ED
:10399000A1962CAD3DAD4EAD5FADA197E5966CAD5A
:1039A0007DAD8EAD9FADE5970E9479B50F900F90DC
:1039B0000F900F906A966FAF6A976B967FAF6B9779
:1039C0006C968FAF6C976D969FAF6D977F928F922D
:1039D0009F926F92E996ACACBDACCEACDFACE997F0
:1039E000AD96ECACFDAC0EAD1FADAD97A5962CAD74
:1039F0003DAD4EAD5FADA597ED966CAD7DAD8EAD99
:103A00009FADED970E9479B50F900F900F900F909A
:103A1000162F072FB82EA92E262F372F482F592FB4
:103A2000CB57DF4F688179818A819B81C558D0400F
:103A30000E947AEE20E030E040E05FE30E9462EA1C
:103A40006B017C016A962FAD6A976B963FAD6B97C1
:103A50006C964FAD6C976D965FAD6D97CF57DF4FFE
:103A6000688179818A819B81C158D0400E947AEE19
:103A700020E030E040E05FE30E9462EA9B01AC019D
:103A800062966FAD629763967FAD639764968FADD4
:103A9000649765969FAD65970E9479EE1B012C0196
:103AA00020E030E0A9010E94A0F087FF04C057FA8F
:103AB000509457F85094A701960166966FAD66979B
:103AC00067967FAD679768968FAD689769969FAD4B
:103AD00069970E9479EE6B017C0120E030E0A9013A
:103AE0000E94A0F087FF04C0F7FAF094F7F8F09472
:103AF000A2019101C701B6010E947AEE2DEC3CECC7
:103B00004CEC5DE30E94A0F018165CF166961FAFC6
:103B1000669767960FAF67976896BFAE6897699686
:103B2000AFAE69976A965FAD6A9762965FAF62972C
:103B30006B966FAD6B9763966FAF63976C967FAD27
:103B40006C9764967FAF64976D968FAD6D97659611
:103B50008FAF65976CAA98AE8CAE21967FAE2197F9
:103B6000BCCE25967FAD259729966FAD29972D96CA
:103B70009FAD2D9761968FAD6197272F362F492FD7
:103B8000582FBCA9A8ADFCAD2196EFAD21976B2FA6
:103B90007A2F8F2F9E2F0E9479EE4B015C01629647
:103BA0008FAD629763969FAD63976496AFAD649750
:103BB0006596BFAD659789839A83AB83BC83669610
:103BC0008FAD669767969FAD67976896AFAD68971C
:103BD0006996BFAD69978D839E83AF83B8877CA9B3
:103BE00068AD9CAD21968FAD2197272F362F492F99
:103BF000582F60E070E080E89FE30E9479EE6B014F
:103C00007C01209148043091490440914A0450912C
:103C10004B040E9462EA2B013C012091151830915F
:103C200016184091171850911818BCA9A8ADFCADF2
:103C30002196EFAD21976B2F7A2F8F2F9E2F0E9409
:103C400062EA9B01AC01C301B2010E947AEE69876E
:103C50007A878B879C8720914C0430914D0440914A
:103C60004E0450914F04C701B6010E9462EA6B01F5
:103C70007C012091191830911A1840911B1850910D
:103C80001C18BCA9A8ADFCAD2196EFAD21976B2FF8
:103C90007A2F8F2F9E2F0E9462EA9B01AC01C701F1
:103CA000B6010E947AEE6D877E878F87988BCE0152
:103CB00001960E946BCD1CA61DA61EA61FA689817B
:103CC0009A81AB81BC8188A399A3AAA3BBA38D8150
:103CD0009E81AF81B8858CA39DA3AEA3BFA3898528
:103CE0009A85AB85BC8588A799A7AAA7BBA7AE0173
:103CF000485D5F4FBE016C5D7F4FCE0180960E9494
:103D000014BFDE019C966D01C657DF4FE880CA588C
:103D1000D0408E01005D1F4F9E01235F3F4FAE01DB
:103D2000485D5F4FBE016C5D7F4FCE0180960E9463
:103D3000145A882329F120E030E040E85FE3BCA971
:103D4000A8ADFCAD2196EFAD21976B2F7A2F8F2F69
:103D50009E2F0E94FDE987FF13C03CA925963FAF27
:103D6000259748AD29964FAF29975CAD2D965FAF4B
:103D70002D9721966FAD219761966FAF619752CBCA
:103D800080E1EDE0F8E1A0E4B4E001900D928A95C5
:103D9000E1F70C94E52E0E947E4E0C94E52E80E017
:103DA0000E9455930C94E52E83E50E94E14C8823F4
:103DB00021F10E94414C182F863070F0E5EEF2E0C0
:103DC00084918F010F5F1F4F882311F40C94E52E0F
:103DD0000E94A78AF801F4CF833009F44AC130F475
:103DE000813091F1823009F43FC008C0843009F479
:103DF0009FC1853009F4ACC101C010E00E94089356
:103E0000811103C0E5ECF2E013C08091DB17882339
:103E100019F063E173E002C067E173E08DEB92E0BB
:103E20000E9497B48AE00E94A78A0E944EBF96C162
:103E300084917F01BFEFEB1AFB0A882309F48EC13E
:103E40000E94A78AF701F4CF0E9401C010920102DC
:103E50001092000282EB92E090932C0780932B0744
:103E60000E94D38A0C94E52E809100029091010269
:103E700097FF0EC0E9E8F2E084918F010F5F1F4FBA
:103E8000882311F40C94E52E0E94A78AF801F4CF40
:103E90000097A1F48091520280932C0419821A8217
:103EA0001B821C8218A219A21AA21BA2BE016F5F5C
:103EB0007F4FCE0180960E9488C427C0815065E064
:103EC0000E9442F180FF03C024E0291B922F25E0CD
:103ED0009202F0011124E80FF11D87FDFA95EE0F13
:103EE000FF1FEE0FFF1FE25AF84E80914804909199
:103EF0004904A0914A04B0914B0480839183A2832A
:103F0000B38380912C04809352028091000290919F
:103F10000102893191050CF067C0109252029C0198
:103F20002F5F3F4F309301022093000265E00E9413
:103F300042F180FF03C024E0291B922F40914804E6
:103F40005091490460914A0470914B0448A359A3CD
:103F50006AA37BA319821A821B821C8244E084021A
:103F600090011124B9016F58764F4B01DB012D915F
:103F70003D914D915C91B4E09B02C0011124FC0184
:103F8000EB57F64F5F016081718182819381DE0181
:103F900011966D01E12CF12C00EA10E40E94B8C3E7
:103FA00019821A821B821C82B601CE0180960E9461
:103FB00088C4F50180819181A281B38180934004FE
:103FC00090934104A0934204B0934304F401808190
:103FD0009181A281B3818093440490934504A0937E
:103FE0004604B0934704BCC080E090E0A0EAB0E48F
:103FF0008093480490934904A0934A04B0934B04DF
:104000000E9449940E94386A8FEF9FEF90930102BB
:1040100080930002E5E7F2E084918F010F5F1F4F6C
:10402000882321F00E94A78AF801F6CF83E992E065
:104030009A83898304E610E019A308A3BE016F5F89
:104040007F4FCE0180960E94A3C58AEB92E09A83AF
:10405000898319A308A3BE016F5F7F4FCE018096AD
:104060000E94A3C581E00E94559381E00E94359390
:1040700077C088E50E94E14C8823A1F00E94314C72
:104080001FEF160F1530A8F0EEE5F2E084918F01D6
:104090000F5F1F4F882311F40C94E52E0E94A78A0E
:1040A000F801F4CF88E50E94A78A0E942BE50C94C2
:1040B000E52E89E50E94E14C8823A1F00E94314C55
:1040C0000FEF060F0530A8F0E7E4F2E084918F01CE
:1040D0000F5F1F4F882311F40C94E52E0E94A78ACE
:1040E000F801F4CF89E50E94A78A0E942BE50C9481
:1040F000E52E8AE50E94E14C882399F00E94614CEC
:1041000025E0129FF0011124E00FF11DEE0FFF1FBB
:10411000EE0FFF1FE25AF84E608371838283938310
:1041200035C08AE50E94A78A0E942BE50C94E52EF3
:104130008AE50E94E14C8823A1F30E94614C6093C0
:104140005A1770935B1780935C1790935D171EC08E
:1041500080E00E9435930E9401C018C01230B1F473
:1041600060910002709101026931710514F069E1FA
:1041700070E088E392E00E947EB469E170E083E33E
:1041800092E00E947EB48AE00E94A78A0E94339F38
:104190000C94E52E80912702882311F40C94E52ECF
:1041A00089E40E94E14CE82E882321F00E94314CE2
:1041B000062F01C000E08AE40E94E14CF82E88231B
:1041C00021F00E94314C162F01C010E0EE2011F0BA
:1041D000053020F4FF2081F0153070F0ECEFF2E0B4
:1041E00084918F010F5F1F4F882311F40C94E52EEB
:1041F0000E94A78AF801F4CF0E94ED4CEE2091F0C6
:1042000034E00302F0011124EB57F64F80819181D5
:10421000A281B38180930D1890930E18A0930F186C
:10422000B0931018FF2091F044E01402F001112423
:10423000EF58F64F80819181A281B381809311184C
:1042400090931218A0931318B093141880E50E944D
:10425000E14C882319F00E94524C03C080E50E9473
:10426000984C86E40E94E14C8823D9F00E94614C6E
:104270006B017C0120E030E0A9010E94A0F018163B
:1042800084F420E030E040E752E4C701B6010E9428
:1042900056EF6093420270934302809344029093DE
:1042A00045020E9402CE0C94E52E20932B040C9420
:1042B000E52E87E5282E82E0382E98E6E92E90E15B
:1042C000F92E60E474E07DAB6CAB28E1C22E24E0F3
:1042D000D22E00E010E0D1018D911D010E94E14C31
:1042E000882309F44BC00E94614C2B013C01133020
:1042F00049F0F60120813181428153810E9479EE9B
:104300002B013C01ACA9BDA92D913D914D915C9132
:10431000C301B2010E9479EE4B015C012DEB37E342
:1043200046E855EB0E94A0F087FD0AC02DEB37E36D
:1043300046E855E3C501B4010E94FDE91816F4F4FE
:10434000133051F440924C0450924D0460924E044C
:1043500070924F0401E012C0A5019401F701608141
:104360007181828193810E947AEED7016D937D9352
:104370008D939C931397812F0E94A0941F5FB4E0AC
:10438000EB0EF11CECA9FDA93496FDABECABF4E00F
:10439000CF0ED11C143009F09ECF002309F4F6CEC5
:1043A0000E9454C3F3CE0E94D7C50C94E52E809191
:1043B000491890914A188537910511F40C94E52E0F
:1043C0000CF0DAC08D34910509F4D3C30CF072C03F
:1043D0008B31910509F452C2ACF58631910509F48F
:1043E00001C20CF58231910509F440C584F441976E
:1043F00011F00C94942E5F988A9847988091080148
:10440000817080930601479812980C94E52E8431B0
:10441000910509F4A7C1459711F00C94942E0E94C0
:10442000A86B0C94E52E8831910509F4F7C10CF4C2
:10443000DFC18931910509F4FCC14A9709F410C222
:104440000C94942E8032910509F4BEC2FCF48D3197
:10445000910511F40C94E52E0CF4A8C28E3191054F
:1044600009F4AEC24F9711F00C94942E0E94168559
:1044700068A379A38AA39BA3BE016F5F7F4FCE0180
:1044800080960E94C589E1E8FAE1EAC2813391058C
:1044900009F431C32CF48A9709F4F8C20C94942ED1
:1044A0008B34910509F44CC38C34910509F44CC349
:1044B0000C94942E8A36910509F487C4B4F584359A
:1044C000910509F4D3C4E4F48135910509F4A9C434
:1044D0004CF48E34910511F00C94942E0E948C9023
:1044E0000C94E52E8235910509F4BDC48335910500
:1044F00011F00C94942E81E080932A040C94E52E04
:104500008C35910509F4FAC434F48535910509F424
:10451000DCC40C94942E8836910509F42EC3893698
:10452000910509F4F2C30C94942E8F36910509F489
:1045300060C384F48C36910509F4AEC30CF461C4F5
:104540008D36910509F423C48E36910509F43EC3D6
:104550000C94942E8137910509F4AAC30CF4A0C3DE
:104560008237910509F452C58337910511F00C94F7
:10457000942EE7EAF4E087C58E3221E0920711F429
:104580000C94D02C0CF071C08B3C910509F495C6AD
:10459000CCF58C38910509F4FEC3ACF4873791054E
:1045A00009F419C60CF4CAC58837910509F416C672
:1045B0008937910511F00C94942E10924C051092AD
:1045C0004B050C94E52E8E3B910509F4FAC334F4A7
:1045D0008B39910509F4B4C30C94942E883C910551
:1045E00009F402C6893C910511F00C94942EF7E56C
:1045F000EF2EF2E0FF2E02EB10E1A2ECCA2EA0E1BA
:10460000DA2E42C68C3D910511F40C94632B9CF478
:104610008D3C910509F4E2C60CF46BC68E3C910505
:1046200009F469C7833D910511F00C94942E0E9402
:104630001E9E0C94E52E823E910511F40C94DE2B07
:104640003CF48D3D910511F40C94702B0C94942E38
:104650008C3241E0940711F40C94072C8D32914078
:1046600011F40C94302C0C94942E853F61E0960745
:1046700011F40C94BD2DDCF58A39A1E09A0709F4F8
:1046800013C3BCF48033E1E09E0711F40C94272D92
:1046900014F40C94242D833621E0920709F45EC0B3
:1046A0008039914011F00C94942E0E94386A0C9439
:1046B000E52E853A41E0940711F40C94BA2D4CF4A0
:1046C000843A914011F00C94942E0E94FD9F0C941A
:1046D000E52E8C3A71E0970709F430C7843F91408A
:1046E00011F00C94942E0E94CD760C94E52E8A390C
:1046F000B2E09B0711F40C94FC2DB4F4873FF1E079
:104700009F0711F40C94C32D14F40C94C02D883F12
:1047100031E0930711F40C94CF2D8C30924011F4BA
:104720000C94F32D0C94942E8B3853E0950711F4D0
:104730000C94E52E3CF48438934011F40C94292E0B
:104740000C94942E803AA3E09A0709F47CC1873E2A
:10475000934011F40C94812E0C94942EECE6FAE123
:104760000C94A72DEAE2F3E084918F010F5F1F4FB5
:10477000882321F00E94A78AF801F6CF1092370C07
:104780008AEE99E00E9424A48BE1EAEEF9E0DE01D2
:10479000159601900D928A95E1F78091E809909124
:1047A000E9099C838B8385E692E09A83898340E0C4
:1047B00050E0BE016F5F7F4F80E090E00E94D96DB6
:1047C000CE0101960E9480AAEBE1F3E084918F0173
:1047D0000F5F1F4F882311F40C94E52E0E94A78AC7
:1047E000F801F4CF1092B9091092BA090C94E52E91
:1047F000E0914718F09148188081882329F0803291
:1048000009F410823196F8CF40E061E080914718BA
:10481000909148180E9432D90C94E52E8091BA09E3
:10482000882319F081E08093B9090E94B2B40C94F6
:10483000E52E1092B9098091630F813011F00C942C
:10484000E52E82E08093630F0E941F5960935F0FF3
:104850007093600F8093610F9093620F0C94E52E1C
:104860008091BA09882311F40C94E52E83E50E9407
:10487000E14C81110C94EF2E0C94E52E83E40E9400
:10488000984C882309F450C0E8E6F3E084918F0146
:104890000F5F1F4F882321F00E94A78AF801F6CFEF
:1048A0008091850B811103C0EBE3F3E012C0BE01E0
:1048B0006F5F7F4F82E89BE00E94ECA28E010F5F4A
:1048C0001F4FF80181918F01882349F10E94A78A27
:1048D000F8CF84918F010F5F1F4F882301F10E9451
:1048E000A78AF801F6CF0AE9C02E03E0D02EE12C0A
:1048F000F12C20E08091250790E00E2C02C09595C8
:1049000087950A94E2F780FDA4C1FFEFEF1AFF0A32
:1049100032E0C30ED11C45E0E416F10459F78AE0F9
:104920000E94A78A0C94E52E8091BA09882339F059
:104930008091B909882319F0E5E4F3E003C0E7E5C5
:10494000F3E028C084918F010F5F1F4F882321F06F
:104950000E94A78AF801F6CF6091330C7091340C55
:104960008091350C9091360C4AE00E94CA8D8FE2FE
:104970000E94A78A60912F0C7091300C8091310CAD
:104980009091320C4AE00E94CA8D8AE00E94A78A68
:104990000C94E52E84918F010F5F1F4F882311F433
:1049A0000C94E52E0E94A78AF801F4CF40E060E065
:1049B00080914718909148180E9432D90C94E52EA6
:1049C0000E941B970C94E52E8091B90981110E94D9
:1049D000386A8091BA09882311F40C94E52E80E599
:1049E0000E94E14C882319F00E94524C03C080E5DC
:1049F0000E94984C182F482F61E0809147189091A1
:104A000048180E9432D983E50E94E14C882381F046
:104A10000E94314CAB01BC014093330C5093340CD9
:104A20006093350C7093360C82E89BE00E94DDA108
:104A30008091BA09882319F081E08093B909111196
:104A40000C94E52EF2CE809147189091481821E001
:104A50002093B80940E060E00E9432D90C94E52E22
:104A600084918F010F5F1F4F882321F00E94A78A36
:104A7000F801F6CFBE016F5F7F4F87E793E00E949A
:104A800097B48AE00E94A78A0C94E52E83E50E94E1
:104A9000E14C882311F40C94E52E0E94414CE82E41
:104AA00080E50E94E14C882339F00E94414C182F88
:104AB00087FF03C00C94E52E1DE089E40E94E14CC1
:104AC000882351F00E94524C81110C94682FE2EF20
:104AD000F5E082E296E00AC089E40E94984CF4CFA7
:104AE00031968E179F0711F40C94682F249112139E
:104AF000F7CF0C943D2FF090240481E0F826F0923B
:104B00002404EFE8F3E084918F010F5F1F4F8823A7
:104B100021F00E94A78AF801F6CFFF2019F0E4E8FF
:104B2000F3E002C0E9E8F3E084918F010F5F1F4FCB
:104B3000882311F40C94E52E0E94A78AF801F4CF83
:104B40000E94B2B40C94E52E8091630F813011F075
:104B50000C94E52E82E08093630F0E941F596093AE
:104B60005F0F7093600F8093610F9093620F0C94AE
:104B7000E52E0E94F9B40C94E52E88E690E00E94A0
:104B8000E09481110C94E52E8091250783FF02C0EB
:104B90000C94E52E83E50E94E14C882399F00E9455
:104BA000614C0E94BEEFCB010E94467C0E94614C8A
:104BB00020E030E04AEA52E40E94FDE9181614F0C1
:104BC0000E94F9B40E9487B70C94E52E8EE40E94EF
:104BD000E14C882311F40C94E52E0E94314C609333
:104BE000F4187093F5188093F6189093F7180C94B6
:104BF000E52E83E50E94984C882359F083E50E94B6
:104C0000E14C882319F00E94414C01C080E0809360
:104C10002507E1E8FAE184918F010F5F1F4F8111B1
:104C200003C0E8EAF3E004C00E94A78AF801F3CFCA
:104C300084918F010F5F1F4F882321F00E94A78A64
:104C4000F801F6CF8091250781114DCEE4EAF3E01B
:104C500018C0BB24B394B20E222319F08CE20E9438
:104C6000A78AF60185919491FC0184918F010F5FD1
:104C70001F4F882321F00E94A78AF801F6CF2B2D21
:104C800044CE84918F010F5F1F4F882309F447CED4
:104C90000E94A78AF801F5CF109220020C94E52E0D
:104CA0008FEA93E00E94A3AA0E94AC980C94E52E90
:104CB00083E50E94E14C811103C0E1E8FAE10DC0F7
:104CC0000E94414C8D3320F480932B020C94E52EEE
:104CD0008CE380932B020C94E52E84918F010F5F5F
:104CE0001F4F882321F00E94A78AF801F6CF409138
:104CF0002B0250E060E070E088EB93E00E9444B447
:104D00008AE00E94A78A0C94E52E89E690E00E9432
:104D1000E094811111C0EFEBF3E084918F010F5FFC
:104D20001F4F882321F00E94A78AF801F6CF0E9426
:104D3000E07C8AE00E94A78A10925A100C947D2F82
:104D400083E50E94E14C882311F40C94E52E0E9427
:104D5000414C182F8D3308F01CE3109367100E940C
:104D60001F596B017C01212F30E0A8EEB3E00E94B7
:104D70006AEEC60ED71EE81EF91EC0926310D092CE
:104D80006410E0926510F09266100C94E52E0E947B
:104D90001F950C94E52E8091250783FF02C00C948B
:104DA000E52E83E50E94E14C882311F40C94E52E56
:104DB0000E94614C0E94BEEFCB010E94704E0C9489
:104DC000E52E0E94C08E0C94E52E80E50E94E14CF9
:104DD000811106C083E50E94E14C882359F005C08B
:104DE0000E94414C8111F1C7F5CF0E94314C6F3FB9
:104DF000710510F06FEF70E0709337046093360424
:104E0000E4C780E50E94E14C811105C0109237048F
:104E100010923604DAC70E94314C672B09F0D5C7CF
:104E2000F5CF0E94E67D0E94F8B9109237041092E7
:104E3000360400E010E062E370E080E090E00E9461
:104E40004DC70E94C6810F5F1F4F0331110599F7AF
:104E500062E370E080E090E00E944DC70E94C6814E
:104E60000E94972FB2C710922A04AFC783E50E9411
:104E7000E14C882399F00E94614C20E030E04AE741
:104E800054E40E9462EA0E94C3EF60932C02709384
:104E90002D0280932E0290932F0297C788E50E94DF
:104EA000984C8111ADC789E50E94984C8111A8C723
:104EB0008AE50E94984C8111A3C785E40E94984C12
:104EC00081119EC70E94F8B980C783E50E94984C63
:104ED000882309F47AC70E94614C20E030E04AE759
:104EE00054E40E9462EA0E94C3EF60935F107093E3
:104EF0006010809361109093621067C7B7E5CB2E66
:104F0000B2E0DB2E11EFE12E17E1F12E10E0D60119
:104F10008D916D010E94984C882309F46DC0133067
:104F200009F063C00E94614C4B015C0120E030E05D
:104F300040EA51E40E94FDE987FF4EC0A5019401BB
:104F40006091FD177091FE178091FF1790910018E6
:104F50000E9456EF2B013C019B01AC016091F406CD
:104F60007091F5068091F6069091F7060E9462EA2C
:104F70006093F4067093F5068093F6069093F70617
:104F8000A301920160911407709115078091160793
:104F9000909117070E9462EA6093140770931507B7
:104FA00080931607909317076091AE107091AF1021
:104FB0008091B0109091B1100E9401EAA30192017A
:104FC0000E9462EA0E94C3EF6093AE107093AF102C
:104FD0008093B0109093B1108092FD179092FE17BD
:104FE000A092FF17B092001807C00E94614CF70111
:104FF00060837183828393831F5FF4E0EF0EF11C63
:10500000143009F084CF0E9428B9DFC60E94386AA4
:1050100083E50E94E14C882309F4B8C80E94314C12
:105020006230710509F0B2C80E944FCD8BE50E9435
:10503000A78A6091DA187091DB188091DC18909142
:10504000DD1842E00E944F8E4091DE185091DF182B
:105050006091E0187091E11885EC93E00E9461B4D2
:105060004091E2185091E3186091E4187091E518AE
:1050700082EC93E00E9461B48DE50E94A78A8AE0E9
:105080000E94A78AA2C684918F010F5F1F4F8823B9
:1050900021F00E94A78AF801F6CF60E087E994E04A
:1050A0000E94FC9E61E080E994E00E94FC9E61E029
:1050B00085E894E00E94FC9E61E085E794E00E9410
:1050C000FC9E60E08CE694E00E94FC9E61E082E63B
:1050D00094E00E94FC9E60E088E594E00E94FC9EC3
:1050E00060E080E594E00E94FC9E61E082E494E050
:1050F0000E94FC9E60E084E394E00E94FC9E60E0DD
:1051000085E294E00E94FC9E60E087E194E00E94CA
:10511000FC9E60E081E094E00E94FC9E60E080EFF5
:1051200093E00E94FC9E60E08BED93E00E94FC9E69
:1051300061E088EC93E00E94FC9E47C6009147180E
:105140001091481883E0D12C40E08150E9F0D8015B
:105150009C91292F2B7F2134C1F711962C9121335B
:10516000A1F7913421F0953421F441E002C0DD240F
:10517000D39498012E5F3F4F89012F5F3F4FF80175
:1051800090819032C9F3E1CF442369F0E1E8FAE17C
:1051900084917F012FEFE21AF20A882321F00E9406
:1051A000A78AF701F5CFDD2069F0E0E8F5E084910A
:1051B0007F013FEFE31AF30A882321F00E94A78AB8
:1051C000F701F5CFD8018D918D01882309F4A7CB84
:1051D0000E94A78AF7CF0E94C0C0F7C581E08093E4
:1051E0004C0580934B05F1C588EC90E00E94E0945B
:1051F0008111EBC584E40E94984C882309F441C0D6
:105200000E94614C6B017C0111E020E030E0A901BB
:105210000E94FDE9811101C010E01093C21720E047
:1052200030E0A901C701B6010E94FDE9882349F1D8
:105230000E94614CE091860FB4E0EB9FF0011124D5
:10524000E953F84E608371838283938320E030E0DA
:10525000A9016091C7177091C8178091C9179091E3
:10526000CA170E94FDE981110CC080E090E0A0EE19
:10527000BFE38093C7179093C817A093C917B09343
:10528000CA170E9436BAA1C5F70181917F010E9419
:10529000984C882351F00E94614C0E94C3EFD801C2
:1052A0006D937D938D939C9313970C5F1F4FC01646
:1052B000D10651F70E94B7B788C5E7E5EE2EE2E0C8
:1052C000FE2E08E017E0F70181917F010E94984CC3
:1052D000882341F00E94614CD8016D937D938D939A
:1052E0009C9313970C5F1F4FB7E008311B0759F7CA
:1052F0006CC583E50E94E14C8823A1F00E94614CBB
:10530000609300077093010780930207909303074F
:105310006093FC067093FD068093FE069093FF0653
:1053200010E001C011E080E50E94E14C882359F0B3
:105330000E94614C609300077093010780930207FD
:105340009093030710E082E50E94E14C882359F016
:105350000E94614C609304077093050780930607D1
:105360009093070710E084E50E94E14C882359F0F0
:105370000E94614C6093FC067093FD068093FE06CC
:105380009093FF0622C5112309F41FC54091000721
:105390005091010760910207709103078AE895E038
:1053A0000E9461B44091040750910507609106077F
:1053B0007091070787E895E00E9461B44091FC0670
:1053C0005091FD066091FE067091FF0684E895E01D
:1053D0000E9461B48AE00E94A78AF7C481E50E9416
:1053E000984C8823C1F08091250490912604009761
:1053F00039F04AE050E060E070E00E947CE803C0D1
:1054000060E070E0CB0160931807709319078093F8
:105410001A0790931B0783E50E94984C882351F04C
:105420000E94614C609320077093210780932207AC
:105430009093230784E50E94984C882351F00E94A2
:10544000614C60931C0770931D0780931E07909317
:105450001F0788E50E94984C882351F00E94614CF8
:105460006093E8067093E9068093EA069093EB0652
:1054700089E50E94984C882351F00E94614C60930A
:10548000EC067093ED068093EE069093EF068AE5A6
:105490000E94984C8823F1F00E94614C6093F006C2
:1054A0007093F1068093F2069093F3062DEC3CEC9A
:1054B0004CEC5DE30E94FDE9181664F0EAE9F5E0C2
:1054C00084918F010F5F1F4F882321F00E94A78ACC
:1054D000F801F6CF85E40E94984C882309F475C43E
:1054E0000E94614C6093F4067093F5068093F60673
:1054F0009093F7066AC467E5C62E62E0D62E7DE477
:10550000E72E75E0F72E10E0F60181916F010E9401
:10551000984C882359F00E94614CD7016D937D937C
:105520008D939C931397812F0E94A0941F5FB4E0EA
:10553000EB0EF11C133041F70C94C6200E94A6C458
:10554000811143C404E514E2E0E4F4E0FDABECAB0C
:105550009E012F5F3F4F59015DE9852E54E2952E44
:105560001901F8016591759185919491ACA9BDA936
:10557000CD90DD90ED90FD90BDABACABA701960159
:105580000E9479EE2B013C01F101608371838283DB
:10559000938320E030E040EA51EC0E94A0F087FDC8
:1055A0000AC020E030E040EA51E4C301B2010E94A9
:1055B000FDE918162CF4F401849118160CF452C469
:1055C000D101CD90DD90ED90FD901D0120E030E007
:1055D00040EA51ECC701B6010E94A0F087FD0AC065
:1055E00020E030E040EA51E4C701B6010E94FDE945
:1055F00018164CF5ECE6FAE184918F010F5F1F4F0E
:10560000811103C0ECECF5E004C00E94A78AF80108
:10561000F3CF84918F010F5F1F4F882321F00E94E9
:10562000A78AF801F6CF88E290E099A388A388ECD6
:1056300090E09DA78CA7BE01605E7F4FCE018C9647
:105640000E94A3C5C2C30C5F1F4FBFEF8B1A9B0AFA
:10565000E4E200361E0709F084CF4DE4E42E45E075
:10566000F42E10E0F50181919191A191B1915F012A
:10567000F70181939193A193B1937F01812F0E94B0
:10568000A0941F5F133071F70E94339F83E992E06B
:105690009DA78CA704E610E019A308A3BE01645DD2
:1056A0007F4FCE0180960E94A3C58AEB92E09DA712
:1056B0008CA719A308A3BE01645D7F4FCE0180961D
:1056C0000E94A3C582C383E50E94E14C882309F4AC
:1056D0007CC30E94314C709303026093020275C335
:1056E0008DED90E00E94E09481116FC383E50E94EC
:1056F000E14C811103C0E1E8FAE13AC00091860F64
:1057000010E00E94314C000F111FF801E05CFD4FCA
:10571000718360838091860F90E07C01EE0CFF1C0A
:10572000EE0CFF1C87010F5D1D4F880F991FFC01B8
:10573000E05CFD4F60817181072E000C880B990B96
:105740000E9403EA2AE037ED43E25CE30E9462EA4A
:10575000F701ED53F84E20813181428153810E943F
:1057600062EAD8016D937D938D939C9313972DC31B
:1057700084918F010F5F1F4F882321F00E94A78A19
:10578000F801F6CF85E40E94A78A8091860F805D9C
:105790000E94A78AE091860FF0E0EE0FFF1FE05C09
:1057A000FD4F608171818AEE95E00E947EB485E2B2
:1057B0000E94A78A8AE00E94A78A07C380E50E9408
:1057C000984C882309F401C30E94314C6B017C0181
:1057D00083E50E94E14C882321F00E94314C8B012B
:1057E00002C00FEF1FEFC8010196039708F0EDC24A
:1057F000D7FCEBC28C2DE2EFF5E09491891709F408
:105800003CC33196B6E0E232FB07B9F739C383E512
:105810000E94E14C882319F00E94314C02C064E0E0
:1058200071E079A368A380E50E94E14C882339F0F8
:105830000E94314C6938E3E17E0730F402C068EE23
:1058400073E07A83698304C088E893E19A8389834B
:10585000BE01605E7F4FCE0101960E94A3C5B5C216
:1058600085E40E94E14C811110C080E50E94984CB3
:10587000882391F00E94614C6093740F7093750FB0
:105880008093760F9093770F07C00E94414C882336
:1058900061F3ECE6FAE171C089E40E94984C882338
:1058A00081F00E94614C2CEA35EC47E25EE30E94F5
:1058B00062EA6093700F7093710F8093720F9093F0
:1058C000730F84E40E94984C882381F00E94614CFD
:1058D0002CEA35EC47E25EE30E9456EF6093780FC6
:1058E0007093790F80937A0F90937B0FE1E8FAE140
:1058F00084918F010F5F1F4F882321F00E94A78A98
:10590000F801F6CF4091740F5091750F6091760FAA
:105910007091770F8AE296E00E9461B42CEA35EC30
:1059200047E25EE36091700F7091710F8091720F8A
:105930009091730F0E9456EFAB01BC0186E296E096
:105940000E9461B42CEA35EC47E25EE36091780F87
:105950007091790F80917A0F90917B0F0E9462EA8B
:10596000AB01BC0182E296E00E9461B48AE00E9431
:10597000A78A2BC20E94A78AF80184918F010F5F2A
:105980001F4F8111F7CFEEE2F6E084918F010F5F98
:105990001F4F882309F419C20E94A78AF801F5CF86
:1059A00083E50E94984C182F882371F00E94614C67
:1059B0000E94BEEF709326026093250221E0672BC0
:1059C00009F020E02093240780E50E94984C88236A
:1059D00059F02091250230912602232B11F00E94CC
:1059E000524C80932407F1C11111EFC1E1E8FAE1B3
:1059F00084918F010F5F1F4F882321F00E94A78A97
:105A0000F801F6CF80912407882319F06BE173E049
:105A100002C06EE173E085E596E00E9497B4609164
:105A200025027091260284E496E00E947EB4E0E4B0
:105A3000F6E084918F010F5F1F4F882309F4C5C1E1
:105A40000E94A78AF801F5CF0E94E998BEC180E5BF
:105A50000E94984C882351F00E94614C60936C0F17
:105A600070936D0F80936E0F90936F0F89E40E9477
:105A7000984C882381F00E94614C2CEA35EC47E277
:105A80005EE30E9462EA6093680F7093690F8093EF
:105A90006A0F90936B0F84E40E94984C882381F0E6
:105AA0000E94614C2CEA35EC47E25EE30E9456EF1F
:105AB0006093640F7093650F8093660F9093670FE8
:105AC000E1E8FAE184918F010F5F1F4F882321F0F5
:105AD0000E94A78AF801F6CF40916C0F50916D0F8C
:105AE00060916E0F70916F0F80E796E00E9461B435
:105AF0002CEA35EC47E25EE36091680F7091690F24
:105B000080916A0F90916B0F0E9456EFAB01BC0120
:105B10008CE696E00E9461B42CEA35EC47E25EE345
:105B20006091640F7091650F8091660F9091670F7F
:105B30000E9462EAAB01BC0188E696E00E9461B473
:105B40008AE00E94A78A41C10E94A78AF801849135
:105B50008F010F5F1F4F8111F7CFE4E7F6E08491CB
:105B60008F010F5F1F4F882309F42FC10E94A78A5E
:105B7000F801F5CF0E94C19728C10E94C17625C1C6
:105B80000E941CCC22C183E50E94984C882321F0FE
:105B90000E94524C91E089270E9487C716C181E07C
:105BA0008093470F0E94BD701092470F882309F41D
:105BB0000CC1E1E8FAE184918F010F5F1F4F811161
:105BC00003C0E3E8F6E004C00E94A78AF801F3CF1F
:105BD00084918F010F5F1F4F882309F4F6C00E9444
:105BE000A78AF801F5CF8091B909882309F4EDC09F
:105BF00081E08093BC09E9C08AE50E94E14C8111F3
:105C000003C0E1E9F6E00BC00E94614C60932518E7
:105C1000709326188093271890932818D6C08491E3
:105C20008F010F5F1F4F882321F00E94A78AF80180
:105C3000F6CF409125185091261860912718709141
:105C400028188EE896E00E9461B48AE00E94A78A34
:105C5000BCC08BE40E94E14C811103C0E1E8FAE191
:105C600036C08BE40E94E14C8823C1F00E94614C55
:105C70006B017C0120E030E0A9010E94A0F087FDCB
:105C80000AC020E030E040E251E4C701B6010E94C2
:105C9000FDE9181634F4E0EBF6E00EC0C12CD12C6F
:105CA00076010E94386AC092F806D092F906E09216
:105CB000FA06F092FB0689C084918F010F5F1F4F97
:105CC000882309F482C00E94A78AF801F5CF849145
:105CD0008F010F5F1F4F882321F00E94A78AF801D0
:105CE000F6CF4091F8065091F9066091FA0670914E
:105CF000FB068FEC96E00E9461B48AE00E94A78ABE
:105D000064C081E08093270283E50E94E14C8823F0
:105D100039F00E94524C811158C00E94F3D155C0F5
:105D200083E50E94984CF7CF0E94D7C54EC0F090F3
:105D300049180E94386A1091DB1780E00E94359361
:105D4000FF2029F1E1E8FAE184918F010F5F1F4FF5
:105D5000882321F00E94A78AF801F6CF84E50E94EB
:105D6000A78A6F2D70E080E090E04AE00E94CA8D23
:105D700080E20E94A78AECEEF6E084918F010F5F2B
:105D80001F4F882311F10E94A78AF801F6CF1092C5
:105D90005910812F0E943593E1E8FAE184918F0137
:105DA0000F5F1F4F882321F00E94A78AF801F6CFCA
:105DB0006091591070E08AED96E00E947EB48AE00E
:105DC0000E94A78A02C00E94D7C510925A100E9452
:105DD000D6D193C00E9489910E9402CEF6CF0E9434
:105DE000314CAB01BC014093330C5093340C6093A5
:105DF000350C7093360C82E89BE00E94DDA1E5CF64
:105E00000E94386A88E50E94984C882331F05F9A96
:105E1000809135048E7F8093350489E50E94984CEB
:105E2000882339F08A9A479A809135048D7F809330
:105E300035048AE50E94984C882361F0809108011E
:105E40008095817080930601479A809135048B7FFD
:105E50008093350485E40E94984C882309F4B5CFDB
:105E6000129AB3CFF7FAF094F7F8F094D101CD92EB
:105E7000DD92ED92FC921397A3CB0E9410E5A5CF83
:105E80000E94386ABC2C60E08C2D0E944AC60F3FED
:105E9000BFEF1B0759F48C2D0E94F4C531E020E0C0
:105EA000892B09F030E0032F122F05C001301105B6
:105EB00061F401E010E08B2D0E94F4C5801791077A
:105EC00009F483CF0E94EAAAF6CF00E010E0F3CFF6
:105ED00061E0812F0E944AC66E2D812F0E941CC650
:105EE000F12CB701812F0E9486C6193009F06DCFC1
:105EF000F0923704E092360468CFC657DF4F0FB6F2
:105F0000F894DEBF0FBECDBFDF91CF911F910F91EF
:105F1000FF90EF90DF90CF90BF90AF909F908F90C9
:105F20007F906F905F904F903F902F9008952F92A9
:105F30003F924F925F926F927F928F929F92AF9219
:105F4000BF92CF92DF92EF92FF920F931F93CF9366
:105F5000DF93CDB7DEB76F970FB6F894DEBF0FBEF5
:105F6000CDBFC0905004D0905104E0905204F09006
:105F7000530420E030E040EA50E4C701B6010E943B
:105F8000FDE987FD44C120E030E041E953E4C70169
:105F9000B6010E94A0F018160CF439C11092D60D6B
:105FA0001092D50D809109014091D40D042E000C62
:105FB000550B817021E0822790E04817590709F4BA
:105FC00033C080910901817028272093D40D81115D
:105FD0001BC00E94A86BEFE4FDE084918F01882331
:105FE00051F0082E000C990B0E94A36B0F5F1F4FFE
:105FF000F8018491F4CF8DE090E00E94A36B8AE0D9
:1060000090E00E94A36B10C0E3E5FDE084918F0156
:10601000882389F3082E000C990B0E94A36B0F5F55
:106020001F4FF8018491F4CF8091C70D833009F49C
:106030004CC02CF4882351F08130D9F09DC08430BD
:1060400009F43EC0853009F44DC096C08091B9096D
:10605000882309F491C081E08093C70D0E941F59E5
:106060006093CB0D7093CC0D8093CD0D9093CE0D9E
:1060700083C08091B90981117FC08091850B8823ED
:1060800021F082E08093C70D77C01092C70DEBE43A
:10609000FDE084918F01882351F0082E000C990BAC
:1060A0000E94A36B0F5F1F4FF8018491F4CF8DE026
:1060B00090E00E94A36B8AE090E00E94A36B5CC01A
:1060C0008091140E8823E9F257C08091B90981119B
:1060D00053C080913B0990913C09891B8F7009F452
:1060E000C1C04AC08091B909811146C080913B0965
:1060F00090913C09891B8F7009F4D6C03DC08DE09A
:1061000090E00E94A36B8AE090E00E94A36B109243
:10611000C70DC0904804D0904904E0904A04F09024
:106120004B0420E030E048E453E4C701B6010E948C
:10613000A0F018160CF0C9C08BE29DE090932C07DC
:1061400080932B070E94D38A80E29DE090932C07D6
:1061500080932B070E94D38A8CE19DE090932C07BB
:1061600080932B070E94D38A80EF9CE090932C07AA
:1061700080932B070E94D38A8091BC0D9091BD0D16
:1061800003974CF57AE1272E79E0372EE0E68E2E44
:10619000EAEE9E2EA12CB12C82E29FE00E94B34B2E
:1061A00018161906C4F48091BC0D9091BD0D04978A
:1061B00094F482E29FE00E94774B8093C20DE091BD
:1061C000C30DF091C40D8A3019F08D3009F0B7C0BD
:1061D000309709F0BDC08091BC0D9091BD0D009726
:1061E00011F40C946F3F01979093BD0D8093BC0DFB
:1061F0008091BE0D9091BF0D019664E070E00E9409
:1062000063F19093BF0D8093BE0D0C946F3F80910E
:10621000D50D9091D60D8136FAEE9F07E8F01092D9
:10622000D60D1092D50DE7E5FDE084918F0188230E
:1062300051F0082E000C990B0E94A36B0F5F1F4FAB
:10624000F8018491F4CF8DE090E00E94A36B8AE086
:1062500090E00E94A36BA6CE01969093D60D8093FA
:10626000D50DA0CE87E39DE090932C0780932B075C
:106270000E94D38A8091140E882311F082E001C01D
:1062800084E08093C70DE3E3FDE084918F018823D0
:1062900009F40DCF082E000C990B0E94A36B0F5F21
:1062A0001F4FF8018491F3CFEFE2FDE084918F015D
:1062B000882309F424CF082E000C990B0E94A36BAD
:1062C0000F5F1F4FF8018491F3CF20E030E04EE3E1
:1062D00053E4C701B6010E94FDE987FF13C088E1BE
:1062E0009DE090932C0780932B070E94D38A8CE02B
:1062F0009DE090932C0780932B070E94D38A88E01F
:106300009DE02CCF20E030E046E153E4C701B60128
:106310000E94FDE987FF28CF84E09DE090932C0741
:1063200080932B070E94D38A88EF9CE090932C07E0
:1063300080932B070E94D38A84EF9CE00FCF8A338F
:1063400009F446CFEF35F10514F40C94033D40CF2A
:106350008091C00D9091C10D20E6289F7001299F6A
:10636000F00C11248701045C134FE00FF11F108221
:1063700061E470E0C8010E94CAF1009711F40C9426
:10638000E73C9093C60D8093C50D801B910B8E0D3D
:106390009F1D60E070E0835C934F0E94FEE50E94C9
:1063A000BEEFCB01770FAA0BBB0B8232910510F029
:1063B0000C94E73CFC018827EE58FF4F8F4F0C945C
:1063C00076F1EBEEFCE084918F01882351F0082EEA
:1063D000000C990B0E94A36B0F5F1F4FF801849173
:1063E000F4CF20E030E040E05FE360915004709132
:1063F000510480915204909153041EC0E6EEFCE0DB
:1064000084918F01882351F0082E000C990B0E9473
:10641000A36B0F5F1F4FF8018491F4CF60913E048E
:1064200070913F04072E000C880B990B0E9403EA21
:1064300020E030E040E05FE30E947AEE0E94BEEF91
:10644000CB010E943A4E0E946EDB8DE090E00E94EC
:10645000A36B8AE090E00E94A36B0C94E73CE1EE12
:10646000FCE084918F01882351F0082E000C990BD9
:106470000E94A36B0F5F1F4FF8018491F4CF20E0BF
:1064800030E040E05FE360913A0470913B0480911A
:106490003C0490913D04D0CFECEDFCE084918F0161
:1064A000882351F0082E000C990B0E94A36B0F5FFC
:1064B0001F4FF8018491F4CF609138047091390432
:1064C000B1CF209136043091370444E6429FC00199
:1064D000439F900D11246FEF70E00E9463F18B01D8
:1064E0006536710510F004E610E0E7EDFCE08491FC
:1064F0007F01882359F0082E000C990B0E94A36B92
:10650000FFEFEF1AFF0AF7018491F3CFB80180E0A3
:1065100090E028C7E3EDFCE084918F01882351F0DF
:10652000082E000C990B0E94A36B0F5F1F4FF80100
:106530008491F4CF80E290E00E94A36BEFECFCE04A
:1065400084918F01882351F0082E000C990B0E9432
:10655000A36B0F5F1F4FF8018491F4CF609140044B
:106560007091410480914204909143040E946FDB3A
:1065700080E290E00E94A36BEBECFCE084918F0141
:10658000882351F0082E000C990B0E94A36B0F5F1B
:106590001F4FF8018491F4CF609144047091450439
:1065A00080914604909147040E946FDB80E290E066
:1065B0000E94A36BE7ECFCE084918F01882351F0EB
:1065C000082E000C990B0E94A36B0F5F1F4FF80160
:1065D0008491F4CF609148047091490480914A04F9
:1065E00090914B040E946FDB80E290E092C5809115
:1065F000B909882309F450C0E2ECFCE084918F01D2
:10660000882351F0082E000C990B0E94A36B0F5F9A
:106610001F4FF8018491F4CF8091BA09882359F172
:106620008091850B882329F180912F0C9091300C5B
:10663000A091310CB091320C0097A105B105C1F0C9
:10664000BC01CD016D597F4F8F4F9F4F24E630E045
:1066500040E050E00E941CEE6091330C7091340CCD
:106660008091350C9091360C0E941CEE822F01C057
:1066700080E090E0E6CEEEEBFCE084918F01882391
:1066800009F4E3CE082E000C990B0E94A36B0F5F58
:106690001F4FF8018491F3CFE6EBFCE084918F016A
:1066A000882309F4D2CE082E000C990B0E94A36B0C
:1066B0000F5F1F4FF8018491F3CFE1EBFCE0849171
:1066C0008F01882351F0082E000C990B0E94A36BB8
:1066D0000F5F1F4FF8018491F4CF8091CB0D909103
:1066E000CC0DA091CD0DB091CE0D892B8A2B8B2B8B
:1066F00009F477C00E941F59A50194010E941CEE65
:1067000069017A016091CB0D7091CC0D8091CD0D16
:106710009091CE0DA50194010E941CEE8601021BF2
:10672000130BC8016CE370E00E944FF1CB01992775
:10673000EAE0F0E0BF010E9463F1282FCB01BF0126
:106740000E9463F1805D80932D04205D20932E04D0
:1067500010922F048DE294E00E946EDB80E290E0C4
:106760000E94A36BEFEAFCE084917F01882359F03B
:10677000082E000C990B0E94A36BFFEFEF1AFF0A83
:10678000F7018491F3CF80E290E00E94A36BC801EF
:106790006CE370E00E944FF16AE070E00E9463F1E8
:1067A000605D60932D04805D80932E0410922F0411
:1067B0008DE294E00E946EDB80E290E00E94A36B89
:1067C000EDEAFCE084918F01882309F43ECE082E87
:1067D000000C990B0E94A36B0F5F1F4FF80184916F
:1067E000F3CF80E290E00E94A36BE5EAFCE08491A5
:1067F0008F01882309F429CE082E000C990B0E94E2
:10680000A36B0F5F1F4FF8018491F3CF1092F50D2A
:106810008091090180FF11C0E1EAFCE084918F01C1
:10682000882309F412CE082E000C990B0E94A36B4A
:106830000F5F1F4FF8018491F3CF83E50E9404DBC3
:10684000882341F00E941FDB0E94C3EF7093CA0DA2
:106850006093C90DEDE9FCE084918F01882351F02C
:10686000082E000C990B0E94A36B0F5F1F4FF801BD
:106870008491F4CF8DE090E00E94A36B8AE090E0D9
:106880000E94A36B8091130E882309F442C2809169
:10689000C90D9091CA0D8430910509F4C8C08830A3
:1068A000910509F47DC1892B09F0D9C3E1ECFAE027
:1068B00084918F01882351F0082E000C990B0E94BF
:1068C000A36B0F5F1F4FF8018491F4CF8DE090E030
:1068D0000E94A36B8AE090E00E94A36BE6EBFAE0D3
:1068E00084918F01882351F0082E000C990B0E948F
:1068F000A36B0F5F1F4FF8018491F4CF8DE090E000
:106900000E94A36B8AE090E00E94A36BEAEAFAE09F
:1069100084918F01882351F0082E000C990B0E945E
:10692000A36B0F5F1F4FF8018491F4CF8DE090E0CF
:106930000E94A36B8AE090E00E94A36BEEE9FAE06C
:1069400084918F01882351F0082E000C990B0E942E
:10695000A36B0F5F1F4FF8018491F4CF8DE090E09F
:106960000E94A36B8AE090E00E94A36BE0E9FAE04A
:1069700084918F01882351F0082E000C990B0E94FE
:10698000A36B0F5F1F4FF8018491F4CF8DE090E06F
:106990000E94A36B8AE090E00E94A36BE2E8FAE019
:1069A00084918F01882351F0082E000C990B0E94CE
:1069B000A36B0F5F1F4FF8018491F4CF8DE090E03F
:1069C0000E94A36B8AE090E00E94A36BE5E7FAE0E7
:1069D00084918F01882351F0082E000C990B0E949E
:1069E000A36B0F5F1F4FF8018491F4CF8DE090E00F
:1069F0000E94A36B8AE090E00E94A36BE8E6FAE0B5
:106A000084918F01882351F0082E000C990B0E946D
:106A1000A36B0F5F1F4FF8018491F4CF8DE090E0DE
:106A20000E94A36B8AE090E00E94A36B18C3EAE582
:106A3000FAE084918F01882351F0082E000C990B05
:106A40000E94A36B0F5F1F4FF8018491F4CF8DE07C
:106A500090E00E94A36B8AE090E00E94A36BECE4BC
:106A6000FAE084918F01882351F0082E000C990BD5
:106A70000E94A36B0F5F1F4FF8018491F4CF8DE04C
:106A800090E00E94A36B8AE090E00E94A36BE6E393
:106A9000FAE084918F01882351F0082E000C990BA5
:106AA0000E94A36B0F5F1F4FF8018491F4CF8DE01C
:106AB00090E00E94A36B8AE090E00E94A36BE0E26A
:106AC000FAE084918F01882351F0082E000C990B75
:106AD0000E94A36B0F5F1F4FF8018491F4CF8DE0EC
:106AE00090E00E94A36B8AE090E00E94A36BEEE02E
:106AF000FAE084918F01882351F0082E000C990B45
:106B00000E94A36B0F5F1F4FF8018491F4CF8DE0BB
:106B100090E00E94A36B8AE090E00E94A36BECEFF0
:106B2000F9E084918F01882351F0082E000C990B15
:106B30000E94A36B0F5F1F4FF8018491F4CF8DE08B
:106B400090E00E94A36B8AE090E00E94A36BEEEEBF
:106B5000F9E084918F01882351F0082E000C990BE5
:106B60000E94A36B0F5F1F4FF8018491F4CF8DE05B
:106B700090E00E94A36B8AE090E00E94A36BE0EE9D
:106B8000F9E084918F01882309F448CF082E000C86
:106B9000990B0E94A36B0F5F1F4FF8018491F3CFF5
:106BA000E9EDF9E084918F01882351F0082E000C63
:106BB000990B0E94A36B0F5F1F4FF8018491F4CFD4
:106BC0008DE090E00E94A36B8AE090E00E94A36BAE
:106BD000E2EDF9E084918F01882351F0082E000C3A
:106BE000990B0E94A36B0F5F1F4FF8018491F4CFA4
:106BF0008DE090E00E94A36B8AE090E00E94A36B7E
:106C0000EBEBF9E084918F01882351F0082E000C02
:106C1000990B0E94A36B0F5F1F4FF8018491F4CF73
:106C20008DE090E00E94A36B8AE090E00E94A36B4D
:106C3000E4EAF9E084918F01882351F0082E000CDA
:106C4000990B0E94A36B0F5F1F4FF8018491F4CF43
:106C50008DE090E00E94A36B8AE090E00E94A36B1D
:106C6000EDE8F9E084918F01882351F0082E000CA3
:106C7000990B0E94A36B0F5F1F4FF8018491F4CF13
:106C80008DE090E00E94A36B8AE090E00E94A36BED
:106C9000E6E7F9E084918F01882351F0082E000C7B
:106CA000990B0E94A36B0F5F1F4FF8018491F4CFE3
:106CB0008DE090E00E94A36B8AE090E00E94A36BBD
:106CC000E3E6F9E084918F01882351F0082E000C4F
:106CD000990B0E94A36B0F5F1F4FF8018491F4CFB3
:106CE0008DE090E00E94A36B8AE090E00E94A36B8D
:106CF000E0E5F9E084918F01882309F48FCE082E16
:106D0000000C990B0E94A36B0F5F1F4FF801849139
:106D1000F3CF8091BA09882309F478C181E0809388
:106D2000370C1092390C1092380C89E09AE00E94CE
:106D300024A48BE1E9E0FAE0DE01159601900D92C2
:106D40008A95E1F78091070A9091080A9C838B83CA
:106D500085E692E09A83898340E050E0BE016F5F50
:106D60007F4F80E090E00E94D96DCE0101960E9495
:106D700080AAC090380CD090390C0091C90D1091A8
:106D8000CA0DC601801B910B049720F06801F3E047
:106D9000CF0ED11C51E4452E59E0552E62E3662EEC
:106DA00069E0762EC016D10608F459C10115110507
:106DB00009F09DC06DEB79E089E09AE00E94ECA2B9
:106DC00062E273E08DEB99E00E94D5F1892B09F026
:106DD00048C0F201849141E4E42E49E0F42E882376
:106DE00059F0082E000C990B0E94A36BFFEFEF1ACD
:106DF000FF0AF7018491F3CF8DE090E00E94A36B2E
:106E00008AE090E00E94A36BF301849132E3E32EC9
:106E100039E0F32E882359F0082E000C990B0E94BC
:106E2000A36BFFEFEF1AFF0AF7018491F3CF8DE018
:106E300090E00E94A36B8AE090E00E94A36B80E048
:106E400090E00E9468DBE2E2F9E084917F012FEF9D
:106E5000E21AF20A882309F4D6C00E94A78AF70131
:106E6000F4CFEEE1F9E084917F01882359F0082EF8
:106E7000000C990B0E94A36BFFEFEF1AFF0AF701BA
:106E80008491F3CF8DE090E00E94A36B8AE090E0C4
:106E90000E94A36BF10184912AE1E22E29E0F22EF7
:106EA000882359F0082E000C990B0E94A36BFFEF6A
:106EB000EF1AFF0AF7018491F3CF8DE090E00E9472
:106EC000A36B8AE090E00E94A36B80E090E00E94B8
:106ED00068DBE5E1F9E084917F012FEFE21AF20A25
:106EE000882309F490C00E94A78AF701F4CF60E0DC
:106EF00070E0C80101970E949F6F8091BB098823B1
:106F000009F45AC0E3E1F9E084917F01882359F044
:106F1000082E000C990B0E94A36BFFEFEF1AFF0ADB
:106F2000F7018491F3CF8DEB99E00E946EDB8DE049
:106F300090E00E94A36B8AE090E00E94A36BE1E1E5
:106F4000F9E084917F01882359F0082E000C990BF9
:106F50000E94A36BFFEFEF1AFF0AF7018491F3CFB2
:106F60008AEC99E00E946EDB8DE090E00E94A36BBA
:106F70008AE090E00E94A36BC8010E9468DBEFE00A
:106F8000F9E084917F012FEFE21AF20A882321F0C1
:106F90000E94A78AF701F5CF9AECE92E99E0F92E25
:106FA000F70181917F01882319F00E94A78AF8CF09
:106FB0008AE00E94A78A27C08DEB99E00E946EDBD1
:106FC0008DE090E00E94A36B8AE090E00E94A36BAA
:106FD0008AEC99E00E946EDB8DE090E00E94A36B4A
:106FE0008AE090E00E94A36BC8010E9468DB8AECF3
:106FF000E82E89E0F82EF70181917F018823C1F204
:107000000E94A78AF8CF0F5F1F4FCCCEE0E0F9E0D7
:1070100084918F01882351F0082E000C990B0E9457
:10702000A36B0F5F1F4FF8018491F4CF8DE090E0C8
:107030000E94A36B8AE090E00E94A36BE1EFF8E06E
:1070400084918F01882309F4E9CC082E000C990B58
:107050000E94A36B0F5F1F4FF8018491F3CFE9E902
:10706000FCE084918F01882309F4EFC9082E000CFD
:10707000990B0E94A36B0F5F1F4FF8018491F3CF10
:107080008091B909882339F00E940B6DA0C48091CA
:10709000B9098823E9F00E944BC199C48091C70DBA
:1070A000823019F0833609F092C40E94EA6CE5E957
:1070B000FCE084918F01882309F4C7C9082E000CD5
:1070C000990B0E94A36B0F5F1F4FF8018491F3CFC0
:1070D0008091C70D833609F07AC4DDCF8CE89CE03F
:1070E0000E94A3AA80913B0990913C09891B8F7053
:1070F00009F06DC48091C70D823009F468C48336ED
:1071000009F099C464C48DE090E00E94A36B8AE00A
:1071100090E00E94A36B99C980913B0990913C0932
:10712000891B8F7009F053C48091C70D823009F418
:107130004EC4833609F44BC48091850B8111CFC4B2
:1071400046C483E50E9404DB811126C083E40E94CB
:1071500004DB882309F43BC480913B0990913C09EE
:10716000891B8F7009F033C420E030E040E251E425
:10717000609148047091490480914A0490914B04B5
:107180000E94FDE987FF08C089E79CE090932C07E7
:1071900080932B070E94D38A0E941FDB20E030E0FF
:1071A000A9010E94FDE987FD10C00E941FDB20E0BD
:1071B00030E849E853E40E94A0F018164CF00E9411
:1071C0001FDB0E94C3EFCB0105C080E090E002C04E
:1071D00083E191E00E94467CFAC383E50E9404DBD0
:1071E000882309F4F4C30E941FDB20E030E0A901EA
:1071F0000E94FDE987FD10C00E941FDB20E030E007
:1072000046E153E40E94A0F018164CF00E941FDBE8
:107210000E94C3EFCB0105C080E090E002C086E988
:1072200090E00E94704ED3C383E50E9404DB882364
:10723000D9F00E941FDB20E030E04FE753E40E94CA
:1072400062EA20E030E048EC52E40E9456EF0E94EF
:10725000C3EF6F3F710519F010F06FEF70E070939E
:10726000370460933604F1C88FEF90E090933704B1
:1072700080933604EAC880913B0990913C09891BB0
:107280008F7009F0E2C88091B9098111DEC80E94AF
:10729000AC985F9A809135048E7F809335048A9AEA
:1072A000479A809135048D7F809335048091080141
:1072B0008095817080930601479A809135048B7F79
:1072C00080933504129AC1C883E50E9404DB8823A9
:1072D00019F10E941FDB20E030E040E252E40E94FE
:1072E000FDE987FD0FC00E941FDB20E030EC49E77D
:1072F00054E40E94A0F0181644F00E941FDB0E9484
:10730000BEEF05C068E270E002C067EE73E0709304
:107310000302609302025BC3E3E7FCE084918F0108
:10732000882351F0082E000C990B0E94A36B0F5F6D
:107330001F4FF8018491F4CFC0900202D090030255
:107340000D2C000CEE08FF08F7FE0EC06DE282E285
:107350009FE00E942A4B66277727CB016C197D0995
:107360008E099F094AE003C04AE0C701B6010E94A6
:1073700028DB6BC880913B0990913C09891B8F7079
:1073800009F025C38091C70D823009F420C38336EC
:1073900009F0EBC21CC380913B0990913C09891B09
:1073A0008F7009F052C88091C70D823009F44DC822
:1073B000833609F0B6C349C880913B0990913C09D6
:1073C000891B8F7009F003C38091C70D823009F4C7
:1073D000FEC2833609F0FBC4FAC280913B0990914A
:1073E0003C09891B8F7009F0F2C28091C70D823071
:1073F00009F4EDC2833609F020C5E9C280913B094A
:1074000090913C09891B8F7009F0E1C28091C70DF2
:10741000823009F4DCC2833609F045C5D8C28091B8
:10742000F50D811103C00E94A86BC4C18E3271F5A5
:107430008091F60D8E3209F046C180915A0B882357
:1074400009F4B8C1815080935A0B882361F090E011
:1074500001974FE1489F9001499F300D1124C901C8
:107460008C5D954F02C086EE99E02BE1FC013496CD
:10747000A9E0BAE001900D922A95E1F7FC01828122
:1074800093819093080A8093070A94C18C3309F082
:107490001AC164E273E085EF9DE00E94D5F1892B6B
:1074A00021F481E08093130E85C163E373E085EFDF
:1074B0009DE00E94D5F1892B79F4EDECF8E0849100
:1074C0008F010F5F1F4F882321F00E94A78AF801C8
:1074D000F6CF80EB98E0E4C06AE473E085EF9DE0CE
:1074E0000E94D5F1892B79F4ECE8F8E084918F01C2
:1074F0000F5F1F4F882321F00E94A78AF801F6CF63
:1075000089E798E0CDC061E673E085EF9DE00E94D9
:10751000D5F1892B79F4EEE5F8E084918F010F5FC6
:107520001F4F882321F00E94A78AF801F6CF89E532
:1075300098E0B6C06FE673E085EF9DE00E94D5F15C
:10754000892B79F4E9E3F8E084918F010F5F1F4FF5
:10755000882321F00E94A78AF801F6CF84E398E0FF
:107560009FC062E873E085EF9DE00E94D5F1892B12
:1075700079F4E9E1F8E084918F010F5F1F4F8823D0
:1075800021F00E94A78AF801F6CF80E198E088C038
:1075900060E973E085EF9DE00E94D5F1892B71F4DD
:1075A0000DEE17E0F8018491882329F00F5F1F4F3B
:1075B0000E94A78AF7CF86EE97E072C066EA73E072
:1075C00085EF9DE00E94D5F1892B79F4E7ECF7E097
:1075D00084918F010F5F1F4F882321F00E94A78A9B
:1075E000F801F6CF80EC97E05BC068EB73E085EFC5
:1075F0009DE00E94D5F1892B79F4E8EAF7E08491C7
:107600008F010F5F1F4F882321F00E94A78AF80186
:10761000F6CF87E997E044C063EC73E085EF9DE027
:107620000E94D5F1892B79F4EEE7F7E084918F0180
:107630000F5F1F4F882321F00E94A78AF801F6CF21
:107640008CE697E02DC06FEC73E085EF9DE00E9423
:10765000D5F1892B79F4E1E5F7E084918F010F5F93
:107660001F4F882321F00E94A78AF801F6CF8FE3ED
:1076700097E016C06DED73E085EF9DE00E94D5F1B7
:10768000892BA9F4E5E2F7E084918F010F5F1F4F8A
:10769000882321F00E94A78AF801F6CF84E197E0C1
:1076A00090932C0780932B070E94D38A83C06AEEA5
:1076B00073E085EF9DE00E94D5F1892B09F07AC037
:1076C0001092130E77C01D8218861C821B8285E6DD
:1076D00092E09A83898380910C0A811103C066EE3F
:1076E00079E002C065E07AE06115710519F06C5F20
:1076F0007F4F02C060E070E021E045EF5DE0CE0129
:1077000005960E9453A8882361F18BE1FE0135960E
:10771000A9E0BAE001900D928A95E1F72B813C81B6
:107720003093080A2093070A80915A0B8A3008F098
:107730003DC091E0980F90935A0BFFE18F9FC001DD
:107740001124DC01A85DB54F4BE1E9E0FAE00190BE
:107750000D924A95E1F7FC01EC5DF54F33832283EE
:1077600025C0E1E8FAE184918F010F5F1F4F882364
:1077700021F00E94A78AF801F6CFEEEFF6E084919F
:107780008F010F5F1F4F882321F00E94A78AF80105
:10779000F6CF05EF1DE0F80181918F01882319F0E4
:1077A0000E94A78AF8CF8AE00E94A78ACE0101969C
:1077B0000E9480AA1092F50D8091090180FF07C1F7
:1077C000E7EBFBE084918F01882311F40C942532C0
:1077D000082E000C990B0E94A36B0F5F1F4FF8013E
:1077E0008491F2CF8FE40E9404DB81110C94253246
:1077F00083E40E9404DB0C94253283E50E9404DBC1
:10780000811159C08FE40E9404DB882319F08FE7AF
:107810009BE007C084E50E9404DB882349F087E5EC
:107820009BE090932C0780932B070E94D38A43C040
:1078300083E40E9404DB882319F08EE29BE0F1CF01
:1078400081E50E9404DB882319F086E09BE0E9CF04
:1078500088E40E9404DB8823C9F0E2E0FBE0849125
:107860008F01882351F0082E000C990B0E94A36B06
:107870000F5F1F4FF8018491F4CF8DE090E00E94DC
:10788000A36B8AE090E00E94A36B15C08CE40E9479
:1078900004DB882381F0EEEFFAE084918F018823E6
:1078A00061F3082E000C990B0E94A36B0F5F1F4F12
:1078B000F8018491F4CFE6ECFBE084918F018823FA
:1078C00011F40C942532082E000C990B0E94A36B26
:1078D0000F5F1F4FF8018491F2CF80913B09809197
:1078E0003C090C94253283E50E9404DB882309F4CB
:1078F0006EC086ED9AE090932C0780932B070E9430
:10790000D38AE6ECFBE084918F01882311F40C9478
:107910002532082E000C990B0E94A36B0F5F1F4F9E
:10792000F8018491F2CFE1EDFAE084918F01882390
:1079300051F0082E000C990B0E94A36B0F5F1F4F94
:10794000F8018491F4CFECECFAE084918F01882364
:1079500011F40C942532082E000C990B0E94A36B95
:107960000F5F1F4FF8018491F2CF88E50E9404DB7E
:10797000811106C089E50E9404DB882309F4C3C095
:1079800088E50E9404DB882341F08DE69CE090931B
:107990002C0780932B070E94D38A89E50E9404DB81
:1079A000882341F087E69CE090932C0780932B0777
:1079B0000E94D38A8AE50E9404DB882341F081E695
:1079C0009CE090932C0780932B070E94D38A809190
:1079D000C00D9091C10D019664E070E00E9463F1CA
:1079E0009093C10D8093C00D8091BC0D9091BD0D01
:1079F00001969093BD0D8093BC0D1092C40D109212
:107A0000C30D0C94CC304091C00D5091C10D9F011D
:107A10002F5F3F4F3093C40D2093C30D90E6949F8A
:107A20009001959F300D1124245C334FE20FF31F1A
:107A300080830C94CC300091C50D1091C60D780157
:107A400024E0E20EF11C6AE270E0C7010E94CAF174
:107A5000F80124812F3221F4B8016B5F7F4F03C0FE
:107A60002C3339F4B70185EF9DE00E94DEF10C94D0
:107A700025321092F50D009719F0FC013197108214
:107A80008091C50D9091C60D40E061E004960E9482
:107A900032D98091850B882389F0E8E8FCE0849155
:107AA0008F01882309F42FCB082E000C990B0E941C
:107AB000A36B0F5F1F4FF8018491F3CFE4E8FCE064
:107AC00084918F01882309F41ECB082E000C990B9A
:107AD0000E94A36B0F5F1F4FF8018491F3CF0E94A8
:107AE000EA6CE0E8FCE084918F01882311F40C94A7
:107AF0002532082E000C990B0E94A36B0F5F1F4FBD
:107B0000F8018491F2CF8AE50E9404DB811138CF1D
:107B100083E40E9404DB882309F459CF8DE59CE0BF
:107B200050CF86E40E9404DB882309F44DC10E94F3
:107B30001FDB0E94C3EF8B0189E59CE090932C072B
:107B400080932B070E94D38A88E50E9404DB882358
:107B500009F451C00E941FDB2B013C012DEC3CECD1
:107B60004CE45EE30E94FDE99E012F5F3F4F7901E7
:107B7000181674F020E030E0A901C301B2010E94A0
:107B8000A0F018162CF41F930F938EE49CE005C10F
:107B90002DEC3CEC4CEC5DEBC301B2010E94FDE925
:107BA00018167CF020E030E040E85FEBC301B20142
:107BB0000E94A0F018162CF41F930F9382E49CE00F
:107BC000ECC01F930F93C301B2010E94BEEF7F93DD
:107BD0006F9388E39CE09F938F93FF92EF920E94B4
:107BE000CFE90FB6F894DEBF0FBECDBFCE01019630
:107BF0000E94AE8ADFC089E50E9404DB882309F475
:107C000041C00E941FDB2B013C012DEC3CEC4CE4FD
:107C10005EE30E94FDE9FE0131967F01181674F0C3
:107C200020E030E0A901C301B2010E94A0F01816C3
:107C30002CF41F930F938DE29CE0AFC02DEC3CEC35
:107C40004CEC5DEBC301B2010E94FDE918167CF01B
:107C500020E030E040E85FEBC301B2010E94A0F0F9
:107C600018162CF41F930F9381E29CE096C01F938B
:107C70000F93C301B2010E94BEEF7F936F9387E120
:107C80009CE0A9CF8AE50E9404DB882309F441C067
:107C90000E941FDB2B013C012DEC3CEC4CE45EE32D
:107CA0000E94FDE9FE0131967F01181674F020E074
:107CB00030E0A901C301B2010E94A0F018162CF413
:107CC0001F930F938CE09CE068C02DEC3CEC4CECD7
:107CD0005DEBC301B2010E94FDE918167CF020E0C3
:107CE00030E040E85FEBC301B2010E94A0F018163B
:107CF0002CF41F930F9380E09CE04FC01F930F93D1
:107D0000C301B2010E94BEEF7F936F9386EF9BE0A9
:107D100062CF85E40E9404DB882309F44BC00E94F3
:107D20001FDB2B013C012DEC3CEC4CE45EE30E949C
:107D3000FDE9FE0131967F01181674F020E030E075
:107D4000A901C301B2010E94A0F018162CF41F93E0
:107D50000F938BEE9BE021C02DEC3CEC4CEC5DEBEB
:107D6000C301B2010E94FDE918167CF020E030E06A
:107D700040E85FEBC301B2010E94A0F018162CF49A
:107D80001F930F938FED9BE008C0C301B2010E94C7
:107D9000BEEF7F936F9384ED9BE09F938F93FF9251
:107DA000EF920E94CFE90F900F900F900F900F90DD
:107DB0000F901CCF80ED9BE090932C0780932B07B6
:107DC0000E94D38A0C94253200E010E0B5CE20E06A
:107DD00030E040E251E460914804709149048091A0
:107DE0004A0490914B040E94FDE987FF08C089EC8A
:107DF0009BE090932C0780932B070E94D38A82E309
:107E000090E090933904809338040E949A7D88EC26
:107E100090E00E94467CE6ECFBE084918F01882391
:107E200011F40C942532082E000C990B0E94A36BC0
:107E30000F5F1F4FF8018491F2CF20E030E040E265
:107E400051E4609148047091490480914A049091F2
:107E50004B040E94FDE987FF08C08FEB9BE09093E5
:107E60002C0780932B070E94D38A80E590E09093A3
:107E70003904809338040E949A7D80EF90E00E943C
:107E8000467CE6ECFBE084918F01882311F40C948E
:107E90002532082E000C990B0E94A36B0F5F1F4F19
:107EA000F8018491F2CF80E090E00E94467C10922D
:107EB0003904109238040E949A7DEBEBFBE0849128
:107EC0008F01882311F40C942532082E000C990B95
:107ED0000E94A36B0F5F1F4FF8018491F2CF6F9642
:107EE0000FB6F894DEBF0FBECDBFDF91CF911F91CB
:107EF0000F91FF90EF90DF90CF90BF90AF909F9049
:107F00008F907F906F905F904F903F902F9008954B
:107F10002F923F924F925F926F927F928F929F9299
:107F2000AF92BF92CF92DF92EF92FF920F931F9387
:107F3000CF93DF93CDB7DEB762970FB6F894DEBF6D
:107F40000FBECDBFF8948FEF9FEF90938900809381
:107F500088002AE02A8B212C312C78948091A60469
:107F60009091A704A091A804B091A904892B8A2B11
:107F70008B2B09F016C280914A0F8823E1F01092F2
:107F80004A0F8091480F9091490F892B09F409C23B
:107F900010925E041092490F1092480F90913B0985
:107FA00080913C09981709F4FCC180913C098F5FCE
:107FB0008F7080933C098091480F9091490F892BD5
:107FC00009F4EFC14091A2045091A3046091A4046C
:107FD0007091A50480919E0490919F04A091A004AB
:107FE000B091A1040091950410E020E030E0841BE2
:107FF000950BA60BB70B081719072A073B0710F4B8
:10800000D901C801E82F840F951FA61FB71F8093C1
:10801000A2049093A304A093A404B093A504209178
:10802000840030918500225E3F4F40917A04509148
:108030007B0460917C0470917D0480916A0490912E
:108040006B04A0916C04B0916D04840F951FA61F62
:10805000B71F80937A0490937B04A0937C04B09321
:108060007D04B7FD1CC0889A8091E1179091E217BA
:10807000A091E317B091E41740910402042E000C84
:10808000550B660B770B840F951FA61FB71F8093A8
:10809000E1179093E217A093E317B093E417409190
:1080A0007E0450917F0460918004709181048091DE
:1080B0006E0490916F04A0917004B0917104840FCC
:1080C000951FA61FB71F80937E0490937F04A093F3
:1080D0008004B0938104B7FD1CC08E9A8091E5178F
:1080E0009091E617A091E717B091E817409105022B
:1080F000042E000C550B660B770B840F951FA61FE3
:10810000B71F8093E5179093E617A093E717B093F6
:10811000E817409182045091830460918404709127
:1081200085048091720490917304A0917404B091BD
:108130007504840F951FA61FB71F80938204909328
:108140008304A0938404B0938504B7FD3FC080915D
:108150005804F09106028823C9F08091560482FFEA
:1081600002C0F7FD06C080915504882311F40C94D9
:108170003D49809156049091570493FF02C0F7FD4A
:108180000CC080915404811108C006C080910B017D
:108190008095887080930901419A4091E917509128
:1081A000EA176091EB177091EC178F2FFF0F990B67
:1081B000AA0BBB0B840F951FA61FB71F8093E9174F
:1081C0009093EA17A093EB17B093EC1740918604B5
:1081D000509187046091880470918904809176049D
:1081E00090917704A0917804B0917904840F951F41
:1081F000A61FB71F8093860490938704A0938804DA
:10820000B0938904B7FD3AC04091ED175091EE1735
:108210006091EF177091F017C09007020C2C000CC2
:10822000DD08EE08FF084C0D5D1D6E1D7F1D40939F
:10823000ED175093EE176093EF177093F01740917E
:108240006604509167046091680470916904841B0E
:10825000950BA60BB70B8093860490938704A0938D
:108260008804B0938904909159048091930493FFFA
:1082700002C0815001C08F5F80939304809184007D
:108280009091850082179307C8F380917A049091AA
:108290007B04A0917C04B0917D04B7FD15C0409192
:1082A0006604509167046091680470916904841BAE
:1082B000950BA60BB70B80937A0490937B04A09345
:1082C0007C04B0937D04889880917E0490917F0413
:1082D000A0918004B0918104B7FD15C0409166045F
:1082E000509167046091680470916904841B950B38
:1082F000A60BB70B80937E0490937F04A093800419
:10830000B09381048E988091820490918304A0910F
:108310008404B0918504B7FD3AC040916604509141
:1083200067046091680470916904841B950BA60B27
:10833000B70B8093820490938304A0938404B0933A
:108340008504809158048823E1F08091560482FFCF
:1083500004C08091060287FD05C0809155048823E2
:1083600009F493C7809156049091570493FF04C079
:108370008091060287FD0BC080915404811107C0D3
:1083800005C080910B018870809309014198E150EC
:1083900041F0809184009091850082179307C8F383
:1083A00042CE8091110290911202A0911302B091DD
:1083B0001402892B8A2B8B2B09F091C08091940495
:1083C000882309F453C08090A2049090A304A09045
:1083D000A404B090A504C0908F04D0909004E090C5
:1083E0009104F090920440919304C814D904EA04D3
:1083F000FB0480F480915F049091600420916304F9
:10840000309164042817390728F4415040939304AD
:10841000019714C08C149D04AE04BF04E0F4809155
:108420005F0490916004209161043091620482178E
:10843000930788F44F5F40939304019690936004F0
:1084400080935F0440910D0250910E0260910F02E3
:10845000709110020EC08FEF9FEFDC0180930D0230
:1084600090930E02A0930F02B09310024FEF5FEFB4
:10847000BA018091930487FD02C0169A01C0169834
:1084800080918400909185004E9620919304222340
:10849000F1F0149A20918400309185002817390753
:1084A000C8F32091930427FF02C02F5F01C0215021
:1084B00020939304149820919304222331F3209164
:1084C00084003091850028173907C8F3DDCF409329
:1084D0001102509312026093130270931402809160
:1084E000A6049091A704A091A804B091A904892B97
:1084F0008A2B8B2B09F046C6A091480FB091490FEB
:10850000109711F40C94E64A8090A2049090A30472
:10851000A090A404B090A50440919E0450919F04A3
:108520006091A0047091A10484169506A606B70672
:10853000D8F010925E041092490F1092480F90915B
:108540003B0980913C09981711F40C94E64A8091FC
:108550003C098F5F8F7080933C0940EDC42E47E04B
:10856000D42EE12CF12C1AC440919A0450919B0412
:1085700060919C0470919D04481559056A057B051E
:1085800008F4AAC140919604509197046091980410
:1085900070919904D6960D911D912D913C91D9978A
:1085A000401751076207730708F077C1411551055D
:1085B0006105710549F480905A0490905B04A09085
:1085C0005C04B0905D0464C1E12CF980842E952F89
:1085D000862F0A811B81FD81EE813F8128859C8049
:1085E000E0915617E89D912CFF2730915717389D41
:1085F000900CF11D10905817189CF00DE99F900CED
:10860000F11D399FF00DE89FF00D092D1F2F099DD9
:10861000E12D332722270F9FE00D311D2E1D199DBF
:10862000E00D311D2E1D1F9F300D211D032F122F18
:10863000099DF12C332722270F9FF00C311D2E1D91
:10864000199DF00C311D2E1D1F9F300D211D032F74
:10865000122FEE2780905A0490915B0480915C0465
:108660000090B6040E2809F483C03091B204309F04
:10867000E1198E089E098E092091B304209FE0190C
:1086800081089E098E09F090B404F09E801891092B
:108690008E09319FE01981089E098E09219F80185B
:1086A00091098E09F19E90198109099DF12C3327BA
:1086B00022270F9FF00C311D2E1D199DF00C311D2E
:1086C0002E1D1F9F300D211D032F122F3091AE0440
:1086D000309FE10D8E1C9E1D8E1D2091AF04209FAA
:1086E000E00D811C9E1D8E1DF090B004F09E800C4C
:1086F000911D8E1D319FE00D811C9E1D8E1D219FA1
:10870000800C911D8E1DF19E900D811D099DF12CF7
:10871000332722270F9FF00C311D2E1D199DF00CC1
:10872000311D2E1D1F9F300D211D032F122F309143
:10873000AA04309FE1198E089E098E092091AB048E
:10874000209FE01981089E098E09F090AC04F09EEC
:10875000801891098E09319FE01981089E098E09C0
:10876000219F801891098E09F19E9019810982C07C
:108770003091B204309FE10D8E1C9E1D8E1D209104
:10878000B304209FE00D811C9E1D8E1DF090B4044B
:10879000F09E800C911D8E1D319FE00D811C9E1D51
:1087A0008E1D219F800C911D8E1DF19E900D811DAF
:1087B000099DF12C332722270F9FF00C311D2E1D10
:1087C000199DF00C311D2E1D1F9F300D211D032FF3
:1087D000122F3091AE04309FE1198E089E098E0948
:1087E0002091AF04209FE01981089E098E09F09026
:1087F000B004F09E801891098E09319FE01981081C
:108800009E098E09219F801891098E09F19E901969
:108810008109099DF12C332722270F9FF00C311D70
:108820002E1D199DF00C311D2E1D1F9F300D211D79
:10883000032F122F3091AA04309FE10D8E1C9E1D34
:108840008E1D2091AB04209FE00D811C9E1D8E1D6E
:10885000F090AC04F09E800C911D8E1D319FE00DB8
:10886000811C9E1D8E1D219F800C911D8E1DF19ED1
:10887000900D811D11249C82F9820A831B83FD8344
:10888000EE833F832887912C992AA12CB12CA82A0A
:108890008BE595E121E0298B14C0D2968D909D90B7
:1088A000AD90BC90D597F4CFB694A7949794879445
:1088B000D988DD0CD98A049625E18737920709F417
:1088C000EAC4FC010591159125913491081519050B
:1088D0002A053B0548F3DFC440908F045090900474
:1088E0006090910470909204481459046A047B04C7
:1088F00008F0C3C180918E04811121C0FD01EE5B9F
:10890000FF4FE080F18002811381789620813181D0
:1089100042815381D2966D917D918D919C91D59795
:108920000E948DB3DD24D394D0928E04E091480F41
:10893000F091490F82A993A9A4A9B5A98EC140912C
:108940008A0450918B0460918C0470918D04DA96A6
:108950000D911D912D913C91DD97401751076207B4
:10896000730708F073C1411551056105710549F49C
:1089700080915A0490915B04A0915C04B0915D04D5
:108980006CC1F0E0E985842F352F262FAA857B85E1
:108990006C855D85BE854F859889B0915617B89FC7
:1089A000612D552740915717489F600D511D10901C
:1089B0005817189E500DB39F600D511D439F500DC9
:1089C000B29F500DA62F752FA69FB12D4427992732
:1089D000A59FB00D411D9F1F769FB00D411D9F1F8C
:1089E000759F400D911DA42F792FA69FE12D44273F
:1089F0009927A59FE00D411D9F1F769FE00D411D0A
:108A00009F1F759F400D911DA42F792FBB2780912B
:108A10005A0430915B0420915C040090B6040F2A44
:108A200009F483C04091B2044A9FB1198F0B3F0BE8
:108A30002F0B9091B3049A9FB01981093F0B2F0B14
:108A4000E091B404EA9F801931092F0B479FB019B8
:108A500081093F0B2F0B979F801931092F0BE79F3F
:108A600030192109A69FE12D44279927A59FE00DE4
:108A7000411D9F1F769FE00D411D9F1F759F400D5B
:108A8000911DA42F792F4091AE044A9FB10D8F1FE5
:108A90003F1F2F1F9091AF049A9FB00D811D3F1F64
:108AA0002F1FE091B004EA9F800D311D2F1F479FBB
:108AB000B00D811D3F1F2F1F979F800D311D2F1F50
:108AC000E79F300D211DA69FE12D44279927A59FE3
:108AD000E00D411D9F1F769FE00D411D9F1F759F5B
:108AE000400D911DA42F792F4091AA044A9FB119DE
:108AF0008F0B3F0B2F0B9091AB049A9FB0198109FC
:108B00003F0B2F0BE091AC04EA9F801931092F0B2A
:108B1000479FB01981093F0B2F0B979F801931098F
:108B20002F0BE79F3019210982C04091B2044A9F60
:108B3000B10D8F1F3F1F2F1F9091B3049A9FB00D4F
:108B4000811D3F1F2F1FE091B404EA9F800D311D4E
:108B50002F1F479FB00D811D3F1F2F1F979F800D17
:108B6000311D2F1FE79F300D211DA69FE12D4427AA
:108B70009927A59FE00D411D9F1F769FE00D411D88
:108B80009F1F759F400D911DA42F792F4091AE041A
:108B90004A9FB1198F0B3F0B2F0B9091AF049A9FF7
:108BA000B01981093F0B2F0BE091B004EA9F8019A7
:108BB00031092F0B479FB01981093F0B2F0B979F4E
:108BC000801931092F0BE79F30192109A69FE12D4C
:108BD00044279927A59FE00D411D9F1F769FE00D1B
:108BE000411D9F1F759F400D911DA42F792F40910E
:108BF000AA044A9FB10D8F1F3F1F2F1F9091AB04F6
:108C00009A9FB00D811D3F1F2F1FE091AC04EA9F7A
:108C1000800D311D2F1F479FB00D811D3F1F2F1F3E
:108C2000979F800D311D2F1FE79F300D211D1124AF
:108C3000E987AA877B876C875D87BE874F87988B7C
:108C400090E0932BA0E0B0E0A22B07C0A65ABF4F44
:108C50008D919D910D90BC91A02D2BE535E141E0CA
:108C6000498BF901459155916591749148175907C0
:108C70006A077B0708F499C3A6C3809193048823ED
:108C8000E1F0FD01E85BFF4F4081518160E070E061
:108C900000910D0210910E0220910F0230911002EE
:108CA000401751076207730741F0109211021092AA
:108CB0001202109213021092140240910902509174
:108CC0000A0260910B0270910C0277FF5FC0AE5AEE
:108CD000BF4FCD90DD90ED90FC908BE595E121E0CC
:108CE000FC0145915591659174914C155D056E059A
:108CF0007F0550F4F694E794D794C794220F049616
:108D000075E18737970761F72093950480E2C816CD
:108D1000D104E104F10428F470E2C72ED12CE12C37
:108D2000F12C90E2C91AD108E108F108C114A8E0B9
:108D3000DA06E104F10408F402C4B4E0DB9EC001E9
:108D40001124855A9E4EFC01329625913491EC2DCA
:108D50006627E39FA001E29F410D561F0694461F20
:108D6000561F112460E070E0FC0125913491C90187
:108D7000A0E0B0E0841B950BA60BB70B8093090213
:108D800090930A02A0930B02B0930C02C0900902C8
:108D9000D0900A02E0900B02F0900C028091480FF4
:108DA0009091490F892B09F0E5C10E940FB490936F
:108DB000490F8093480F892B09F4DCC1E091480FDB
:108DC000F091490F808183FF3EC085899689A789EC
:108DD000B08D8093E1179093E217A093E317B093BF
:108DE000E417818D928DA38DB48D8093E5179093B8
:108DF000E617A093E717B093E817858D968DA78D9A
:108E0000B0A18093E9179093EA17A093EB17B09362
:108E1000EC1781A192A1A3A1B4A18093ED17909327
:108E2000EE17A093EF17B093F01790913B09809144
:108E30003C09981709F4B9CF80913C098F5F8F7076
:108E400080933C09B2CFC588D688E788F08C81E052
:108E5000C114D104E104F10409F480E0018D128D04
:108E6000238D348D011511052105310509F082602E
:108E7000458D568D678D70A14115510561057105B0
:108E800009F0846080935E0410928A0410928B042F
:108E900010928C0410928D041092960410929704F4
:108EA000109298041092990485A196A1A7A1B0A54B
:108EB00080939E0490939F04A093A004B093A10478
:108EC000882499245401881A990AAA0ABB0A809214
:108ED000860490928704A0928804B09289048092BC
:108EE000820490928304A0928404B09285048092BC
:108EF0007E0490927F04A0928004B09281048092BC
:108F00007A0490927B04A0927C04B0927D04CC0CF5
:108F1000DD1CEE1CFF1CC0926A04D0926B04E09230
:108F20006C04F0926D04000F111F221F331F009379
:108F30006E0410936F042093700430937104440FF7
:108F4000551F661F771F40937204509373046093FC
:108F500074047093750441A152A163A174A1440FDC
:108F6000551F661F771F40937604509377046093D4
:108F7000780470937904880F991FAA1FBB1F8093F0
:108F8000660490936704A0936804B09369041092F8
:108F9000A2041092A3041092A4041092A50482A526
:108FA00093A5A4A5B5A580939A0490939B04A09340
:108FB0009C04B0939D0486A597A5A0A9B1A9809310
:108FC0008F0490939004A0939104B093920481A590
:108FD00080936504DF01A95BBF4F9C91909394043B
:108FE000992339F115962D913C9111973093640492
:108FF0002093630412972D913C9111973093620452
:109000002093610410921102109212021092130226
:109010001092140212972D913C91A90160E070E02A
:1090200040930D0250930E0260930F027093100252
:109030000CC088248A94982C540180920D0290923E
:109040000E02A0920F02B0921002EA5BFF4F9081D5
:109050002091590492130AC02091080230E0482F51
:10906000082E000C550B4217530731F0909359040A
:10907000809308020E94DFB30E9411C02FEF3FEFE0
:10908000A9012093090230930A0240930B025093E6
:109090000C02E091480FF091490FDF01DE96ED9050
:1090A000FD900D911C9122A933A944A955A9EA5A12
:1090B000FF4F60817181828193810E948DB31092F4
:1090C0008E04E091480FF091490FEA5AFF4F8080DB
:1090D0009180A280B3808BE595E121E0FC01459170
:1090E000559165917491481559056A057B0558F4A9
:1090F000B694A79497948794220F0496A7E7B5E1B6
:10910000A817B90759F720939504B0E28B1691047C
:10911000A104B10428F4B0E28B2E912CA12CB12C27
:1091200030E2831A9108A108B108811448E094063E
:10913000A104B10408F427C254E0959EC001112493
:10914000855A9E4EFC01329625913491782D6627E2
:10915000739FA001729F410D561F0694461F561F14
:109160001124FC01C590D490E12CF12CC41AD50A2D
:10917000E108F108C092A604D092A704E092A804E6
:10918000F092A9040091A6041091A7042091A804CC
:109190003091A90440911102509112026091130282
:1091A00070911402F02E198BF22FE32F4017510704
:1091B0006207730720F4F42E598BF62FE72F8F2DBB
:1091C0009989AF2FBE2F0097E1E0AE07B10520F0DF
:1091D0008FEF9FEFA0E0B0E0081B190B2A0B3B0BB1
:1091E0000093A6041093A7042093A8043093A90425
:1091F0004F3FFFEF5F076F077F0761F0481B590B79
:109200006A0B7B0B4093110250931202609313027E
:1092100070931402F8942091840030918500205FAF
:109220003F4F4A8941504A8B442341F0280E391E52
:109230002216330610F40C94AD3F01C01901309290
:10924000890020928800789462960FB6F894DEBF69
:109250000FBECDBFDF91CF911F910F91FF90EF9087
:10926000DF90CF90BF90AF909F908F907F906F9046
:109270005F904F903F902F90089580910B018095C3
:109280008870809309010C94B94080910B0188701B
:109290008093090167C839893093950480E2881664
:1092A0009104A104B10428F430E2832E912CA12C66
:1092B000B12C30E2831A9108A108B108811488E02A
:1092C0009806A104B10420F1E4E09E9EC00111249F
:1092D000855A9E4EFC01329625913491F82DEE2749
:1092E000F39F7001F29FE10CFE1E0694EE1EFE1E1F
:1092F0001124FC01C590D490860120E030E04801A3
:1093000059018E189F08A108B1087501640122C097
:10931000950184013695279517950795F801EC7FFF
:10932000CF01855A924FFC01C590D490FC01329632
:1093300025913491E82DE770E29FC001E39F900DE5
:10934000112423E0969587952A95E1F7C81AD90A42
:10935000E12CF12C4C0D5D1D6E1D7F1D409396047C
:109360005093970460939804709399049091940497
:1093700080919304992309F473C0882309F40ECDD6
:10938000A85BBF4F8D919C91A0E0B0E040910D0291
:1093900050910E0260910F02709110028417950790
:1093A000A607B70709F05FC0F9CCB695A7959795C2
:1093B0008795D988DD0CD98A2C5F3F4F45E1273747
:1093C000340709F04ECC59895093950480329105A9
:1093D000A105B10520F480E290E0A0E0B0E0809724
:1093E000A109B109811558E09507A105B10508F457
:1093F00043C074E0979F90011124255A3E4EF90115
:10940000329645915491EE27859FB001849F610D5E
:109410007E1F06946E1F7E1F1124F901C590D49003
:10942000E12CF12CC61AD70AE108F10880918A04D0
:1094300090918B04A0918C04B0918D048C0D9D1D96
:10944000AE1DBF1D80938A0490938B04A0938C045F
:10945000B0938D0480919404811130C08091930465
:10946000882309F49BCC10921102109212021092E0
:1094700013021092140292CCAC01BD01769567954F
:1094800057954795FA01EC7F9F01255A324FF90114
:10949000C590D490F9013296459154918770849F7C
:1094A0009001859F300D1124F3E036952795FA95AC
:1094B000E1F7C21AD30AE12CF12CB8CF8989480E02
:1094C000511C611C711C8091480F9091490F4814E8
:1094D00059046A047B04D8F420919304222309F4EC
:1094E0005DCCFC01E85BFF4F20813181A90160E088
:1094F00070E000910D0210910E0220910F02309148
:109500001002401751076207730709F447CC109205
:109510001102109212021092130210921402FC0116
:10952000E85BFF4F80819181A0E0B0E080930D0265
:1095300090930E02A0930F02B09310022FCCD7018C
:10954000C601B695A79597958795FC01EC7FCF014D
:10955000855A924FFC0125913491FC013296459138
:1095600054916C2D6770649FC001659F900D11240C
:1095700063E0969587956A95E1F7281B390BC90139
:10958000A0E0B0E0FBCBD501C401B695A7959795B7
:109590008795FC01EC7FCF01855A924FFC01C59065
:1095A000D490FC01329625913491482D4770429F0A
:1095B000C001439F900D1124A3E096958795AA952D
:1095C000E1F7C81AD90AE12CF12CD4CD80EDC82ED0
:1095D00087E0D82EE12CF12CE8CBCF92DF92EF92EE
:1095E000FF92CF93DF936B017C01EA0121E338E026
:1095F00040EA50EC0E94A0F087FD23C022E430E056
:1096000047E553E4C701B6010E94FDE91816CCF006
:10961000C880D980EA80FB802FE632E143E85AEB2C
:10962000C701B6010E94A0F087FD0BC0C1E022E493
:1096300030E047E553E4C701B6010E94FDE9181682
:109640000CF4C0E08C2FDF91CF91FF90EF90DF9072
:10965000CF9008950F931F93CF93DF93FC01A685BE
:10966000B7858D0100581F4FE801888199810196C7
:109670008F779927AD014E575F4FEA0128813981D5
:1096800028173907D1F3E80128813981A20FB31FC8
:109690006C93A685B785A058BF4F11969C938E9367
:1096A000A689B7892C9181E090E0078C02C0880FD1
:1096B000991F0A94E2F7822B8C9381E081A304889E
:1096C000F589E02D80818064808381E090E0DF91E6
:1096D000CF911F910F910895FC0181A1882329F05A
:1096E000A489B5898C9186FFFBCF11A20895FC0156
:1096F000A485B585FD01E058FF4F20813181329668
:10970000808191812817390779F080819181A80F94
:10971000B91F8C91208131812F5F3F4F2F773327E5
:109720003183208390E008958FEF9FEF0895DC014F
:109730001C96ED91FC911D97DF01A058BF4F2D9114
:109740003C91119712968D919C911197281739078A
:1097500039F08D919C91E80FF91F808190E0089578
:109760008FEF9FEF0895FC0124853585F901E058BE
:10977000FF4F8081918132962081318180589F4FA7
:10978000821B930B60E870E00C9463F108950895D8
:1097900080E090E00895CF92DF92EF92FF92C09028
:1097A0004202D0904302E0904402F0904502FC0156
:1097B00080819181A281B381809342029093430280
:1097C000A0934402B09345020E9402CEC09242028E
:1097D000D0924302E0924402F0924502FF90EF9053
:1097E000DF90CF9008958091CC189091CD18981764
:1097F00059F0E92FF0E0E45BF74E80819F5F9F779F
:109800009093CD1890E008958FEF9FEF08951F92E9
:109810000F920FB60F9211240BB60F922F938F93C6
:109820009F93EF93FF932091CD18E091CC1881E0A6
:109830008E0F8F779091C600281729F0F0E0E45B37
:10984000F74E9083E82FE093CC18FF91EF919F9112
:109850008F912F910F900BBE0F900FBE0F901F9006
:1098600018958091250490912604009731F04AE0E4
:1098700050E060E070E00C9451E760E070E0CB01F4
:109880000895EFDF97FD0AC0ECDF6F3F710581059A
:10989000910509F02CF4E5DF862F089580E0089506
:1098A0008FEF08958091250490912604892B31F043
:1098B000E8DF91E0811103C090E001C091E0892FC1
:1098C00008950F931F93CF938091250490912604C0
:1098D000009711F1FC018F01C1912C2F2F7DA9F070
:1098E000C53411F0C536B9F7F801108260E070E0B8
:1098F00080912504909126040E94FEE5F801C08322
:10990000562F472F382F292F0BC060E070E0CF91E2
:109910001F910F910C94FEE550E040E030E020E014
:10992000652F742F832F922FCF911F910F91089540
:1099300081548A3108F042C0E82FF0E0409143188A
:1099400050914418609145187091461804C076955E
:109950006795579547958A95D2F7842F817040FF78
:109960002FC0E75DF74E9081992309F1E091D1175F
:10997000F091D217E90FF11D908120ED290F2A30C7
:1099800098F09E3211F491810CC09D3211F09B32FF
:1099900071F4918120ED290F2A3030F09E3239F494
:1099A000928190539A3018F42E2F9F2F02C020E0FE
:1099B00090E02093250490932604089580E0089574
:1099C0000895B6DF882341F081E02091250430918D
:1099D0002604232B09F480E0089580E1E0E4F4E01C
:1099E000ADE0B8E101900D928A95E1F708952F92CC
:1099F0003F924F925F926F927F928F929F92AF921F
:109A0000BF92CF92DF92EF92FF920F931F93CF936B
:109A1000DF9300D01F921F92CDB7DEB77C018B0180
:109A20006A0119018090400490904104A090420482
:109A3000B0904304A5019401FC0160817181828191
:109A400093810E94FDE9F1E0FD83811112C0209114
:109A50004404309145044091460450914704F80174
:109A600060817181828193810E94FDE9811101C031
:109A70001D82F60140805180628073802091150222
:109A8000309116024091170250911802C301B201A1
:109A90000E94FDE9882309F453C0409215025092B8
:109AA0001602609217027092180220E030E040E443
:109AB00050E4609110077091110780911207909106
:109AC00013070E9456EF69837A838B839C8380926D
:109AD0000D1890920E18A0920F18B0921018809145
:109AE000440490914504A0914604B09147048093AA
:109AF000111890931218A0931318B0931418F6012C
:109B000080819181A281B38180931518909316185A
:109B1000A0931718B093181880914C0490914D049D
:109B2000A0914E04B0914F048093191890931A1885
:109B3000A0931B18B0931C18CE0101962CDE4DDFAC
:109B4000FD81FF2309F160900C0770900D07809054
:109B50000E0790900F07A0900807B0900907C090DB
:109B60000A07D0900B079501A601B301C4010E941A
:109B7000A0F0181614F05301640120E030E040E238
:109B800051E4B501C6010CC020E030E040EC5FE3D9
:109B9000609114077091150780911607909117072F
:109BA0000E9456EF69837A838B839C8320912404DF
:109BB000222349F0AB01BC018BE795E10E9461B41F
:109BC0008AE00E94A78AF70180819181A281B381F6
:109BD00080930D1890930E18A0930F18B09310183F
:109BE000F80180819181A281B381809311189093B3
:109BF0001218A0931318B0931418F1012081318129
:109C0000428153816091191870911A1880911B1824
:109C100090911C180E947AEE6093191870931A188C
:109C200080931B1890931C18CE010196B4DDD5DEED
:109C30000F900F900F900F900F90DF91CF911F9189
:109C40000F91FF90EF90DF90CF90BF90AF909F90DB
:109C50008F907F906F905F904F903F902F900895DE
:109C600080E1EDE0F8E1A0E4B4E001900D928A9586
:109C7000E1F708959C0197FD0EC08436910584F0AC
:109C800064E670E00E9463F1CB016AE070E00E943C
:109C900063F1805D06C03195219531098DE201C0E7
:109CA00080E2809331042A30310564F0EAE0F0E08C
:109CB000C901BF010E9463F1CB01BF010E9463F1A2
:109CC000805D01C080E280933204C9016AE070E0E7
:109CD0000E9463F1805D8093330481E394E00895F2
:109CE000883791051CF028E780E002C0282F892FD3
:109CF00020933804809339040C949A7D2F923F92DC
:109D00004F925F926F927F928F929F92AF92BF928B
:109D1000CF92DF92EF92FF920F931F93CF93DF9337
:109D2000CDB7DEB7C455D1090FB6F894DEBF0FBE6C
:109D3000CDBFEAE3F8E184918F010F5F1F4F8823C5
:109D400021F00E94A78AF801F6CF0E94A6C48111D3
:109D50000C94615880E090E0A0E8BFE38093051880
:109D600090930618A0930718B093081880E090E02D
:109D7000A0ECB0E48093091890930A18A0930B18F4
:109D8000B0930C188DEC9CECACE4BEE3809301180E
:109D900090930218A0930318B093041880E090E009
:109DA000A8ECB1E48093280590932905A0932A0597
:109DB000B0932B058CE390E09093270580932605C4
:109DC00088EC90E09093250580932405109223055C
:109DD0008FE4F7DD882311F074DD04C060E070E0EB
:109DE00080E190E46BAF7CAF8DAF9EAF83E4E9DDA3
:109DF000882311F057DD02C083E49ADD61968FAFAE
:109E000061978BE4DEDD882311F04CDD02C08BE42A
:109E10008FDD60968FAF609782E4D3DD8823E9F011
:109E200050DD0E94BEEF70932705609326056115F3
:109E3000710599F0685271096536710570F0E5E0B9
:109E4000F8E184918F010F5F1F4F882311F40C9468
:109E500061580E94A78AF801F4CF8CE4B2DD882310
:109E600051F12FDD6B017C01609301187093021892
:109E7000809303189093041820E030E0A9010E9419
:109E8000A0F087FD0AC020E030E040E050E4C701C8
:109E9000B6010E94FDE9181674F4EDEDF7E1849126
:109EA0008F010F5F1F4F882311F40C9461580E949B
:109EB000A78AF801F4CF81E53BDD882309F440C08F
:109EC0008091250490912604892B19F4E2EBF7E1A7
:109ED0002BC0F7DC6B017C016093091870930A18A2
:109EE00080930B1890930C182DEC3CEC4CE45DE344
:109EF0000E94A0F087FD0AC020E030E040E751E476
:109F0000C701B6010E94FDE91816D4F4E1E8F7E1B3
:109F100084918F010F5F1F4F882311F40C946158B7
:109F20000E94A78AF801F4CF84918F010F5F1F4F21
:109F3000882311F40C9461580E94A78AF801F4CF89
:109F400083E53FDD882319F1BCDC4B015C012DEC7E
:109F50003CEC4CEC5DE30E94A0F087FD0AC020E0E1
:109F600030E040E85FE3C501B4010E94FDE9181646
:109F7000ACF4EAE5F7E184918F010F5F1F4F88236E
:109F800011F40C9461580E94A78AF801F4CF5DEC9B
:109F9000852E5CEC952EA92C5EE3B52E80E5C8DC01
:109FA000882309F443C08091250490912604892BCD
:109FB00071F4E2E2F7E184918F010F5F1F4F882374
:109FC00011F40C9461580E94A78AF801F4CF809193
:109FD00023058F5F8093230574DC6B017C01609304
:109FE00028057093290580932A0590932B0520E07E
:109FF00030E0A9010E94A0F087FD0AC020E030E017
:10A0000048EC51E4C701B6010E94FDE9181674F44A
:10A01000EAEFF6E184918F010F5F1F4F882311F45F
:10A020000C9461580E94A78AF801F4CF86E4C9DC39
:10A03000882319F146DC6B017C0120E030E040E828
:10A040005FE30E94A0F087FD0AC020E030E040E816
:10A0500050E4C701B6010E94FDE91816A4F4E1ED31
:10A06000F6E184918F010F5F1F4F882311F40C9448
:10A0700061580E94A78AF801F4CFC12CD12C40EE80
:10A08000E42E4FE3F42EA7019601C701B6010E940A
:10A0900062EA9B01AC0160E070E084E490E40E941D
:10A0A00056EF2091051830910618409107185091ED
:10A0B00008180E9462EA2B013C01A5019401C50128
:10A0C000B4010E9462EAA70196010E9462EA2CEEA6
:10A0D00031E548EB5DE30E9456EF9B01AC01C30103
:10A0E000B2010E9462EA609305187093061880938B
:10A0F00007189093081888E464DC8823C9F0E1DB32
:10A100000E94BEEF7093250560932405655A71097E
:10A110006437710568F0E3EAF6E184918F010F5F1F
:10A120001F4F882309F4CDC70E94A78AF801F5CFF5
:10A1300085E5FEDB8823E9F00E941F596115710552
:10A140008105910511F00E94F5E58091250490911B
:10A150002604892B11F0B5DB04C060E070E088E4D0
:10A1600092E460931F0570932005809321059093DE
:10A17000220582E5DDDB81110DC0EFE6F6E1849179
:10A180008F010F5F1F4F882309F49BC70E94A78A86
:10A19000F801F5CF8091250490912604892BA9F030
:10A1A00060DB2F967FAF6EAF2F97161617069CF0C9
:10A1B000EBE3F6E184918F010F5F1F4F882309F4D1
:10A1C00080C70E94A78AF801F5CF8AE190E02F9618
:10A1D0009FAF8EAF2F9788E5F4DB882361F071DBAA
:10A1E000209118043091190440911A0450911B04D5
:10A1F0000E9479EE08C06091400470914104809102
:10A2000042049091430460931B0570931C05809356
:10A210001D0590931E0589E5D4DB882361F051DB91
:10A2200020911C0430911D0440911E0450911F0484
:10A230000E9479EE08C060914404709145048091B9
:10A240004604909147046093170570931805809316
:10A25000190590931A0560911B0570911C0580915A
:10A260001D0590911E0547E155E0B7D981110DC03C
:10A27000E1E1F6E184918F010F5F1F4F882309F41C
:10A2800020C70E94A78AF801F5CF84E451DB91E052
:10A2900089270E94359320E030E040EA50E4609145
:10A2A00048047091490480914A0490914B040E94A3
:10A2B000FDE987FF14C0198A1A8A1B8A1C8A80E06C
:10A2C00090E0A0EAB0E489839A83AB83BC83BE01AB
:10A2D0006F5E7F4FCE0101960E9488C4C1DCAFD76C
:10A2E0006B017C01A8E8CA0EA3E1DA1EE11CF11C97
:10A2F0008091260590912705F3DC609126057091E9
:10A300002705072E000C880B990B0E9403EA9B017E
:10A31000AC0160913A0470913B0480913C049091AF
:10A320003D040E9479EE4B015C0120E030E0A90180
:10A330000E94A0F087FF04C0B7FAB094B7F8B094B9
:10A3400020E030E040E450E4C501B4010E94A0F0F8
:10A350001816F4F474D7DC01CB018C199D09AE09F1
:10A36000BF09B7FD0EC06BD76B017C01B8E8CB0EFF
:10A37000B3E1DB1EE11CF11C0E94E07C8AE00E943C
:10A38000A78A0E94EAAA8091CC188093CD18B5CFF5
:10A3900080912405909125050E94467C60912405BA
:10A3A00070912505072E000C880B990B0E9403EA7B
:10A3B0009B01AC0160915004709151048091520452
:10A3C000909153040E9479EE4B015C0120E030E053
:10A3D000A9010E94A0F087FF04C0B7FAB094B7F8B3
:10A3E000B09420E030E040E450E4C501B4010E94A4
:10A3F000A0F01816F4F423D7DC01CB018C199D09C9
:10A40000AE09BF09B7FD0EC01AD76B017C01E8E8A1
:10A41000CE0EE3E1DE1EE11CF11C0E94E07C8AE02E
:10A420000E94A78A0E94EAAA8091CC188093CD1836
:10A43000B5CF10924C0410924D0410924E0410921D
:10A440004F040E9454C380912305882399F1C5DAF3
:10A45000209128053091290540912A0550912B051E
:10A460006091191870911A1880911B1890911C18FE
:10A470000E947AEE6093191870931A1880931B1833
:10A4800090931C1820E030E040E751E460911407FD
:10A490007091150780911607909117070E9456EF4B
:10A4A00069837A838B839C83CE01019674D995DA74
:10A4B0000E9461C180E2E7EFF4E0DF01282F1D92E6
:10A4C0002A95E9F7E7EDF4E0DF01282F1D922A95A0
:10A4D000E9F7E7EBF4E0DF011D928A95E9F77DDA11
:10A4E0008091011890910218A0910318B09104185E
:10A4F0008093151890931618A0931718B0931818F6
:10A5000019821A821B821C829E012F5F3F4F45E1F8
:10A5100058E161E178E18DE098E169DA9E01255C1E
:10A520003F4F45E158E161E178E18DE098E15FDA84
:10A530006196BFAD6197BB2329F064E474E080E4C9
:10A5400094E004C067E175E08BE195E00E943ADC9D
:10A55000298F3A8F4B8F5C8F6D8F7E8F3FAF2D96FB
:10A560002FAF2D972D96EFAD2D97E7FD81C4FFAD51
:10A57000F7FD7EC424E0E202F0011124EB57F64F10
:10A5800040805180628073803FAD84E03802F001EA
:10A590001124EF58F64FD080C180328023808D2D5A
:10A5A0009C2DA32DB22D8FAB98AFA9AFBAAFAE0142
:10A5B000495C5F4FB201C30110D8882309F45CC421
:10A5C00020E030E040EA50E4B201C3010E947AEE9C
:10A5D000F62E072F182FE92E862F902FA12FBE2D94
:10A5E0008BAB9CABADABBEAB8D2D9C2DA32DB22DFB
:10A5F0008FA798ABA9ABBAAB2D969FAD2D979111B4
:10A6000052C0AFADA11105C05F2D402F312F2E2DAF
:10A6100004C0542D452D362D272D852F942FA32F83
:10A62000B22F8BAB9CABADABBEABBFADB43034F493
:10A63000F42C052D162DE72CBB2369F020E030E02B
:10A6400040EA50E46D2D7C2D832D922D0E9479EEF1
:10A65000362F272F03C09601832D922D432F522F83
:10A66000BC014FA758AB69AB7AABEFADE4300CF04F
:10A67000A7C020E030E040EA50E46D2D7C2D832D12
:10A68000922D0E947AEE21966FAF219723967FAF8D
:10A69000239725968FAF259727969FAF2797FFADD6
:10A6A000F11185C099C02D962FAD2D9724300CF453
:10A6B00053C03FAD34305CF020E030E040EA50E47D
:10A6C000B201C3010E9479EE362F272F03C0342D2B
:10A6D000252DC301432F522FBC014BAB5CAB6DAB9F
:10A6E0007EAB8FAD8111E4C420E030E040EA50E45D
:10A6F000B201C3010E9479EEF62E072F182FE92E22
:10A7000020E030E040EA50E46D2D7C2D832D922D29
:10A710000E947AEE6FA778AB89AB9AAB9FAD992375
:10A7200009F44EC020E030E040EA50E46D2D7C2D6D
:10A73000832D922D0E9479EE21966FAF219723965B
:10A740007FAF239725968FAF259727969FAF2797A3
:10A75000AFADA43064F140C0BFADB1110DC020E079
:10A7600030E040EA50E4B201C3010E9479EEF62ED7
:10A77000072F182FE92E0FC0EFADE430B4F120E021
:10A7800030E040EA50E4B201C3010E9479EE6BABC5
:10A790007CAB8DAB9EAB2196DFAE21972396CFAEDF
:10A7A000239725963FAE259727962FAE279732ED14
:10A7B000832E33E5932E3BE7A32E31E4B32E29C03D
:10A7C0002196DFAE21972396CFAE239725963FAEF5
:10A7D000259727962FAE279722ED822E23E5922EDE
:10A7E0002BEFA22E20E4B22E14C02196DFAE2197CB
:10A7F0002396CFAE239725963FAE259727962FAE6B
:10A80000279792ED892E93E5992E9BEFA92E91E43F
:10A81000B92E8BA99CA9ADA9BEA92C968CAF9DAFD2
:10A82000AEAFBFAF2C979C01AD01B201C3010E9436
:10A8300079EE698B7A8B8B8B9C8B4FA458A869A877
:10A840007AA8A30192016D2D7C2D832D922D0E945B
:10A8500079EE6D8B7E8B8F8B988F2C962CAD3DADCA
:10A860004EAD5FAD2C976091400470914104809192
:10A870004204909143040E9479EE2C966CAF7DAF18
:10A880008EAF9FAF2C97A301920160914404709109
:10A89000450480914604909147040E9479EE2B0173
:10A8A0003C018F2D902FA12FBE2D89839A83AB83DE
:10A8B000BC8321968FAD219723969FAD2397259634
:10A8C000AFAD25972796BFAD27978D839E83AF8326
:10A8D000B8878091011890910218A0910318B09147
:10A8E000041889879A87AB87BC872DEC3CEC4CEC2D
:10A8F0005CE3C501B4010E9462EA20910518309121
:10A90000061840910718509108180E9462EA209199
:10A910004C0430914D0440914E0450914F040E94DC
:10A920007AEE6D877E878F87988B2C962CAD3DAD08
:10A930004EAD5FAD2C97CA01B9010E9462EA6B016E
:10A940007C01A3019201C301B2010E9462EA9B0152
:10A95000AC01C701B6010E947AEE20E030E040E091
:10A9600050E40E94A0F018160CF046C00E9461C18D
:10A970001BA21CA21DA21EA220E030E040E05FE36B
:10A98000609148047091490480914A0490914B046D
:10A990000E947AEE6F8F78A389A39AA39E012D5D02
:10A9A0003F4FAE01415E5F4F64E474E080E494E0A9
:10A9B0001ED81BA21CA21DA21EA220E030E040E077
:10A9C0005FE36091011870910218809103189091D3
:10A9D00004180E947AEE6F8F78A389A39AA39E0130
:10A9E0002D5D3F4FAE01415E5F4FBE01615D7F4F08
:10A9F000CE01C3960E94F74C1F8E18A219A21AA26C
:10AA00009E01215E3F4F41E058E1BE01615D7F4FF5
:10AA1000CE01C3960E94F74C0E948DC14090420225
:10AA2000509043026090440270904502E0900C0701
:10AA3000F0900D0700910E0710910F07A0900807E6
:10AA4000B0900907C0900A07D0900B079501A601A6
:10AA5000B701C8010E94A0F0181614F47501860110
:10AA600020E030E040E251E4B701C8010E9456EF17
:10AA70006093420270934302809344029093450294
:10AA800040E0BE016F5E7F4FCE0101960E943FAF56
:10AA900040924202509243026092440270924502F8
:10AAA0000E94ED4CA5E8B9E02496BFAFAEAF249765
:10AAB00022961FAE1EAE229701E010E021960FAC49
:10AAC000219702C0000F111F0A94E2F72296EEAD03
:10AAD000FFAD229731962296FFAFEEAF229721E08D
:10AAE00030E021960FAC219702C0220F331F0A9449
:10AAF000E2F763963FAF2EAF639787EB282E84E093
:10AB0000382E87EF94E02A969FAF8EAF2A97A7ED55
:10AB1000B4E02896BFAFAEAF2897E1E7F9E02696FC
:10AB2000FFAFEEAF26972A962EAD3FAD2A976596DA
:10AB30003FAF2EAF6597D9018D919C919C01202349
:10AB40003123232B09F4ADC06396EEADFFAD6397BF
:10AB50008E239F23892B09F4A4C02896AEADBFADE8
:10AB600028978D919C9180239123892B09F099C07E
:10AB700020E030E040E050E42496AEADBFAD249735
:10AB80006D917D918D919C910E947AEE6B017C017B
:10AB900020E030E040E050E42496EEADFFAD249795
:10ABA00064817581868197810E9479EE4B015C01F9
:10ABB00020E030E040E850ECC701B6010E94FDE91A
:10ABC00087FD70C120E030E046E553E4C701B601DF
:10ABD0000E94A0F0181634F4C12CD12CB6E5EB2E4F
:10ABE000B3E4FB2ECBA6DCA6EDA6FEA62696AEAD64
:10ABF000BFAD26974D905D906D907C9020E030E049
:10AC000040E85FE3C301B2010E94FDE987FD51C145
:10AC100020E030E046E553E4C301B2010E94A0F019
:10AC2000181634F4412C512CF6E56F2EF3E47F2EE8
:10AC30004F8E58A269A27AA24FA258A669A67AA6F8
:10AC400020E030E040E850ECC501B4010E94FDE98D
:10AC500087FD36C120E030E046E553E4C501B4018C
:10AC60000E94A0F0181634F4812C912C76E5A72EC2
:10AC700073E4B72E8BA29CA2ADA2BEA2AE01495D29
:10AC80005F4FC701B6010E94ED4A811120C128968D
:10AC9000EEADFFAD289780819181802B912B918320
:10ACA00080832A962EAD3FAD2A972E5F3F4F2A967E
:10ACB0003FAF2EAF2A976596AEADBFAD65978D912C
:10ACC0009C9180239123892B09F4A6C0F9018081EE
:10ACD000918180239123892B09F49EC0F101808109
:10ACE000918180239123892B09F096C020E030E0E8
:10ACF00040E050E42696AEADBFAD26976D917D91B4
:10AD00008D919C910E947AEE2B013C0120E030E075
:10AD100040E050E42696EEADFFAD26976481758144
:10AD2000868197810E9479EE4B015C012496AEAD3D
:10AD3000BFAD2497CD90DD90ED90FC9020E030E009
:10AD400040E850ECC701B6010E94FDE987FDFFC055
:10AD500020E030E046E553E4C701B6010E94A0F0D0
:10AD6000181634F4C12CD12C56E5E52E53E4F52EFB
:10AD7000CBA2DCA2EDA2FEA2CBA6DCA6EDA6FEA68F
:10AD800020E030E040E85FE3C301B2010E94FDE94A
:10AD900087FDE4C020E030E046E553E4C301B201A2
:10ADA0000E94A0F0181634F4412C512C36E5632E85
:10ADB00033E4732E4FA258A669A67AA620E030E0AD
:10ADC00040E85FE3C501B4010E94FDE987FDCDC005
:10ADD00020E030E046E553E4C501B4010E94A0F054
:10ADE000181634F4812C912C96E5A92E93E4B92EF3
:10ADF0008F8E98A2A9A2BAA2AE01495D5F4FC7018A
:10AE0000B6010E94ED4A8111B7C0F10180819181A4
:10AE1000802B912B91838083F2E02F0E311C28969A
:10AE20002EAD3FAD28972E5F3F4F28963FAF2EAFF8
:10AE3000289726968EAD9FAD2697049626969FAFAF
:10AE40008EAF269791EC291694E0390609F06BCE67
:10AE50002496AEADBFAD249714962496BFAFAEAF87
:10AE600024972296EEADFFAD2297359709F024CEB8
:10AE70008091CC188093CD182F962EAD3FAD2F9793
:10AE8000215031092F963FAF2EAF2F97232B09F476
:10AE9000B3C02D963FAD2D9737FDAEC08FAD87FF68
:10AEA00047CBAAC0C12CD12CA0E8EA2EA0ECFA2EE8
:10AEB00099CE412C512CE0E86E2EEFE37E2EB8CED9
:10AEC000812C912C60E8A62E60ECB62ED3CEAE017C
:10AED000415E5F4FC501B4010E94ED4A882309F429
:10AEE000D6CE80912404882321F1B701A6018BEEF0
:10AEF00095E10E9461B44FA158A569A57AA585EE98
:10AF000095E10E9461B44BA15CA16DA17EA18BED86
:10AF100095E10E9461B44F8D58A169A17AA185ED98
:10AF200095E10E9461B489E20E94A78A8AE00E94AA
:10AF3000A78A9E01215E3F4FAE014D5D5F4FBE016E
:10AF4000695D7F4FCE018B960E94BDC1A0CEC12C02
:10AF5000D12C40E8E42E40ECF42E0ACF412C512CA9
:10AF600020E8622E2FE3722E25CF812C912C80E8D1
:10AF7000A82E8FE3B82E3CCFAE01415E5F4FC701D4
:10AF8000B6010E94ED4A882309F43FCF8091240442
:10AF9000882321F1B701A60181EB95E10E9461B4FC
:10AFA0004FA158A569A57AA58BEA95E10E9461B4E5
:10AFB0004BA15CA16DA17EA181EA95E10E9461B4E3
:10AFC0004F8D58A169A17AA18BE995E10E9461B4E6
:10AFD00089E20E94A78A8AE00E94A78A9E01215ED8
:10AFE0003F4FAE014D5D5F4FBE01695D7F4FCE01AA
:10AFF0008B960E94BDC109CF0E9461C180E090E0A4
:10B00000A0EAB0E48093151890931618A09317182F
:10B01000B093181819821A821B821C829E012F5F1E
:10B020003F4F45E158E161E178E18DE098E10E9410
:10B03000F74C80911B0590911C05A0911D05B091C6
:10B040001E0580930D1890930E18A0930F18B093BF
:10B0500010188091170590911805A0911905B091CD
:10B060001A058093111890931218A0931318B09397
:10B07000141819821A821B821C829E012F5F3F4F77
:10B0800045E158E161E178E18DE098E10E94F74CFB
:10B090006096FFAD6097F11114C0109239041092C0
:10B0A00038040E949A7D80E090E00E94467C09C0AE
:10B0B0002FADF42C052D162DE72C24300CF032CBBF
:10B0C0001FCBCC5ADF4F0FB6F894DEBF0FBECDBFFB
:10B0D000DF91CF911F910F91FF90EF90DF90CF9074
:10B0E000BF90AF909F908F907F906F905F904F90A8
:10B0F0003F902F9008951F920F920FB60F92112438
:10B100000BB60F922F933F938F939F93EF93FF93E1
:10B1100020919A0E30919B0E80919C0E90919D0EE5
:10B120002817390731F4809131018F7D80933101E7
:10B1300014C0E0919C0EF0919D0EE65EF14F2081CF
:10B1400080919C0E90919D0E01968F7799279093F8
:10B150009D0E80939C0E20933601FF91EF919F915D
:10B160008F913F912F910F900BBE0F900FBE0F90BC
:10B170001F9018951F920F920FB60F9211240BB6C5
:10B180000F922F934F935F938F939F93EF93FF9320
:10B190008091300182FD1CC02091360180911E0FEC
:10B1A00090911F0F4091200F5091210F01968F77A2
:10B1B00099274817590771F0E0911E0FF0911F0F62
:10B1C000E256F14F208390931F0F80931E0F02C011
:10B1D00080913601FF91EF919F918F915F914F91F7
:10B1E0002F910F900BBE0F900FBE0F901F901895D0
:10B1F0000E948AF13FB7F8948091E4069091E506A9
:10B20000A091E606B091E70626B5A89B05C02F3FA2
:10B2100019F00196A11DB11D3FBFBA2FA92F982F7C
:10B220008827820F911DA11DB11DBC01CD0142E0F7
:10B23000660F771F881F991F4A95D1F708952FB77A
:10B24000F8946091E0067091E1068091E206909199
:10B25000E3062FBF08951F920F920FB60F9211248D
:10B260002F933F938F939F93AF93BF938091E0066B
:10B270009091E106A091E206B091E3063091DF06DD
:10B2800023E0230F2D3720F40196A11DB11D05C029
:10B2900026E8230F0296A11DB11D2093DF0680939F
:10B2A000E0069093E106A093E206B093E306809156
:10B2B000E4069091E506A091E606B091E7060196B6
:10B2C000A11DB11D8093E4069093E506A093E606C8
:10B2D000B093E706BF91AF919F918F913F912F91CE
:10B2E0000F900FBE0F901F9018951F920F920FB6E0
:10B2F0000F9211240BB60F922F933F934F935F93AE
:10B300006F937F938F939F93AF93BF93EF93FF932D
:10B3100080912F0590913005A0913105B0913205B3
:10B32000892B8A2B8B2B59F190912E05E0912C05BE
:10B33000F0912D0580818927808380912F05909140
:10B340003005A0913105B0913205181619061A067C
:10B350001B060CF056C080912F0590913005A091EE
:10B360003105B09132050197A109B10980932F05EC
:10B3700090933005A0933105B093320542C080917F
:10B380001902E7E6F8E1E4919FEF90931902E230A9
:10B39000C9F050F4EE2399F0E13081F590916F00FF
:10B3A0009D7F90936F002AC0E43019F1E0F0E53002
:10B3B00029F5909173009D7F909373001FC01092A8
:10B3C0006E001CC0909170009D7F9093700091E082
:10B3D0009093B0009091B100987F94609093B100E9
:10B3E0001092B3000BC0909171009D7F90937100FB
:10B3F00005C0909172009D7F9093720060E00E9462
:10B400001CC6FF91EF91BF91AF919F918F917F915A
:10B410006F915F914F913F912F910F900BBE0F90C5
:10B420000FBE0F901F9018952F923F924F925F92F0
:10B430006F927F928F929F92AF92BF92CF92DF9244
:10B44000EF92FF920F931F93CF93DF93CDB7DEB7A9
:10B45000C857D1090FB6F894DEBF0FBECDBFE0913B
:10B46000820FF091830FEF2B11F00C94D462289689
:10B47000DFAECEAE28976E2C79016A015B01FC012C
:10B4800020813181428153816C962CAF3DAF4EAF0C
:10B490005FAF6C972091F1173091F2174091F3173D
:10B4A0005091F4176C966CAD7DAD8EAD9FAD6C97E1
:10B4B0000E9462EA0E94ABF0E0966CAF7DAF8EAF67
:10B4C0009FAFE097D5018D919D910D90BC91A02DDE
:10B4D000A0968CAF9DAFAEAFBFAFA0972091F517F0
:10B4E0003091F6174091F7175091F817BC01CD0134
:10B4F0000E9462EA0E94ABF0E4966CAF7DAF8EAF23
:10B500009FAFE497D6012D913D914D915C91A4960A
:10B510002CAF3DAF4EAF5FAFA4972091F91730919C
:10B52000FA174091FB175091FC17A4966CAD7DADB6
:10B530008EAD9FADA4970E9462EA0E94ABF0E896A0
:10B540006CAF7DAF8EAF9FAFE897D7012D913D9146
:10B550004D915C9122962CAF3DAF4EAF5FAF2297DD
:10B560002091FD173091FE174091FF175091001860
:10B5700022966CAD7DAD8EAD9FAD22970E9462EAA2
:10B580000E94ABF060966CAF7DAF8EAF9FAF6097BF
:10B590008091250783FF1CC060962CAD3DAD4EAD5C
:10B5A0005FAD609720936D0930936E0940936F09EA
:10B5B0005093700922968CAD9DADAEADBFAD229774
:10B5C00080935D0990935E09A0935F09B093600931
:10B5D000D801BC91B9A7F801F181F9ABD801129655
:10B5E000BC91BEABF801F381FAAF80913B09909119
:10B5F0003C09891B8F708F3019F40E94EAAAF5CF9D
:10B6000000913B09E9960FAFE99780913B09082F1C
:10B6100010E01CA30BA38091610990916209A09195
:10B620006309B0916409E0968CAC9DACAEACBFAC44
:10B63000E097881A990AAA0ABB0A80916509909135
:10B640006609A0916709B0916809E4962CAC3DACFD
:10B650004EAC5FACE497281A390A4A0A5B0A80911B
:10B66000690990916A09A0916B09B0916C09E896FB
:10B670002CAD3DAD4EAD5FADE897281B390B4A0BA5
:10B680005B0B2DA33EA34FA358A780916D0990910A
:10B690006E09A0916F09B091700960960CAD1DAD57
:10B6A0002EAD3FAD6097081B190B2A0B3B0B0DA766
:10B6B0001EA72FA738AB012B022B032B09F4BCC00C
:10B6C0008091240781114BC0609150047091510406
:10B6D00080915204909153040E94BEEF2091250264
:10B6E00030912602621773070CF039C060962CADBA
:10B6F0003DAD4EAD5FAD609720936D0930936E09FF
:10B7000040936F095093700922968CAD9DADAEADFC
:10B71000BFAD229780935D0990935E09A0935F0966
:10B72000B0936009E1E8FAE184918F010F5F1F4F48
:10B73000811103C0EBEDF9E104C00E94A78AF80172
:10B74000F3CF84918F010F5F1F4F882321F00E9458
:10B75000A78AF801F6CF1DA61EA61FA618AA94E078
:10B76000699E800111240F5D1D4F6DA57EA58FA5DB
:10B7700098A90E9403EAD8012D913D914D915C91C9
:10B780000E9462EA6B017C0120E030E0A9010E9486
:10B79000A0F087FF04C0F7FAF094F7F8F0946091F6
:10B7A000FD177091FE178091FF17909100180E946D
:10B7B000BEEF9B01AC01A8ECB0E00E945AEE0E94E3
:10B7C00003EAA70196010E94FDE987FF39C0609650
:10B7D0000CAD1DAD2EAD3FAD609700936D0910937C
:10B7E0006E0920936F093093700922962CAD3DAD00
:10B7F0004EAD5FAD229720935D0930935E09409373
:10B800005F0950936009E1E8FAE184918F010F5FCD
:10B810001F4F811103C0ECEBF9E104C00E94A78A1D
:10B82000F801F3CF84918F010F5F1F4F882321F020
:10B830000E94A78AF801F6CF1DA61EA61FA618AA69
:10B84000D501C4018827B7FD83959927AA27BB276F
:10B85000782E57FE03C0382F3260732E8DA19EA123
:10B86000AFA1B8A5B7FF03C0972D9460792E0DA5A1
:10B870001EA52FA538A937FF03C0172D1860712EFC
:10B8800024E0629E800111240F5D1D4F6DA57EA5F1
:10B890008FA598A90E9403EAD8012D913D914D9161
:10B8A0005C910E9462EA6B017C0120E030E0A9011A
:10B8B0000E94A0F087FF04C0C701B601905802C0E3
:10B8C000C701B60120E030E040E05FE30E947AEE7D
:10B8D0000E94C3EF6AAB7BAB8CAB9DAB88E60BA140
:10B8E0001CA1809FF001819FF00D1124EA52FF4EB0
:10B8F0001082EA5BFF4F7082B501A401B7FE07C05A
:10B9000044275527BA01481959096A097B0988E66D
:10B910000BA11CA1809FF001819FF00D1124EA5220
:10B92000FF4E458B568B678B708F2C962CAE3DAEA1
:10B930004EAE5FAE2C9757FE0DC088279927DC01CD
:10B9400082199309A409B5092C968CAF9DAFAEAFAF
:10B95000BFAF2C9728E60BA11CA1209FF001219FCF
:10B96000F00D1124EA52FF4E2C968CAD9DADAEAD7C
:10B97000BFAD2C97818F928FA38FB48F0DA11EA185
:10B980002FA138A537FF07C0309520951095019558
:10B990001F4F2F4F3F4FE8E67E2EABA1BCA17A9EF2
:10B9A000F0017B9EF00D1124EA52FF4E058F168F99
:10B9B000278F30A38AA99BA9ACA9BDA981A392A373
:10B9C000A3A3B4A323964FAF2397752EF62FE72F8B
:10B9D0002C968CAD9DADAEADBFAD2C9748175907D9
:10B9E0006A077B0778F429969FAD299723969FAF26
:10B9F00023972A967FAC2A972B96FFAD2B972C96F0
:10BA0000EFAD2C9723968FAD2397972DAF2FBE2F99
:10BA100080179107A207B30710F4D901C8010AA93A
:10BA20001BA92CA93DA980179107A207B30710F401
:10BA3000D901C80128E60BA11CA1209FF001219F7C
:10BA4000F00D1124EA52FF4E85A396A3A7A3B0A739
:10BA50000697A105B10508F4A0C5DF01AE59BF4F97
:10BA600080913604909137048D939C9361A6452B69
:10BA7000462B472B09F05F9888E60BA11CA1809FFD
:10BA8000F001819FF00D1124EA52FF4E818D928DBD
:10BA9000A38DB48D892B8A2B8B2B11F08A98479814
:10BAA00088E60BA11CA1809FF001819FF00D11245D
:10BAB000EA52FF4E858D968DA78DB0A1892B8A2BDA
:10BAC0008B2B31F08091080181708093060147989B
:10BAD0002AA93BA94CA95DA9232B242B252B09F4CA
:10BAE00065C580912A07882319F0815080932A0721
:10BAF000611004C0129880E280932A0760902007AA
:10BB00007090210700912207109123079301A8014B
:10BB100069A579A98EA99AAD0E94FDE987FF04C0A5
:10BB200069A679AA0EAB1AAFC501B4010E9403EA57
:10BB30002091C2103091C3104091C4105091C51093
:10BB40000E9462EA26966CAF7DAF8EAF9FAF2697BC
:10BB5000698B7A8B8B8B9C8BC201B1010E9403EAAB
:10BB60002091C6103091C7104091C8105091C91053
:10BB70000E9462EA2B013C016D8B7E8B8F8B988F2C
:10BB80006DA17EA18FA198A50E9403EA2091CA1001
:10BB90003091CB104091CC105091CD100E9462EAB0
:10BBA0004B015C01698F7A8F8B8F9C8F2091CE1017
:10BBB0003091CF104091D0105091D110C701B601F3
:10BBC0000E9462EA6B017C016D8F7E8F8F8F98A33C
:10BBD00088E60BA11CA1809FF001819FF00D11242C
:10BBE000EA52FF4E258936894789508D2DA33EA301
:10BBF0004FA358A7263031054105510508F4DFC48D
:10BC00002896AEADBFAD2897CD90DD90ED90FC901D
:10BC100020E030E0A901C701B6010E94FDE98111D1
:10BC2000EDC426962CAD3DAD4EAD5FAD2697CA0155
:10BC3000B9010E9462EA6B017C01A3019201C30178
:10BC4000B2010E9462EA9B01AC01C701B6010E94E9
:10BC50007AEE6B017C01A5019401C501B4010E943B
:10BC600062EA9B01AC01C701B6010E947AEE0E9414
:10BC7000E5F028E60BA11CA1209FF001219FF00D0B
:10BC80001124EA52FF4E658776878787908B88E676
:10BC90000BA11CA1809FF001819FF00D1124EA529D
:10BCA000FF4E4584568467847088A301920160E04A
:10BCB00070E080E89FE30E9456EF64966CAF7DAF22
:10BCC0008EAF9FAF649729A539A94EA95AAD0E949E
:10BCD00062EA4B015C0180913B0990913909891B13
:10BCE0008F7027968FAF2797A501940160E074E2CB
:10BCF00084E799E40E9456EF0E94ABF06B017C014F
:10BD000027968FAD27978250863008F486C4A50108
:10BD10009401C301B2010E9462EA9B01AC010E943E
:10BD200062EA68966CAF7DAF8EAF9FAF689788E68A
:10BD3000ABA1BCA18A9F80018B9F100D11240A52D8
:10BD40001F4E68962CAD3DAD4EAD5FAD6897D801E6
:10BD500011962D933D934D935C93149795962D9149
:10BD60003D914D915C9198972EAB3FAB48AF59AF49
:10BD7000CA01B9010E9401EA6AAF7BAF8CAF9DAFE7
:10BD80009B01AC01C501B4010E9462EA0E9440EF30
:10BD90000E94C3EFA8966CAF7DAF8EAF9FAFA89700
:10BDA000F801EE5AFF4F60837183828393838E0183
:10BDB0000F5E1F4F2A961FAF0EAF2A970051110931
:10BDC00024961FAF0EAF249708E017E0AC961FAF84
:10BDD0000EAFAC978E010F5D1F4F1AA309A32496D7
:10BDE0000EAD1FAD2497AA961FAF0EAFAA97312CA8
:10BDF000212C10E819A70FE309AB2A96AEADBFAD11
:10BE00002A972D913D914D915D912A96BFAFAEAF8E
:10BE10002A97C501B4010E9462EA6B017C01AA96CF
:10BE2000EEADFFADAA976193719381939193AA961A
:10BE3000FFAFEEAFAA9720E030E0A9010E94A0F08A
:10BE400087FF04C0F7FAF094F7F8F094AC96AEAD23
:10BE5000BFADAC974D905D906D907D90AC96BFAFAF
:10BE6000AEAFAC97A7019601C301B2010E94FDE9F4
:10BE700087FD0DC409A11AA12A962EAD3FAD2A97C0
:10BE80000217130709F0B9CF20E030E040E85FE384
:10BE9000632D722D89A599A90E94FDE987FF58C0DD
:10BEA0007E0131E1E30EF11C24960EAD1FAD249707
:10BEB000232D322D49A559A9D8016D917D918D91E0
:10BEC0009C910E9462EAF80161937193819391932E
:10BED0008F01EE16FF0661F728E60BA11CA1209F3B
:10BEE000C001219F900D11249C012A523F4E7901DF
:10BEF00089010E5A1F4FA8966CAD7DAD8EAD9FADDA
:10BF0000A8970E9401EA232D322D49A559A90E9424
:10BF100062EA0E94C3EFD8016D937D938D939C9349
:10BF20001397232D322D49A559A9632D722D89A56B
:10BF300099A90E9462EA68962CAD3DAD4EAD5FAD09
:10BF400068970E9462EAF701618372838383948316
:10BF50002AAD3BAD4CAD5DAD64966CAD7DAD8EADA7
:10BF60009FAD64970E9462EA69A77AA78BA79CA7F6
:10BF70000DA11EA12FA138A5012B022B032B09F027
:10BF80009EC388E62BA13CA1829F8001839F100D58
:10BF900011240A521F4EF801818D928DA38DB48D0C
:10BFA000892B8A2B8B2B09F08AC3858D968DA78DC3
:10BFB000B0A1892B8A2B8B2B09F081C32091040718
:10BFC00030910507409106075091070769A57AA5AA
:10BFD0008BA59CA50E9462EA0E9440EF0E94C3EFDD
:10BFE0002B013C01F801E95BFF4F108288E62BA191
:10BFF0003CA1829F8001839F100D11240A521F4E85
:10C00000F801E25AFF4F4082518262827382C3017B
:10C01000B2010E9401EA29A53AA54BA55CA50E94A0
:10C0200056EF6AAF7BAF8CAF9DAFD80151966D9341
:10C030007D938D939C935497F801E95BFF4F80812A
:10C04000882381F17801B8E4EB0EF11C379620913A
:10C05000F8063091F9064091FA065091FB0660818E
:10C060007181828193810E9462EA2AAD3BAD4CAD21
:10C070005DAD0E9462EA2091FD173091FE1740915C
:10C08000FF17509100180E9462EA9B01AC0160E02A
:10C0900074E284EF99E40E9456EF0E94C3EFF70127
:10C0A0007183608388E60BA11CA1809FF001819FB2
:10C0B000F00D1124EA52FF4E2181328143815481D7
:10C0C0002C962CAF3DAF4EAF5FAF2C97CA01B90194
:10C0D0000E94E5F0362E272E8C0148EE56E062963F
:10C0E0005FAF4EAF62973E0151E1650E711C88EE65
:10C0F00096E09FAB8EAB24964EAC5FAC24973DA6EA
:10C100002DA209A719AB1AAAD201CD90DD90ED900E
:10C11000FD902D0120E030E0A901C701B6010E9489
:10C12000A0F087FF04C0F7FAF094F7F8F094EEA9B6
:10C13000FFA981909190A190B190FFABEEABA701C8
:10C140009601C501B4010E94FDE987FDD8C56414BC
:10C150007504D1F627965FAD2797552309F448C695
:10C16000C0903D09D0903E09E0903F09F090400911
:10C170002DEB37E346E855E3C701B6010E94FDE920
:10C1800087FD36C6C701B6010E94E5F06B017C0150
:10C190009B01AC01632D722DC8010E94FDE987FD52
:10C1A00003C03C2C2D2C87019601A701632D722D15
:10C1B000C8010E9456EF68966CAF7DAF8EAF9FAFFF
:10C1C000689781E499E028969FAF8EAF289720E08A
:10C1D00030E040E85FE32AAB3BAB4CAB5DAB1EAA63
:10C1E0002896AEADBFAD28972D913D914D915D91B3
:10C1F0002896BFAFAEAF289768966CAD7DAD8EAD7B
:10C200009FAD68970E9462EA4B015C012496EEADF7
:10C21000FFAD2497C190D190E190F1902496FFAFAB
:10C22000EEAF2497FEA9FF2391F02AA93BA94CA9C0
:10C230005DA90E9462EA4B015C012AA93BA94CA9B5
:10C240005DA9C701B6010E9462EA6B017C01A701EA
:10C250009601C501B4010E94A0F020E030E0A901E0
:10C2600018160CF092C5C701B6010E94A0F018166E
:10C270000CF486C520E030E0A901C501B4010E949C
:10C28000FDE987FD7DC52601370177FA709477F8BF
:10C290007094A3019201C501B4010E94A0F0181688
:10C2A00014F4240135016296AEADBFAD6297CD9016
:10C2B000DD90ED90FD906296BFAFAEAF6297A301A7
:10C2C0009201C701B6010E94FDE987FF15C0A301D5
:10C2D0009201C701B6010E9456EF9B01AC016AA909
:10C2E0007BA98CA99DA90E9462EA6AAB7BAB8CAB4F
:10C2F0009DABBEA9BF5FBEABE1E5F9E028962EADD0
:10C300003FAD2897E217F30709F06ACF3EA9332320
:10C3100061F02AA93BA94CA95DA9632D722DC80122
:10C320000E9462EA362E272E8C0124EA30E74DE780
:10C330005FE3632D722DC8010E9462EA6B017C01EC
:10C34000209126073091270740912807509129070F
:10C350000E94FDE987FD42C58DA59DA1A9A5B9A9AA
:10C360008093260790932707A0932807B093290767
:10C3700028E64BA15CA1249FC001259F900D1124AC
:10C38000DC01AA52BF4E7D01232D322DA801632D61
:10C39000722DC8010E9462EAF70161877287838764
:10C3A00094876AAD7BAD8CAD9DAD90589B01AC017F
:10C3B0000E947AEED7011D962D913D914D915C9191
:10C3C00050970E9462EA9B01AC016BE077ED83E23B
:10C3D0009BE30E9479EE9B01AC018BE097EDA3E219
:10C3E000BBE3F70185839683A783B08710812C96E2
:10C3F0006CAD7DAD8EAD9FAD2C970E94FDE91816FA
:10C400000CF4FBC483E0182B88E62BA13CA1829F8F
:10C41000F001839FF00D1124EA52FF4E108380E15A
:10C42000FE013196A1E4B9E001900D928A95E1F701
:10C430002C968CAD9DADAEADBFAD2C9780933D09D4
:10C4400090933E09A0933F09B0934009E0960CAD4C
:10C450001DAD2EAD3FADE0970093610910936209C9
:10C460002093630930936409E4962CAD3DAD4EAD45
:10C470005FADE4972093650930936609409367099F
:10C4800050936809E8968CAD9DADAEADBFADE89711
:10C490008093690990936A09A0936B09B0936C0922
:10C4A00060960CAD1DAD2EAD3FAD609700936D094C
:10C4B00010936E0920936F09309370096C962CAD20
:10C4C0003DAD4EAD5FAD6C9720935109309352094D
:10C4D0004093530950935409A0968CAD9DADAEADD9
:10C4E000BFADA0978093550990935609A093570923
:10C4F000B0935809A4960CAD1DAD2EAD3FADA497D9
:10C500000093590910935A0920935B0930935C09F1
:10C5100022962CAD3DAD4EAD5FAD229720935D09C7
:10C5200030935E0940935F095093600990913B09F5
:10C5300080913C09981303C084E680933809E996FA
:10C540008FADE9978F5F8F7080933B0980913B0996
:10C5500090913A0981508F70891351C410913C0910
:10C560001BA300913B090DA728E61BA10DA51013E5
:10C57000D1C4812C912CA12CB12C1DA219A619AAD1
:10C580001EAE212C312C00E010E02DA53BA1231381
:10C59000CEC42114310409F07FC580916F00826000
:10C5A00080936F0081E0ECC680E0EAC660901C07D3
:10C5B00070901D0700911E0710911F07A7CA818D5B
:10C5C000928DA38DB48D0697A105B10508F018CB07
:10C5D000858D968DA78DB0A10697A105B10508F0B0
:10C5E0000FCB20E030E0A901C701B6010E94A0F006
:10C5F00087FF04C0F7FAF094F7F8F09488E60BA1EF
:10C600001CA1809FF001819FF00D1124EA52FF4E82
:10C61000C586D686E786F08A3ACB80911807909136
:10C620001907A0911A07B0911B07C816D906EA0688
:10C63000FB0608F06CCB8C199D09AE09BF09BC0143
:10C64000CD01660F771F881F991F27964FAD27973B
:10C65000042F10E020E030E0A90198010E941CEEB8
:10C66000CA01B9010E9401EA0E94ABF06C0D7D1D68
:10C670008E1D9F1D0E9401EA9B01AC0160E074E2E7
:10C6800084E799E40E9456EF4B015C0140CBA7017F
:10C690009601C301B2010E9456EF7B018C019B0100
:10C6A000AC01632D722D89A599A90E94A0F01816DE
:10C6B0000CF0E0CB3E2C2F2C09A719ABDBCB0AA941
:10C6C0001BA92CA93DA9012B022B032B49F020917A
:10C6D000000730910107409102075091030708C0FD
:10C6E0002091FC063091FD064091FE065091FF0618
:10C6F00069A57AA58BA59CA50E9462EA0E9440EFDD
:10C700000E94C3EF2B013C012AA93BA94CA95DA9BA
:10C71000232B242B252BC9F020E030E0A9016091C8
:10C72000F8067091F9068091FA069091FB060E9436
:10C73000FDE9882351F081E00DA51EA52FA538A99C
:10C7400010161106120613060CF080E098E62BA1D5
:10C750003CA1929F8001939F100D11240A521F4EFD
:10C76000180137E4230E311CD1018C93882309F47E
:10C77000B3C0209151093091520940915309509111
:10C7800054096C966CAD7DAD8EAD9FAD6C970E94DB
:10C7900079EE6DA77EA78FA798AB209155093091B0
:10C7A00056094091570950915809A0966CAD7DAD3E
:10C7B0008EAD9FADA0970E9479EE4B015C01209158
:10C7C000590930915A0940915B0950915C09A4962E
:10C7D0006CAD7DAD8EAD9FADA4970E9479EE6B01DF
:10C7E0007C012DA53EA54FA558A9CA01B9010E94FB
:10C7F00062EA6DA77EA78FA798ABA5019401C5013A
:10C80000B4010E9462EA9B01AC016DA57EA58FA5D3
:10C8100098A90E947AEE4B015C01A7019601C7011D
:10C82000B6010E9462EA9B01AC01C501B4010E94FD
:10C830007AEE0E94E5F06B017C0120915D09309158
:10C840005E0940915F095091600922966CAD7DAD03
:10C850008EAD9FAD22970E9479EEA70196010E94AE
:10C8600056EF6B017C01F801E25BFF4F608371833F
:10C870008283938320E030E040E450E40E94A0F003
:10C8800018161CF4F101108227C02091F80630918F
:10C89000F9064091FA065091FB06C701B6010E94C5
:10C8A00062EA9B01AC016091F4067091F5068091FB
:10C8B000F6069091F7060E9456EF29A53AA54BA5DA
:10C8C0005CA50E9462EA0E94C3EF641575058605A7
:10C8D000970510F42B013C0180919E1090919F10C0
:10C8E000A091A010B091A1100EA91FA928AD39AD3B
:10C8F00080179107A207B30708F4DFC02DA13EA15E
:10C900004FA158A5232B242B252B41F16091A21078
:10C910007091A3108091A4109091A51064157505D5
:10C9200086059705D8F42EA93FA948AD59AD0E94B8
:10C930000DEE6B017C012DA13EA14FA158A5C301B5
:10C94000B2010E940DEEC616D706E806F90630F4CD
:10C95000C701B6010E941CEE29013A0188E60BA12D
:10C960001CA1809FF001819FF00D1124EA52FF4E1F
:10C97000C18CD28CE38CF48CC114D104E104F10499
:10C9800031F16091A6107091A7108091A81090913C
:10C99000A9106415750586059705C8F42EA93FA949
:10C9A00048AD59AD0E940DEE4B015C01A701960107
:10C9B000C301B2010E940DEE86169706A806B906BD
:10C9C00030F4C501B4010E941CEE29013A0188E649
:10C9D0000BA11CA1809FF001819FF00D1124EA5250
:10C9E000FF4EC58CD68CE78CF0A0C114D104E104B5
:10C9F000F10431F16091AA107091AB108091AC10EC
:10CA00009091AD106415750586059705C8F42EA99B
:10CA10003FA948AD59AD0E940DEE4B015C01A70145
:10CA20009601C301B2010E940DEE86169706A80674
:10CA3000B90630F4C501B4010E941CEE29013A0187
:10CA400088E60BA11CA1809FF001819FF00D1124AD
:10CA5000EA52FF4EC1A0D2A0E3A0F4A0C114D104B9
:10CA6000E104F10409F4C2CA6091AE107091AF10F4
:10CA70008091B0109091B1106415750586059705E9
:10CA800008F0B4CA2EA93FA948AD59AD0E940DEED9
:10CA90004B015C01A7019601C301B2010E940DEE9A
:10CAA00086169706A806B90608F0A0CAC501B40103
:10CAB0000E941CEE29013A0199CA2DA13EA14FA165
:10CAC00058A5232B242B252BC9F16091A21070911E
:10CAD000A3108091A4109091A5106415750586058A
:10CAE000970560F50E9401EA2AAD3BAD4CAD5DAD06
:10CAF0000E9462EA6B017C016DA17EA18FA198A5C5
:10CB00000E9401EA4B015C01C301B2010E9401EAEB
:10CB1000A50194010E9462EA9B01AC01C701B60124
:10CB20000E94FDE987FF0AC0A5019401C701B60173
:10CB30000E9456EF0E94C3EF2B013C0188E60BA137
:10CB40001CA1809FF001819FF00D1124EA52FF4E3D
:10CB5000818C928CA38CB48C81149104A104B104B7
:10CB6000B9F16091A6107091A7108091A8109091D2
:10CB7000A910641575058605970550F50E9401EA10
:10CB80002AAD3BAD4CAD5DAD0E9462EA6B017C010C
:10CB9000C501B4010E9401EA4B015C01C301B2016D
:10CBA0000E9401EAA50194010E9462EA9B01AC0186
:10CBB000C701B6010E94FDE987FF0AC0A5019401E3
:10CBC000C701B6010E9456EF0E94C3EF2B013C0142
:10CBD00088E60BA11CA1809FF001819FF00D11241C
:10CBE000EA52FF4E858C968CA78CB0A081149104DC
:10CBF000A104B104B9F16091AA107091AB108091B9
:10CC0000AC109091AD10641575058605970550F52B
:10CC10000E9401EA2AAD3BAD4CAD5DAD0E9462EAD7
:10CC20006B017C01C501B4010E9401EA4B015C016A
:10CC3000C301B2010E9401EAA50194010E9462EAC7
:10CC40009B01AC01C701B6010E94FDE987FF0AC044
:10CC5000A5019401C701B6010E9456EF0E94C3EFDF
:10CC60002B013C0188E60BA11CA1809FF001819F54
:10CC7000F00D1124EA52FF4EC1A0D2A0E3A0F4A00F
:10CC8000C114D104E104F10409F4B0C96091AE10FB
:10CC90007091AF108091B0109091B110641575052E
:10CCA0008605970508F0A2C90E9401EA2AAD3BADAE
:10CCB0004CAD5DAD0E9462EA4B015C01C701B6015B
:10CCC0000E9401EA6B017C01C301B2010E9401EAEA
:10CCD000A70196010E9462EA9B01AC01C501B40163
:10CCE0000E94FDE987FF82C9A7019601C501B40131
:10CCF0000E9456EF0E94C3EF2B013C0177C9FAA9AD
:10CD0000FF2331F1A5019401632D722DC8010E940A
:10CD100062EA4B015C012DA53DA149A559A9C701B6
:10CD2000B6010E9462EA9B01AC01C501B4010E94F8
:10CD3000FDE987FF22C0A7019601C501B4010E9449
:10CD400056EF6DA77DA389A799AB21E02AABFFC958
:10CD5000A7019601C501B4010E9456EF9B01AC01E9
:10CD60006DA57DA189A599A90E9462EA6DA77DA301
:10CD700089A799AB31E03AABEAC941E04AABE7C9D0
:10CD8000A7019601C501B40113C0C701B6010E94F5
:10CD9000FDE987FD09C020E030E0A901C501B4012B
:10CDA0000E94A0F018164CF4A5019401C701B60129
:10CDB0000E9479EE2B013C0176CA2401350177FAF5
:10CDC000709477F87094A3019201C701B6010E9494
:10CDD000FDE987FD68CA2601370165CA2DA53DA179
:10CDE00049A559A9C701B6010E94FDE987FFB4CA48
:10CDF0003DA42DA009A519A9AFCA81E004CBF090EC
:10CE00003B098FEF8F0D8F708BA3B0903A09809103
:10CE10003B09B81609F454C0C12CD12C0BA10B1539
:10CE200009F44EC0602E712C28E6269D8001279DB6
:10CE3000100D11240A521F4ED8018C9183FD2BC076
:10CE40000EAF1AAB0115110541F11996BC91BDA7A2
:10CE5000F801F285FDA3D8011B96BC91B9A7F80192
:10CE6000F485F9ABD80115962D903D904D905C90CE
:10CE70001897A20191016DA57DA189A59F2F0E9400
:10CE8000FDE9811186C1C114D10439F0F601808118
:10CE900080FD7FC102C0CEAEDAAA8BA181508F7017
:10CEA0008BA380913A098B1103C0CEACDAA8B6CF20
:10CEB0000BA10B1529F081E08B0D8F70B82EF1CFEF
:10CEC00010913A091BA3C12CD12C80913B090BA1D5
:10CED000801709F443CB802E912C28E6289D8001F1
:10CEE000299D100D11240A521F4ED8018C9183FDEB
:10CEF0000AC05801C114D10439F0C6010E948D85C1
:10CF0000811102C0C5C156018BA18F5F8F708BA3A9
:10CF10006501DBCF802F81508F70289FF001112495
:10CF2000EA52FF4E908193FF24CB8DA71ECB48E69B
:10CF3000439FC0011124DC01AA52BF4E1D018C91F8
:10CF400083FD19C015966D917D918D919C911897D7
:10CF50000E94E5F0F62EE72ED82EC92E01151105F8
:10CF600009F48CC0F801808180FD0AC0D1018C9148
:10CF700080FD06C083C0FDA0E9A4D9A8CEAC83C0C3
:10CF8000F801808181608083C8010E948D858111B4
:10CF900071C0F80161817281838194810E94E5F002
:10CFA0002B013C019B01AC0160E070E080E89FE355
:10CFB0000E9456EF4B015C019B01AC016F2D7E2D51
:10CFC0008D2D9C2D0E9462EA69837A838B839C83DA
:10CFD0002DA139A549A95EADC501B4010E9462EA3F
:10CFE000698B7A8B8B8B9C8BAE014F5F5F4FBE0141
:10CFF0006F5E7F4FC8010E949BBAF801E95BFF4F4B
:10D0000080818823B9F12091F8063091F90640918A
:10D01000FA065091FB063796608171818281938177
:10D020000E9462EA2091FD173091FE174091FF1790
:10D03000509100180E9462EA4B015C019B01AC0117
:10D04000C301B2010E9462EA0E94C3EFF801E65BED
:10D05000FF4F71836083A50194016F2D7E2D8D2D6F
:10D060009C2D0E9462EA0E94C3EFF801E45BFF4F2F
:10D0700071836083D8018C918E7F8C938F2C9E2C32
:10D08000AD2CBC2C81018BA18F5F8F708BA3FDA277
:10D09000E9A6D9AACEAE79CAF101808181608083E8
:10D0A000C8010E948D8581116FC0D10111966D91CB
:10D0B0007D918D919C9114970E94E5F06B017C010C
:10D0C0009B01AC0160E070E080E89FE30E9456EFB6
:10D0D0002B013C012DEC3CEC4CE45DE30E9462EA48
:10D0E00069837A838B839C839401A501C301B20178
:10D0F0000E9462EA698B7A8B8B8B9C8BAE014F5FAF
:10D100005F4FBE016F5E7F4FC1010E949BBAF1016C
:10D11000E95BFF4F80818823B9F12091F8063091B7
:10D12000F9064091FA065091FB06379660817181AD
:10D13000828193810E9462EA2091FD173091FE174F
:10D140004091FF17509100180E9462EA4B015C0168
:10D150009B01AC01C701B6010E9462EA0E94C3EFC5
:10D16000F101E65BFF4F718360832DEC3CEC4CE4F6
:10D170005DE3C501B4010E9462EA0E94C3EFF101C0
:10D18000E45BFF4F71836083F10180818E7F808338
:10D1900004CA28E6269DF001279DF00D1124EA52CD
:10D1A000FF4E808181FD43C0C114D10441F0D601FE
:10D1B0001596CD90DD90ED90FC90189708C08BE00F
:10D1C000C82E87EDD82E83E2E82E8BE3F82EB8E642
:10D1D000B69DF001B79DF00D1124EA52FF4E8189F2
:10D1E0009289A389B489BC01CD0190589B01AC01FF
:10D1F0000E947AEEF80125853685478550890E9480
:10D2000062EA9B01AC01C701B6010E9479EEE62EED
:10D21000872E982EA92E262F372F482F592F6DA5F0
:10D220007DA189A599A90E94FDE987FF04C0EDA40D
:10D230008DA099A4A9A82E2D382D492D5A2DC201B3
:10D24000B1010E94FDE9882309F427CEF8E6F69D96
:10D25000C001F79D900D11249C012A523F4E690197
:10D26000D9018C9181608C93C8010E948D8588239F
:10D2700029F0F60180818E7F80830FCE8E2D982D30
:10D28000A92DBA2DF60185839683A783B08705CE95
:10D29000D6018C9181FD52C0D60115962D913D91FC
:10D2A0004D915C9118972DA73EA74FA758AB15013C
:10D2B000B5E02B0E311CF8014580568067807084E4
:10D2C000A30192016DA57EA58FA598A90E94FDE9F5
:10D2D00087FF34C0F60181899289A389B489BC0192
:10D2E000CD0190589B01AC010E947AEED6011D96AB
:10D2F0002D913D914D915C9150970E9462EA9B0166
:10D30000AC016DA57EA58FA598A90E9479EE6B0151
:10D310007C019B01AC01C301B2010E94A0F0181670
:10D320006CF4D8018C9181608C93C5010E948D852D
:10D330008823E1F0F80180818E7F808318E6189DB4
:10D34000F001199DF00D1124EA52FF4E218532851E
:10D350004385548565817681878190850E94FDE9AA
:10D360008111D2CD0BA100933A09CECDD101CD923E
:10D37000DD92ED92FC9213970BA100933A09DECF58
:10D38000C858DF4F0FB6F894DEBF0FBECDBFDF9198
:10D39000CF911F910F91FF90EF90DF90CF90BF90B2
:10D3A000AF909F908F907F906F905F904F903F9045
:10D3B0002F90089580913B0990913C09891B8F70B3
:10D3C0008F3019F40E94EAAAF5CF80913B098F5F54
:10D3D0008F70E0913B0998E69E9FF0011124EA527C
:10D3E000FF4EDF011D929A95E9F798E090834091F6
:10D3F0006109509162096091630970916409458BDC
:10D40000568B678B708F40916509509166096091CA
:10D41000670970916809418F528F638F748F4091B3
:10D42000690950916A0960916B0970916C09458F87
:10D43000568F678F70A340916D0950916E0960916E
:10D440006F097091700941A352A363A374A3209143
:10D450003B0990913C09291303C094E69093380945
:10D4600080933B0980916F00826080936F000895E4
:10D4700090913B0980913C09981306C08091820FDE
:10D480009091830F892B19F00E94EAAAF1CF089599
:10D490008F929F92AF92BF92CF92DF92EF92FF92C4
:10D4A0001F93CF93DF93C82F8BE59BE090933709B1
:10D4B000809336091092770B82E090E0A0E0B0E014
:10D4C0008093600B9093610BA093620BB093630BFE
:10D4D00010923509109231091092320910923309D5
:10D4E000109234098FEF9FEFDC0180932D09909308
:10D4F0002E09A0932F09B0933009CC2379F1C530C0
:10D5000008F0F8C040E060E070E0CB010E9448D530
:10D51000882309F4EFC020E1C29FC0011124835E7B
:10D52000984FFC01E254FE4F20812F7709F0E2C0B2
:10D530003C96408151816281738144365105610579
:10D54000710508F4D7C03497C080D180E280F380A1
:10D55000C114D104E104F10421F4CCC0C12CD12CBC
:10D56000760140E0C701B6010E9448D5182F8823F4
:10D5700009F4C0C080913807909139078115924015
:10D5800009F0B8C0A0913D07AA2309F4B3C0609187
:10D590003B0770913C076115710509F4ABC0209100
:10D5A0003A07222309F4A6C0A093720B2093640BC0
:10D5B00080E030E041E050E0C82FFA01082E02C0C0
:10D5C000EE0FFF1F0A94E2F72E173F0739F08F5F27
:10D5D000C83091F789E080936D0B8CC080936D0B00
:10D5E00020914307309144072115310519F040E09F
:10D5F00050E008C0209151073091520740915307E5
:10D60000509154072093650B3093660B4093670B42
:10D610005093680B46015701860E971EA11CB11C42
:10D620008092730B9092740BA092750BB092760B54
:10D63000E0913E07F0913F07F093790BE093780B70
:10D64000B0E00E945AEE860E971EA81EB91E809268
:10D650007A0B90927B0BA0927C0BB0927D0B85E0B5
:10D66000EE0FFF1F8A95E1F7E150FE4FEF2FFF27E6
:10D67000E6958E0E9F1EA11CB11C80926E0B90929F
:10D680006F0BA092700BB092710B209140073091FC
:10D6900041072115310521F0A90160E070E008C0C3
:10D6A00040914D0750914E0760914F077091500780
:10D6B000D701C60188199909AA09BB09840F951FCA
:10D6C000A61FB71F04C0B695A79597958795CA95CD
:10D6D000D2F78093690B90936A0BA0936B0BB09376
:10D6E0006C0B853F2FE09207A105B10528F48CE073
:10D6F0008093770B10E01AC0853F9F4FA105B105BD
:10D7000010F480E111C08091590790915A07A091BF
:10D710005B07B0915C0780937A0B90937B0BA0938F
:10D720007C0BB0937D0B80E28093770B812FDF9190
:10D73000CF911F91FF90EF90DF90CF90BF90AF906F
:10D740009F908F900895682F82E29FE00C942A4B5F
:10D75000CF92DF92EF92FF921F93CF93DF931092BD
:10D76000BA098091ED09882321F08AEE99E00E94A0
:10D77000C7A210925F0B10925C0B85E380935B0B4A
:10D780000E941F59EB01A89561E080915B0B0E94FC
:10D790004AC68BE59BE00E9428A42398229A219AEE
:10D7A000209A289A85E080935D0B82E58CBD1DBC94
:10D7B0001AE08FEF0E942DA41150D9F720E030E03D
:10D7C000A90160E08BE59BE00E9432A4182F8093B2
:10D7D0005E0B813049F00E941F596C1B7D0B613D2F
:10D7E000774060F381E054C02AEA31E040E050E045
:10D7F00068E08BE59BE00E9432A482FF03C0109397
:10D800005F0B0EC014E00E9440A980935E0B115084
:10D81000D1F78A3A11F082E03BC082E080935F0B3F
:10D8200080915F0B823021F0C12CD12C760105C094
:10D83000C12CD12CE12C80E4F82E20E030E0A901AD
:10D8400067E38BE59BE00E9432A4A701960169E2A1
:10D850008BE59BE00E9432A480935E0B882349F005
:10D860000E941F596C1B7D0B613D774030F38AE0AD
:10D870000FC080915F0B823011F520E030E0A901EC
:10D880006AE38BE59BE00E9432A4882351F088E094
:10D8900080935C0B8BE59BE00E9428A4E1E8FAE111
:10D8A00019C00E9440A9807C803C19F483E08093D9
:10D8B0005F0B0E9440A90E9440A90E9440A98BE5ED
:10D8C0009BE00E9428A410925D0B81E0E1DD8111B4
:10D8D00031C015C08491EF012196882321F00E9468
:10D8E000A78AFE01F7CFE3E7FAE18491EF012196E1
:10D8F000882309F456C00E94A78AFE01F6CF80E073
:10D90000C7DD811117C0ECE6FAE18491EF012196A1
:10D91000882321F00E94A78AFE01F7CFE8E5FAE10B
:10D920008491EF012196882309F43BC00E94A78AC5
:10D93000FE01F6CF60E67BE08AEE99E00E9474A2D9
:10D94000811116C0ECE6FAE18491EF01219688235B
:10D9500021F00E94A78AFE01F7CFE7E4FAE1849163
:10D96000EF0121968823E9F00E94A78AFE01F7CFF4
:10D9700081E08093BA09E1E8FAE18491EF01219610
:10D98000882321F00E94A78AFE01F7CFEBE3FAE19A
:10D990008491EF012196882321F00E94A78AFE013D
:10D9A000F7CF8BE1EAEEF9E0A9E0BAE001900D9241
:10D9B0008A95E1F78091E8099091E9099093080A26
:10D9C0008093070ADF91CF911F91FF90EF90DF9036
:10D9D000CF9008958091C70D823041F486E29AE19C
:10D9E00090932C0780932B070E94D38A0E941F5983
:10D9F0006093CB0D7093CC0D8093CD0D9093CE0D95
:10DA00008091BA09882319F081E08093B90981E0F7
:10DA10008093C70D0895CF93DF931092B90983E0E7
:10DA20008093C70D8091140E8823B1F0EEE1FAE1E6
:10DA30008491EF01882341F0082E000C990B83DEBE
:10DA40002196FE018491F6CF8DE090E07CDE8AE0A5
:10DA500090E0DF91CF9177CEE2E2FAE18491EF019D
:10DA6000882391F3082E000C990B6DDE2196FE01A0
:10DA70008491F6CF8F929F92AF92BF92CF92DF9216
:10DA8000EF92FF920F931F93CF93DF9300D01F92DB
:10DA9000CDB7DEB7FC018381813079F5818181FFCB
:10DAA0002CC081899289A389B489892B8A2B8B2BDD
:10DAB00009F448C07F0140E050E0BA01CF010E9464
:10DAC000DDA18823D1F0F70185889688A788B08CDE
:10DAD000C18CD28C82E090E0A0E0B0E0F6018083BF
:10DAE0009183A283B3839E012F5F3F4FB501A401B1
:10DAF000C6010E9411D6811102C080E03CC000E046
:10DB000010E09801B501A401C6010E9480D58823C8
:10DB1000A1F389809A80AB80BC80F601878980312F
:10DB200041F4F8EF8F16FFEF9F06A104B10460F4F3
:10DB3000DACF88EF88168FEF9806A8068FE0B80630
:10DB400018F4D1CF81E017C0F701158A168A178A19
:10DB5000108E118A128A138A148A818180688183C7
:10DB6000C7010E945FD7882341F240E050E0BA012C
:10DB7000C7010E94DDA10F900F900F900F90DF91D1
:10DB8000CF911F910F91FF90EF90DF90CF90BF90BA
:10DB9000AF909F908F9008951092BC091092B90990
:10DBA0008091850B882321F082E89BE00C94C7A22A
:10DBB00008952F923F924F925F926F927F928F9231
:10DBC0009F92AF92BF92CF92DF92EF92FF920F930C
:10DBD0001F93CF93DF93CDB7DEB7C257D1090FB6EE
:10DBE000F894DEBF0FBECDBF8C013B014A014DB79B
:10DBF0005EB7E1965FAF4EAFE197AD961FAEAD97C2
:10DC00001B0154E0250E311C7E018FE5E80EF11C4E
:10DC100095E6492E92E0592EE0E4F0E0EC0FFD1F6E
:10DC20003496E396FFAFEEAFE397F301878182303E
:10DC300008F462C184859585A685B7858F7199277B
:10DC4000AA27BB27892B8A2B8B2B09F055C1109251
:10DC5000CA094AEC59E0BE016F5F7F4FC1010E94C3
:10DC6000F7D618160CF048C18C85982F9871903112
:10DC700029F42091370C2150223078F42981222375
:10DC800009F43AC1253E89F22E3279F22091CA096F
:10DC90002E3259F28A7049F6B8C04DB75EB7AF96CA
:10DCA0005FAF4EAFAF97BE016F5F7F4FC7010E945E
:10DCB000F2D40115110521F0F801808181119BC07A
:10DCC00021E081E090E0F70101900020E9F7319731
:10DCD000EE19FF098E0F9F1F02964DB75EB7481BC6
:10DCE000590B0FB6F8945EBF0FBE4DBF8DB79EB7F0
:10DCF00001965C01211102C0B80102C062E273E02A
:10DD0000C5010E94DEF1B701C5010E94BFF162E2C8
:10DD100073E0C5010E94BFF125961FAE2597289696
:10DD20001FAE289724961FAE1EAE249722965FAE94
:10DD30004EAE229721E0A701B101E3968EAD9FADD3
:10DD4000E3970E9453A881112AC08091370C81115A
:10DD500026C0E1E8FAE184916F019FEFC91AD90A60
:10DD6000882321F00E94A78AF601F5CFEAE0FAE1C4
:10DD700084916F012FEFC21AD20A882321F00E94EA
:10DD8000A78AF601F5CF6701F60181916F0188231B
:10DD900019F00E94A78AF8CF8AE00E94A78A8BE137
:10DDA000FE01EC5BFF4FDE01959601900D928A9586
:10DDB000E1F724968EAD9FAD24979CA38BA35AA226
:10DDC00049A240E050E0BE016F5D7F4FC501F1DE2A
:10DDD000CE0181960E9480AACE01805C9F4F0E9456
:10DDE00080AAAF964EAD5FADAF970FB6F8945EBF09
:10DDF0000FBE4DBF1ACFF80101900020E9F731970F
:10DE0000CF01801B910B20E05ECF81E0903109F0C3
:10DE100080E08093BB09903141F08985873409F017
:10DE200004CF8A858E3709F400CF8091370C81307A
:10DE300029F08230D9F18111F8CE0AC08091380CD6
:10DE40009091390C01969093390C8093380CEDCE5B
:10DE5000BE016F5F7F4F8DEB99E00E94F2D40115F8
:10DE6000110529F48DEBC82E89E0D82E09C0680170
:10DE7000F60181916F018823A9F30E94A78AF8CF48
:10DE8000F60181916F01882319F00E94A78AF8CFCB
:10DE900080E20E94A78A6D8D7E8D8F8D98A14AE0C9
:10DEA0000E94CA8D8AE00E94A78ABFCEBE016F5F22
:10DEB0007F4F8DEB99E00E94F2D48114910441F0E0
:10DEC0006DEB79E0C4010E94ACF1892B69F414C0B8
:10DED000AD96FFADAD978F2F90E02091440F30911C
:10DEE000450F8217930741F0AD962FADAD972F5F89
:10DEF000AD962FAFAD9799CEE1968EAD9FADE197E0
:10DF00000FB6F8949EBF0FBE8DBFCE58DF4F0FB631
:10DF1000F894DEBF0FBECDBFDF91CF911F910F915F
:10DF2000FF90EF90DF90CF90BF90AF909F908F9039
:10DF30007F906F905F904F903F902F9008950F9338
:10DF40001F93CF93DF93CDB7DEB76F970FB6F894DB
:10DF5000DEBF0FBECDBF8B0122E02093370C909324
:10DF6000450F8093440F89E09AE00E9424A48BE13E
:10DF7000E9E0FAE0DE01159601900D928A95E1F74D
:10DF80008091070A9091080A9C838B8385E692E032
:10DF90009A838983A801BE016F5F7F4F80E090E084
:10DFA00008DECE0101960E9480AA6F960FB6F89403
:10DFB000DEBF0FBECDBFDF91CF911F910F910895AE
:10DFC0002F923F924F925F926F927F928F929F9289
:10DFD000AF92BF92CF92DF92EF92FF920F931F9377
:10DFE000CF93DF93CDB7DEB76F970FB6F894DEBF50
:10DFF0000FBECDBF6C012DB63EB61D8218861C82A9
:10E000001B8285E692E09A838983FB0180819E01D1
:10E010002F5F3F4F39018F3241F085E09AE0F601E2
:10E0200091838083F62E172F64C086EE99E0F60167
:10E03000918380838B010F5F1F4F0115110509F438
:10E0400056C04DB65EB66FE270E0C8010E94CAF1DC
:10E050004C010817190708F048C07C01E01AF10AC2
:10E06000FF24C70101962DB73EB7281B390B0FB609
:10E07000F8943EBF0FBE2DBF8DB79EB701965C01D1
:10E08000A701B8010E94F3F1F501EE0DFF1D10820A
:10E09000F601608171816115710511F06C5F7F4F30
:10E0A00021E0A501CE0105960E9453A8811111C05F
:10E0B000B50186EF99E10E9497B48EE20E94A78A8B
:10E0C0008AE00E94A78A0FB6F8945EBE0FBE4DBECE
:10E0D0000EC0F6017182608284010F5F1F4F0FB680
:10E0E000F8945EBE0FBE4DBEA8CFF02E02C0F12C3C
:10E0F00010E0C3010E9480AA8F2D912F0FB6F894D3
:10E100003EBE0FBE2DBE6F960FB6F894DEBF0FBE9B
:10E11000CDBFDF91CF911F910F91FF90EF90DF90D6
:10E12000CF90BF90AF909F908F907F906F905F90B7
:10E130004F903F902F900895CF93DF938B3D924067
:10E14000B1F0ECE6FAE18491EF012196882321F009
:10E150000E94A78AFE01F7CFE7E8FAE18491EF0178
:10E160002196882331F00E94A78AFE01F7CF80E034
:10E1700001C081E0DF91CF9108952F923F924F929D
:10E180005F926F927F928F929F92AF92BF92CF9247
:10E19000DF92EF92FF920F931F93CF93DF93CDB750
:10E1A000DEB7C757D1090FB6F894DEBF0FBECDBF9B
:10E1B0002DB63EB6A7961FAE1EAEA79784E690E09A
:10E1C000A9969FAF8EAFA99701E09E012B593F4FB3
:10E1D00044E050E0BE01655A7F4FCE0189599F4F00
:10E1E0000E949ED39E012B593F4F42E050E0BE015A
:10E1F00067597F4FCE0189599F4F0E949ED343E0BC
:10E2000050E0BE01655A7F4F8FE093E00E94E5F138
:10E21000892B09F43FC06F968FAD6F97882339F033
:10E220008FE36C968FAF6C976D961FAE6D97E1E89C
:10E23000FAE184917F012FEFE21AF20A811103C003
:10E24000EAE4FBE104C00E94A78AF701F2CF8491BF
:10E250007F013FEFE31AF30A882321F00E94A78A87
:10E26000F701F5CFBE01655A7F4F81E49BE10E9423
:10E2700097B4E3E3FBE184917F019FEFE91AF90A88
:10E28000882321F00E94A78AF701F5CF81E08093CF
:10E29000460F4EC5EDB7FEB7E696FFAFEEAFE69779
:10E2A0006B961CAE1DAE1EAE1FAE6B97A7961FAE33
:10E2B0001EAEA79701E09E012B593F4F41E050E071
:10E2C000BE0160597F4FCE0189599F4F0E949ED356
:10E2D00080E1EBE8F2E0DE01919601900D928A95E3
:10E2E000E1F780E1EBE9F2E0DE01519601900D9259
:10E2F0008A95E1F780E1EBEAF2E0DE011196019008
:10E300000D928A95E1F7E1964FADE19750E04D5FB0
:10E310005F4F440F551F440F551F2DB73EB7241BA9
:10E32000350B0FB6F8943EBF0FBE2DBF8DB79EB70D
:10E3300001967C0100E09E012B593F4FBC01CE01AC
:10E3400089599F4F0E949ED39E012B593F4F44E015
:10E3500050E068E177E0CE0189599F4F0E949ED33B
:10E36000E1968FACE197912C93E0890E911C880C7B
:10E37000991C880C991CEDB7FEB7E819F9090FB67E
:10E38000F894FEBF0FBEEDBF2DB73EB72F5F3F4FD6
:10E3900069018DB79EB7881999090FB6F8949EBF89
:10E3A0000FBE8DBFEDB7FEB731965F019E012B59B1
:10E3B0003F4FA401B601CE0189599F4F0E949ED3C1
:10E3C0009E012B593F4FA401B501CE0189599F4FA2
:10E3D0000E949ED31091470F112309F4A7C000E0BB
:10E3E0009E012B593F4F44E050E060E077E0CE01C2
:10E3F00089599F4F0E949ED39E012B593F4F44E065
:10E4000050E064E077E0CE0189599F4F0E949ED38F
:10E410009E012B593F4F44E050E06CEF76E0CE0177
:10E4200089599F4F0E949ED39E012B593F4F44E034
:10E4300050E060E277E0CE0189599F4F0E949ED361
:10E440009E012B593F4F44E050E06CE177E0CE0154
:10E4500089599F4F0E949ED39E012B593F4F40E107
:10E4600050E068EE76E0CE0189599F4F0E949ED31E
:10E470009E012B593F4F44E050E0BE01695A7F4F47
:10E48000CE0189599F4F0E949ED39E012B593F4F29
:10E490004CE050E06DE475E0CE0189599F4F0E9439
:10E4A0009ED39E012B593F4F44E050E061E278E15A
:10E4B000CE0189599F4F0E949ED39E012B593F4FF9
:10E4C00044E050E0BE01695A7F4FCE0189599F4F09
:10E4D0000E949ED301E09E012B593F4F41E050E046
:10E4E000BE0161597F4FCE0189599F4F0E949ED333
:10E4F0009E012B593F4F41E050E0BE0162597F4FD2
:10E50000CE0189599F4F0E949ED311118AC06B96EC
:10E510008CAD9DADAEADBFAD6B9780935A17909308
:10E520005B17A0935C17B0935D177BC0E1968FAD2E
:10E53000E19790E0029628E037E0E4963FAF2EAFF7
:10E54000E497B501DE011196E1EF8E2EE7E19E2EF4
:10E55000AE014F5E5F4FF2EBAF2EF0E1BF2EE896BB
:10E56000FFAEEEAEE8977E0131E2E30EF11C20E053
:10E5700030E0821793072CF0E896EEADFFADE897F8
:10E5800001C0F7014080518062807380F5014192A3
:10E590005192619271925F018217930714F0F60114
:10E5A00001C0FA014080518062807380F401419281
:10E5B0005192619271924F018217930734F0FB01DF
:10E5C000408051806280738005C04D905D906D9059
:10E5D0007C901397E496EEADFFADE4974192519293
:10E5E00061927192E496FFAFEEAFE4972F5F3F4FD9
:10E5F0006C5F7F4F1496F4E0CF0ED11C4C5F5F4FE1
:10E60000E896EEADFFADE8973496E896FFAFEEAF33
:10E61000E897F4E0EF0EF11C2430310509F0A9CFA2
:10E62000DECEE0968FADE097853099F4AF968FAD52
:10E63000AF97853071F400E09E012B593F4F44E6BF
:10E6400050E06EE577E1CE0189599F4F0E949ED33D
:10E6500024C0111102C00E9401C0E0968FADE09766
:10E66000AF96CFACAF978C9D60011124E12CF12CBB
:10E67000EC14FD0491F000E09E012B593F4F44E063
:10E6800050E0BE01695A7F4FCE0189599F4F0E94C9
:10E690009ED32FEFE21AF20AEBCF00E09E012B5936
:10E6A0003F4F44E050E0BE016D5A7F4FCE01895983
:10E6B0009F4F0E949ED31AE0115079F000E09E0116
:10E6C0002B593F4F44E050E0BE01695A7F4FCE01C5
:10E6D00089599F4F0E949ED3EFCF01E09E012B5995
:10E6E0003F4F41E050E0BE0163597F4FCE01895951
:10E6F0009F4F0E949ED39E012B593F4F41E050E017
:10E70000BE0164597F4FCE0189599F4F0E949ED30D
:10E7100000E09E012B593F4F44E050E0BE01635C96
:10E720007F4FCE0189599F4F0E949ED39E012B5946
:10E730003F4F44E050E0BE016F5C7F4FCE018959EE
:10E740009F4F0E949ED3AE968FADAE97AD96CFAC45
:10E75000AD978C9D60011124E12CF12C00E09E010D
:10E760002B593F4FEC14FD0471F044E050E0BE0122
:10E77000695A7F4FCE0189599F4F0E949ED33FEF28
:10E78000E31AF30AEBCF41E050E0BE016F587F4F30
:10E79000CE0189599F4F0E949ED39E012B593F4F16
:10E7A00041E050E0BE0165597F4FCE0189599F4F2E
:10E7B0000E949ED39E012B593F4F44E050E0BE0182
:10E7C000695A7F4FCE0189599F4F0E949ED39E0167
:10E7D0002B593F4F44E050E0BE01695A7F4FCE01B4
:10E7E00089599F4F0E949ED39E012B593F4F44E071
:10E7F00050E065E278E1CE0189599F4F0E949ED397
:10E800009E012B593F4F44E050E0BE01615B7F4FBA
:10E81000CE0189599F4F0E949ED39E012B593F4F95
:10E8200044E050E0BE01655B7F4FCE0189599F4FA8
:10E830000E949ED39E012B593F4F44E050E0BE0101
:10E84000695B7F4FCE0189599F4F0E949ED310E094
:10E8500000E09E012B593F4F44E050E0BE01695A51
:10E860007F4FCE0189599F4F0E949ED3111110C036
:10E870006B96CCACDDACEEACFFAC6B9720E030E837
:10E880004BE355E4C701B6010E94FDE9811103C0C5
:10E8900054E0F52E33C08091470F811108C0C0921B
:10E8A000740FD092750FE092760FF092770F00E020
:10E8B0009E012B593F4F44E050E060E77FE0CE01DE
:10E8C00089599F4F0E949ED39E012B593F4F44E090
:10E8D00050E068E77FE0CE0189599F4F0E949ED3A8
:10E8E0009E012B593F4F44E050E0BE01695A7F4FD3
:10E8F000CE0189599F4F0E949ED312C0FA94FF20E7
:10E9000079F000E09E012B593F4F44E050E0BE01FA
:10E91000695A7F4FCE0189599F4F0E949ED3EECFF7
:10E920001F5F153009F094CF00E09E012B593F4F37
:10E9300042E050E0BE016D597F4FCE0189599F4F93
:10E940000E949ED39E012B593F4F44E050E0BE01F0
:10E95000695A7F4FCE0189599F4F0E949ED36B9673
:10E96000CCACDDACEEACFFAC6B9720E030E84BE319
:10E9700055E4C701B6010E94FDE9882329F1809181
:10E98000470F811108C0C0926C0FD0926D0FE092BA
:10E990006E0FF0926F0F00E09E012B593F4F44E045
:10E9A00050E068E67FE0CE0189599F4F0E949ED3D8
:10E9B0009E012B593F4F44E050E064E67FE0CE01DA
:10E9C00089599F4F0E949ED300E09E012B593F4FD3
:10E9D00042E050E0BE016F597F4FCE0189599F4FF1
:10E9E0000E949ED39E012B593F4F41E050E0BE0153
:10E9F0006F587F4FCE0189599F4F0E949ED319E0D7
:10EA0000115000E09E012B593F4F112359F044E073
:10EA100050E0BE01695A7F4FCE0189599F4F0E9435
:10EA20009ED3EECF41E050E062EC77E1CE01895910
:10EA30009F4F0E949ED3F12C00E09E012B593F4F27
:10EA400044E050E0BE01695A7F4FCE0189599F4F83
:10EA50000E949ED31091470F111110C0F1100EC0EB
:10EA60006B968CAD9DADAEADBFAD6B978093C71768
:10EA70009093C817A093C917B093CA17F39485E071
:10EA8000F812DACF111102C00E94DFB34CE0F42E6D
:10EA9000FA94F11003C03CE0F32E0FC000E09E0199
:10EAA0002B593F4F42E050E0BE01615A7F4FCE01EB
:10EAB00089599F4F0E949ED3EBCFFA9400E09E01AC
:10EAC0002B593F4FFF2059F044E050E0BE016D5BF1
:10EAD0007F4FCE0189599F4F0E949ED3EECF46E0D3
:10EAE00050E0BE01635C7F4FCE0189599F4F0E9469
:10EAF0009ED39E012B593F4F44E050E068EF76E0F3
:10EB0000CE0189599F4F0E949ED39E012B593F4FA2
:10EB10004CE050E0BE016F5C7F4FCE0189599F4FA2
:10EB20000E949ED32CE1F22EFA94F11003C094E0DF
:10EB3000F92E1DC000E09E012B593F4F44E050E0EC
:10EB4000BE01695A7F4FCE0189599F4F0E949ED3C3
:10EB5000EBCF00E09E012B593F4F44E050E0BE0157
:10EB6000695A7F4FCE0189599F4F0E949ED3FA94D4
:10EB7000F110EFCF8BE0F82EFA94FF2079F000E04F
:10EB80009E012B593F4F44E050E0BE01695A7F4F30
:10EB9000CE0189599F4F0E949ED3EECFA9968EAD8C
:10EBA0009FADA99784569109C7DA8093460F8823B1
:10EBB00009F1E1E8FAE184917F019FEFE91AF90A8E
:10EBC000882321F00E94A78AF701F5CFA9966EADA0
:10EBD0007FADA997645671098BE29BE10E947EB4D8
:10EBE0006BED72E083E29BE10E947EB48AE00E94BA
:10EBF000A78A93C0A7962EAD3FADA797AB968EADD3
:10EC00009FADAB972817390709F445C081E0809381
:10EC1000460FECE6FAE184917F012FEFE21AF20A47
:10EC2000811103C0E3E0FBE104C00E94A78AF70161
:10EC3000F2CF84917F013FEFE31AF30A882321F09A
:10EC40000E94A78AF701F5CFAB968EAD9FADAB972B
:10EC50000E9468DBEEEFFAE184917F019FEFE91AF1
:10EC6000F90A882321F00E94A78AF701F5CFA79619
:10EC70008EAD9FADA7970E9468DBEEEEFAE184911E
:10EC80007F012FEFE21AF20A882309F446C00E949E
:10EC9000A78AF701F4CF111142C0E1E8FAE18491AB
:10ECA0007F013FEFE31AF30A811103C00FE013E085
:10ECB00004C00E94A78AF701F2CFF80181918F0169
:10ECC000882319F00E94A78AF8CFA9966EAD7FAD70
:10ECD000A9976456710981ED9AE10E947EB4A796C6
:10ECE0004EAD5FADA79760E070E084EC9AE10E94C2
:10ECF00044B4E1ECFAE184917F012FEFE21AF20AC9
:10ED0000811107C08091460F811109C00E945FD414
:10ED100006C00E94A78AF701EECF112399F3E69669
:10ED20008EAD9FADE6970FB6F8949EBF0FBE8DBF18
:10ED30008091470F811102C00E9487C79091460FB2
:10ED400081E089270FB6F8943EBE0FBE2DBEC9588C
:10ED5000DF4F0FB6F894DEBF0FBECDBFDF91CF916E
:10ED60001F910F91FF90EF90DF90CF90BF90AF90E9
:10ED70009F908F907F906F905F904F903F902F90DB
:10ED8000089581E08093470FF8D91092470F8111C1
:10ED9000F4C90E941CCC81E008958F929F92AF929B
:10EDA000BF92CF92DF92EF92FF920F931F93CF9378
:10EDB000DF93CDB7DEB7CA5AD1090FB6F894DEBFDC
:10EDC0000FBECDBFE9961CAE1DAE1EAE1FAEE997BD
:10EDD0008091F1039091F203A091F303B091F403B9
:10EDE000ED968CAF9DAFAEAFBFAFED97C556DF4F81
:10EDF00019821882CB59D04084E690E0C356DF4F89
:10EE000099838883CD59D0401092460F9E01255694
:10EE10003F4F44E050E0BE0167587F4FCE0183561C
:10EE20009F4F0E94EBD3C356DF4F88819981CD5904
:10EE3000D0400296C356DF4F99838883CD59D04086
:10EE4000C556DF4F19821882CB59D04081E0CD558D
:10EE5000DF4F8883C35AD0409E0125563F4F41E083
:10EE600050E0BE016D557F4FCE0183569F4F0E94EB
:10EE7000EBD39E0125563F4F40E150E062EB70E13D
:10EE8000CE0183569F4F0E94EBD39E0125563F4FE4
:10EE900044E050E068E177E0CE0183569F4F0E9446
:10EEA000EBD39E0125563F4F40E150E061EF77E103
:10EEB000CE0183569F4F0E94EBD39E0125563F4FB4
:10EEC00040E150E068E077E0CE0183569F4F0E941A
:10EED000EBD39E0125563F4F44E050E060E077E0E1
:10EEE000CE0183569F4F0E94EBD39E0125563F4F84
:10EEF00044E050E064E077E0CE0183569F4F0E94EB
:10EF0000EBD39E0125563F4F44E050E06CEF76E096
:10EF1000CE0183569F4F0E94EBD39E0125563F4F53
:10EF200044E050E060E277E0CE0183569F4F0E94BC
:10EF3000EBD39E0125563F4F44E050E06CE177E073
:10EF4000CE0183569F4F0E94EBD39E0125563F4F23
:10EF500040E150E068EE76E0CE0183569F4F0E947C
:10EF6000EBD38AE097EDA3EABCE3E9968CAF9DAFC3
:10EF7000AEAFBFAFE9979E0125563F4F44E050E04A
:10EF8000BE016B587F4FCE0183569F4F0E94EBD33B
:10EF90009E0125563F4F4CE050E06DE475E0CE01F8
:10EFA00083569F4F0E94EBD38091DC179091DD1721
:10EFB000A091DE17B091DF17C358DF4F8883998384
:10EFC000AA83BB83CD57D0409E0125563F4F44E0D6
:10EFD00050E0BE0163587F4FCE0183569F4F0E9481
:10EFE000EBD385E0CC55DF4F8883C45AD040CB5556
:10EFF000DF4F8883C55AD0409E0125563F4F44E0DD
:10F0000050E06AE577E1CE0183569F4F0E94EBD333
:10F010009E0125563F4F41E050E0BE016C557F4FA9
:10F02000CE0183569F4F0E94EBD39E0125563F4F42
:10F0300041E050E0BE016B557F4FCE0183569F4F9C
:10F040000E94EBD39E0125563F4F44E650E06EE50B
:10F0500077E1CE0183569F4F0E94EBD3CF57DF4F0E
:10F06000188219821A821B82C158D0409E012556EF
:10F070003F4F44E050E0BE016F577F4FCE018356B3
:10F080009F4F0E94EBD3E9961CAE1DAE1EAE1FAE85
:10F09000E9971AE0115071F09E0125563F4F44E068
:10F0A00050E0BE016B587F4FCE0183569F4F0E94A8
:10F0B000EBD3F0CF83E0CA55DF4F8883C65AD040E8
:10F0C000C955DF4F8883C75AD040CB57DF4F1882CE
:10F0D00019821A821B82C558D040C757DF4F188249
:10F0E00019821A821B82C958D040E9961CAE1DAE07
:10F0F0001EAE1FAEE9979E0125563F4F41E050E0FE
:10F10000BE016A557F4FCE0183569F4F0E94EBD3BD
:10F110009E0125563F4F41E050E0BE0169557F4FAB
:10F12000CE0183569F4F0E94EBD39E0125563F4F41
:10F1300044E050E0BE0167577F4FCE0183569F4F9A
:10F140000E94EBD39E0125563F4F44E050E0BE01A4
:10F150006B577F4FCE0183569F4F0E94EBD30AE03F
:10F1600010E00150110971F09E0125563F4F44E017
:10F1700050E0BE016B587F4FCE0183569F4F0E94D7
:10F18000EBD3EFCFC855DF4F1882C85AD0408FEF6E
:10F19000C755DF4F8883C95AD0409E0125563F4F3F
:10F1A00041E050E0BE0168557F4FCE0183569F4F2E
:10F1B0000E94EBD39E0125563F4F41E050E0BE0137
:10F1C00067557F4FCE0183569F4F0E94EBD3E99640
:10F1D0001CAE1DAE1EAE1FAEE9979E0125563F4FD9
:10F1E00044E050E0BE016B587F4FCE0183569F4FE5
:10F1F0000E94EBD39E0125563F4F44E050E0BE01F4
:10F200006B587F4FCE0183569F4F0E94EBD39E01D8
:10F2100025563F4F44E050E065E278E1CE01835649
:10F220009F4F0E94EBD38091BB029091BC02A091B2
:10F23000BD02B091BE02C357DF4F88839983AA8372
:10F24000BB83CD58D0408091BF029091C002A09165
:10F25000C102B091C202CF56DF4F88839983AA833F
:10F26000BB83C159D040CB56DF4F19821882C55994
:10F27000D040C956DF4F19821882C759D0409E012D
:10F2800025563F4F44E050E0BE0163577F4FCE010B
:10F2900083569F4F0E94EBD39E0125563F4F44E07B
:10F2A00050E0BE016F567F4FCE0183569F4F0E94A4
:10F2B000EBD39E0125563F4F44E050E0BE016B5614
:10F2C0007F4FCE0183569F4F0E94EBD310E0C12C9D
:10F2D00080E8D82E8BE3E82E85E4F82E812C912C43
:10F2E00090E8A92E9FE3B92E111138C09E01255632
:10F2F0003F4F44E050E064E77FE0CE0183569F4FEC
:10F300000E94EBD39E0125563F4F44E050E060E75A
:10F310007FE0CE0183569F4F0E94EBD39E0125567E
:10F320003F4F44E050E068E77FE0CE0183569F4FB7
:10F330000E94EBD3E9968CAE9DAEAEAEBFAEE99720
:10F340009E0125563F4F44E050E0BE016B587F4F71
:10F35000CE0183569F4F0E94EBD32AC0E996CCAED4
:10F36000DDAEEEAEFFAEE9979E0125563F4F44E07D
:10F3700050E0BE016B587F4FCE0183569F4F0E94D5
:10F38000EBD3E9961CAE1DAE1EAE1FAEE99704E0AE
:10F39000015071F09E0125563F4F44E050E0BE0100
:10F3A0006B587F4FCE0183569F4F0E94EBD3F0CF17
:10F3B0001F5F153009F098CF84E190E0C156DF4F10
:10F3C00099838883CF59D0409E0125563F4F42E014
:10F3D00050E0BE0161567F4FCE0183569F4F0E9481
:10F3E000EBD39E0125563F4F44E050E06CE67FE0B2
:10F3F000CE0183569F4F0E94EBD39E0125563F4F6F
:10F4000044E050E068E67FE0CE0183569F4F0E94C3
:10F41000EBD39E0125563F4F44E050E064E67FE089
:10F42000CE0183569F4F0E94EBD380E290E0CF55F0
:10F43000DF4F99838883C15AD0409E0125563F4FA4
:10F4400042E050E0BE016F557F4FCE0183569F4F83
:10F450000E94EBD3C655DF4F1882CA5AD04080E2D3
:10F46000E3ECF2E0DE019D9601900D928A95E1F7C2
:10F470009E0125563F4F41E050E0BE0166557F4F4B
:10F48000CE0183569F4F0E94EBD39E0125563F4FDE
:10F4900040E250E0BE01635D7F4FCE0183569F4F37
:10F4A0000E94EBD39E0125563F4F41E050E062ECB5
:10F4B00077E1CE0183569F4F0E94EBD310E01111EC
:10F4C0000EC08091C7179091C817A091C917B0912D
:10F4D000CA17E9968CAF9DAFAEAFBFAFE9979E015B
:10F4E00025563F4F44E050E0BE016B587F4FCE01A0
:10F4F00083569F4F0E94EBD31F5F153001F7BE016B
:10F50000635B7F4F86E1FB0111928A95E9F79E01CB
:10F5100025563F4F46E150E0CE0183569F4F0E9453
:10F52000EBD38CE2E3EEF2E0DE01119601900D9256
:10F530008A95E1F79E0125563F4F4CE250E0BE010F
:10F540006F5F7F4FCE0183569F4F0E94EBD3BE016A
:10F5500061597F4F86E0FB0111928A95E9F79E0180
:10F5600025563F4F46E050E0CE0183569F4F0E9404
:10F57000EBD39E0125563F4F44E050E068EF76E024
:10F58000CE0183569F4F0E94EBD3BE016D597F4F32
:10F590008CE0FB0111928A95E9F79E0125563F4FB9
:10F5A0004CE050E0CE0183569F4F0E94EBD3E9968A
:10F5B0001CAE1DAE1EAE1FAEE9971CE1115071F0DE
:10F5C0009E0125563F4F44E050E0BE016B587F4FEF
:10F5D000CE0183569F4F0E94EBD3F0CFE9961CAE2D
:10F5E0001DAE1EAE1FAEE99714E0115071F09E01E2
:10F5F00025563F4F44E050E0BE016B587F4FCE018F
:10F6000083569F4F0E94EBD3F0CFE9961CAE1DAE00
:10F610001EAE1FAEE9971BE0115071F09E012556FA
:10F620003F4F44E050E0BE016B587F4FCE01835600
:10F630009F4F0E94EBD3F0CF8091460F811167C09E
:10F64000C356DF4FE880F980CD59D040F4E6EF1A79
:10F65000F108C556DF4F88819981CB59D040C756F4
:10F66000DF4F99838883C959D04084E690E0C35620
:10F67000DF4F99838883CD59D0409E0125563F4F57
:10F6800044E050E06FE073E0CE0183569F4F0E944C
:10F69000EBD39E0125563F4F42E050E0BE01675636
:10F6A0007F4FCE0183569F4F0E94EBD3E1E8FAE1F2
:10F6B00084918F010F5F1F4F882321F00E94A78A3A
:10F6C000F801F6CFB7018FEA9AE10E947EB4C756DF
:10F6D000DF4F48815981C959D04060E070E082EA2B
:10F6E0009AE10E9444B4EFE9FAE184918F010F5F3F
:10F6F0001F4F882321F00E94A78AF801F6CFC70187
:10F700000E949C709091460F892B8093460F909198
:10F71000460F81E08927C655DF4F0FB6F894DEBF4C
:10F720000FBECDBFDF91CF911F910F91FF90EF9052
:10F73000DF90CF90BF90AF909F908F900895CF9221
:10F74000DF92EF92FF920F931F93CF93DF936C01A1
:10F750007A018B01C0E0D0E0CE15DF0581F0D80141
:10F760006D918D01D601ED91FC910190F081E02D1C
:10F77000C6011995892B11F02196EECF7E01C701A4
:10F78000DF91CF911F910F91FF90EF90DF90CF907D
:10F790000895FF920F931F93CF93DF938C01EB019A
:10F7A000F42E80E20E94A78A8FEFF81611F084E50C
:10F7B00001C082E40E94A78A8AE30E94A78AF80116
:10F7C000608171818281938142E00E944F8E4881E5
:10F7D00059816A817B818EEF9DE10E9461B462E074
:10F7E00070E080E090E0DF91CF911F910F91FF904A
:10F7F0000C944DC7CF92DF92EF92FF92C0905004CD
:10F80000D0905104E0905204F090530460913E0473
:10F8100070913F0467507109072E000C880B990BFB
:10F820000E9403EA9B01AC01C701B6010E94FDE9F9
:10F8300087FF1FC020E030E040E450E4C701B6017C
:10F840000E947AEE0E94C3EF7093B00F6093AF0FE7
:10F850000E941F59DC01CB01805A9541AF4FBF4F29
:10F860008093AB0F9093AC0FA093AD0FB093AE0FFE
:10F8700008C01092AB0F1092AC0F1092AD0F109207
:10F88000AE0FFF90EF90DF90CF90089590933F04DC
:10F8900080933E0480E0AECF8F929F92AF92BF9252
:10F8A000CF92DF92EF92FF920F931F93CF93DF934C
:10F8B000F0E2FF2EE12CAE2DB0E0BD016F0D711D09
:10F8C000759567956E1511F0F6120BC0E1EEFBE130
:10F8D00065917491072E000C880B990B0E9403EA26
:10F8E00062C09B0121503109220F331F220F331FA9
:10F8F000F901ED59F44E05911491AB01440F551FD8
:10F90000440F551FFA01ED59F44EC591D49180175B
:10F91000910714F4F62ED1CFC817D90714F4E62EA8
:10F92000CACFF901EB59F44EE590F490FA01EB5986
:10F93000F44EC590D490BC01601B710B072E000CD7
:10F94000880B990B0E9403EA4B015C01B6016E190A
:10F950007F09072E000C880B990B0E9403EA9B017C
:10F96000AC01C501B4010E9462EA4B015C01C01BFD
:10F97000D10BBE01DD0F880B990B0E9403EA9B019E
:10F98000AC01C501B4010E9456EF4B015C01B70107
:10F99000FF0C880B990B0E9403EA9B01AC01C50187
:10F9A000B4010E947AEEDF91CF911F910F91FF90E9
:10F9B000EF90DF90CF90BF90AF909F908F90089581
:10F9C0000F931F93CF93DF93CDB7DEB728970FB672
:10F9D000F894DEBF0FBECDBF60913E0470913F042E
:10F9E000072E000C880B990B0E9403EA6D837E831F
:10F9F0008F8398878091500490915104A091520474
:10FA0000B091530489839A83AB83BC834DEFBE01CD
:10FA10006B5F7F4FCE010196BCDE60913804709120
:10FA20003904072E000C880B990B0E9403EA6D83A2
:10FA30007E838F83988780913A0490913B04A091B4
:10FA40003C04B0913D0489839A83AB83BC834FEF20
:10FA5000BE016B5F7F4FCE0101969BDEE6E0FEE1CB
:10FA600084918F010F5F1F4F882321F00E94A78A86
:10FA7000F801F6CFE091860FF0E0EC57F04F60818F
:10FA800070E080E090E00E94358EE1E0FEE184913C
:10FA90008F010F5F1F4F882321F00E94A78AF80172
:10FAA000F6CF6091850F70E080E090E00E94358E87
:10FAB00028960FB6F894DEBF0FBECDBFDF91CF9171
:10FAC0001F910F9108950F930FB70F9300916E0040
:10FAD0000B7F00936E0078940F930BB70F930CB7C6
:10FAE0000F921F922F933F934F935F936F937F9348
:10FAF0008F939F93AF93BF93EF93FF93112494D170
:10FB0000FF91EF91BF91AF919F918F917F916F91F5
:10FB10005F914F913F912F911F900F900CBF0F91CC
:10FB20000BBF0F910460F89400936E000F910FBF0C
:10FB30000F911895CF92DF92EF92FF92C0903A0406
:10FB4000D0903B04E0903C04F0903D046091380478
:10FB50007091390466507109072E000C880B990BBF
:10FB60000E9403EA9B01AC01C701B6010E94FDE9B6
:10FB700087FF1FC020E030E040E050E4C701B6013D
:10FB80000E947AEE0E94C3EF7093B60F6093B50F98
:10FB90000E941F59DC01CB01805A9541AF4FBF4FE6
:10FBA0008093B10F9093B20FA093B30FB093B40FA3
:10FBB00008C01092B10F1092B20F1092B30F1092B2
:10FBC000B40FFF90EF90DF90CF9008951092800FC8
:10FBD00080E090E05BDE1092390410923804AADFD6
:10FBE0000E94F9B480E090E051DE1092840F2C98CE
:10FBF00010923904109238041092850F80910201FE
:10FC000080728093000108958F929F92AF92BF926D
:10FC1000CF92DF92EF92FF920F931F93CF93DF93D8
:10FC2000F0E4FF2EE12CAE2DB0E0BD016F0D711D93
:10FC3000759567956E1511F0F6120BC0E3E5FDE1C1
:10FC400065917491072E000C880B990B0E9403EAB2
:10FC500062C09B0121503109220F331F220F331F35
:10FC6000F901EB5AF34E05911491AB01440F551F66
:10FC7000440F551FFA01EB5AF34EC591D4918017EA
:10FC8000910714F4F62ED1CFC817D90714F4E62E35
:10FC9000CACFF901E95AF34EE590F490FA01E95A16
:10FCA000F34EC590D490BC01601B710B072E000C65
:10FCB000880B990B0E9403EA4B015C01B6016E1997
:10FCC0007F09072E000C880B990B0E9403EA9B0109
:10FCD000AC01C501B4010E9462EA4B015C01C01B8A
:10FCE000D10BBE01DD0F880B990B0E9403EA9B012B
:10FCF000AC01C501B4010E9456EF4B015C01B70194
:10FD0000FF0C880B990B0E9403EA9B01AC01C50113
:10FD1000B4010E947AEEDF91CF911F910F91FF9075
:10FD2000EF90DF90CF90BF90AF909F908F9008950D
:10FD300060E08091C10F9091C20FAEDD60935004DE
:10FD40007093510480935204909353048091BF0F99
:10FD50009091C00F59DF60933A0470933B048093F5
:10FD60003C0490933D04A8951092810F0895DF9272
:10FD7000EF92FF920F931F93CF93DF93F82ED62E1F
:10FD8000E72E8A0180912702882309F439C0ECE626
:10FD9000FAE18491EF012196882321F00E94A78A3D
:10FDA000FE01F7CFED2DFE2D8491EF0121968823E2
:10FDB00021F00E94A78AFE01F7CFE4EFFBE18491D6
:10FDC000EF012196882321F00E94A78AFE01F7CF38
:10FDD000F7FC0BC06F2DFF0C770B880B990B0E9463
:10FDE000358E8AE00E94A78A0BC0EFEEFBE184917A
:10FDF000EF012196882321F00E94A78AFE01F7CF08
:10FE00008091870F811108C01092270281E08093B2
:10FE1000870FC8010E94A3AADF91CF911F910F9174
:10FE2000FF90EF90DF90D2CE0F931F93CF93DF938D
:10FE300080912A028F37A0F08F579091840F909372
:10FE4000D20F992311F02C9A01C02C982091850F84
:10FE50002093D10F90910201222369F090950BC05D
:10FE60009091D20F891708F02C989091D10F891793
:10FE700028F0909102019072909300018F5F80931F
:10FE80002A029091D00F81E089278093D00F809132
:10FE9000290285301CF4C1E0C80F01C0C0E08230E7
:10FEA00009F4B8C054F4882301F1813009F0E7C0A7
:10FEB00088E080937B0085E4C4C0843009F4C9C025
:10FEC0000CF4BBC0853009F0DAC09091CF0F9111CE
:10FED00002C08093CF0F8091CF0F81508093CF0FBE
:10FEE000882309F4CCC0C5E0CAC0809128028F5F86
:10FEF00080311CF480932802C2C0109228028091A5
:10FF0000810F811113C08091C50F9091C60F9093FE
:10FF1000C20F8093C10F8091C30F9091C40F909333
:10FF2000C00F8093BF0F81E08093810F8AE0E5ECE2
:10FF3000FFE0DF011D928A95E9F71092C40F10923D
:10FF4000C30F0091C10F1091C20F119501951109B6
:10FF500080913E0490913F04D1E0181619062CF0D0
:10FF60008091840F811101C0D0E08091360590917D
:10FF700037059195819591098017910734F44CE8E4
:10FF80005DE16DEA7DE180E0F2DE80911C029091FE
:10FF90001D029195819591090817190744F4DD23F5
:10FFA00031F04FEB5DE160EE7DE180E0E0DE8091DD
:10FFB00038049091390411E0181619062CF080913C
:10FFC000850F811101C010E02091BF0F3091C00F4B
:10FFD00080913405909135058217930734F04CE9F0
:10FFE0005DE16DEA7DE18FEFC2DE20911A02309172
:10FFF0001B028091BF0F9091C00F821793070CF4E2
:020000021000EC
:100000003EC01123E1F14FEC5DE160EE7DE18FEF49
:10001000AEDE35C080917A0086FD2EC080917800DA
:10002000909179002091C50F3091C60F820F931FD8
:100030009093C60F8093C50F22C088E080937B0009
:1000400086E480937C0080917A00806480937A00BB
:1000500016C080917A0086FD11C080917800909141
:1000600079002091C30F3091C40F820F931F90939A
:10007000C40F8093C30F03C0C2E001C0C4E0C093AB
:1000800029020E9411C08091820F9091830F0097E6
:1000900099F001979093830F8093820F892B61F4DD
:1000A00082EF9DE190932C0780932B07DF91CF91F6
:1000B0001F910F910C94D38ADF91CF911F910F91D3
:1000C00008952F923F924F925F926F927F928F92FC
:1000D0009F92AF92BF92CF92DF92EF92FF920F93D7
:1000E0001F93CF93DF9300D01F92CDB7DEB75C0193
:1000F0007A8369834A01170107FD07C0802F002E0C
:10010000000C990B9C838B8304C0E1E0F0E0FC833E
:10011000EB83F90140805180628073808B819C81E8
:10012000880F991F880F991F9C838B838954904F48
:100130007C01A3019201FC01608171818281938124
:100140000E94FDE9882391F0F7014082518262828A
:10015000738211E020E030E0A901C301B2010E94E6
:10016000A0F018160CF010E0F5011083F501808165
:100170008230D1F0833009F45EC0813009F07CC058
:10018000EB81FC81E954F04F208131814281538120
:10019000F40160817181828193810E94FDE987FD74
:1001A0006BC082E0F50180838B819C818954904FE4
:1001B0009C838B83B60180E090E00E9401EA9B0162
:1001C000AC01EB81FC8160817181828193810E940D
:1001D00079EE9B01AC01F401608171818281938190
:1001E0000E94A0F087FD14C00E941F596B017C0182
:1001F0009101A8EEB3E00E946AEEC60ED71EE81E7B
:10020000F91EE981FA81C082D182E282F38234C090
:100210000E941F59E981FA81C080D180E280F38079
:10022000DC01CB018C199D09AE09BF09B7FD24C0C3
:1002300083E0F50180830F3F19F045E55DE102C0E1
:1002400048E65DE16CE77DE1802F0F900F900F9005
:100250000F90DF91CF911F910F91FF90EF90DF9062
:10026000CF90BF90AF909F908F907F906F905F9056
:100270004F903F902F907BCD0F900F900F900F904D
:10028000DF91CF911F910F91FF90EF90DF90CF9072
:10029000BF90AF909F908F907F906F905F904F90A6
:1002A0003F902F9008957F928F929F92AF92BF922E
:1002B000CF92DF92EF92FF920F931F93CF93DF9332
:1002C00020E030E048E452E4609150047091510421
:1002D00080915204909153040E94A0F018164CF49F
:1002E000E9EEFBE1E491C1E001C0CC0FEA95EAF749
:1002F00001C0C0E083EEE82E8BE1F82E09EE1BE191
:1003000096E0A92E912CD0E0CC24C394D12CF701F7
:100310007490F801849077FC23C0892D90E0082C1C
:1003200002C0959587950A94E2F780FD19C0BE0139
:10033000082C02C0759567950A94E2F76170B62E95
:10034000B1946B2D872D0E941CC66B2D70E0872DFC
:100350000E9486C6C60101C0880F8A94EAF7982ACF
:10036000AA94FFEFEF1AFF0A0F5F1F4FA110CFCF24
:10037000DF91CF911F910F91FF90EF90DF90CF9081
:10038000BF90AF909F908F907F9008954F925F9213
:100390006F927F928F929F92AF92BF92CF92DF9295
:1003A000EF92FF920F931F93CF93DF93CDB7DEB7FA
:1003B00060970FB6F894DEBF0FBECDBF8091810F5E
:1003C000811117C060960FB6F894DEBF0FBECDBF87
:1003D000DF91CF911F910F91FF90EF90DF90CF9021
:1003E000BF90AF909F908F907F906F905F904F9055
:1003F00008959EDC0E941F594B015C0160913E04F0
:1004000070913F04072E000C880B990B0E9403EAA1
:1004100069837A838B839C8344E1C42ED12C5CE373
:10042000E52EF12C00E09E012F5F3F4F40E554E0A8
:1004300067EA7FE086EA9FE044DEC0905004D090F7
:100440005104E0905204F09053046091380570918B
:100450003905072E000C880B990B0E9403EA9B01BB
:10046000AC01C701B6010E94A0F018160CF009C13A
:1004700060911E0270911F02072E000C880B990BD1
:100480000E9403EA9B01AC01C701B6010E94FDE98D
:1004900087FFF7C000913E0410913F04B801012E80
:1004A000000C880B990B0E9403EAA70196010E9499
:1004B00079EE2B013C0120ED3CEC4CE45DE36091D6
:1004C000780F7091790F80917A0F90917B0F0E9435
:1004D00062EA6D837E838F83988720919D0F309190
:1004E0009E0F40919F0F5091A00FC701B6010E942F
:1004F00079EE9B01AC016D817E818F8198850E9490
:1005000062EA6D837E838F83988723E333E343E737
:100510005FE36091990F70919A0F80919B0F90917A
:100520009C0F0E9462EA9B01AC016D817E818F81EC
:1005300098850E947AEE6D837E838F83988760937F
:10054000990F70939A0F80939B0F90939C0FC0927A
:100550009D0FD0929E0FE0929F0FF092A00F20E08F
:1005600030E040E251E4C301B2010E94A0F018164D
:100570000CF430C220E030E040E251ECC301B201A3
:100580000E94FDE987FD2FC2012B09F42CC2809146
:10059000980F81112CC22091940F3091950F4091AA
:1005A000960F5091970F29873A874B875C87209148
:1005B000740F3091750F4091760F5091770FC301F2
:1005C000B2010E9462EA6B017C01A301920169857C
:1005D0007A858B859C850E947AEE69877A878B87DE
:1005E0009C876093940F7093950F8093960F9093D0
:1005F000970F2091700F3091710F4091720F5091B1
:10060000730F0E9462EAA70196010E947AEE2D8183
:100610003E814F8158850E9479EE6B017C0120E07C
:1006200030E04FE753E40E94A0F020E030E0A90161
:1006300018160CF4E3C1C701B6010E94FDE987FD5D
:1006400007C0C701B6010E94BEEF759567951AC035
:1006500020E030E0A901C301B2010E94FDE987FF5B
:1006600010C0A301920169857A858B859C850E94C3
:1006700079EE6093940F7093950F8093960F9093FB
:10068000970F60E06093840F8091AB0F9091AC0F57
:10069000A091AD0FB091AE0F0097A105B10521F16A
:1006A000A5019401281B390B4A0B5B0B57FD1CC09D
:1006B0006091AF0F7091B00F80E090E00E9401EA6E
:1006C0009B01AC01609150047091510480915204DF
:1006D000909153040E94FDE987FF81C144E35CE1EE
:1006E00066E47CE180E043DB80917C0F90917D0F9C
:1006F000A0917E0FB0917F0FA5019401281B390BAB
:100700004A0B5B0B57FD0FC0CEDDD501C4018C53E6
:10071000964FAF4FBF4F80937C0F90937D0FA09368
:100720007E0FB0937F0F8091B10F9091B20FA09187
:10073000B30FB091B40F0097A105B10511F1881A5C
:10074000990AAA0ABB0AB7FC1CC06091B50F709148
:10075000B60F80E090E00E9401EA9B01AC0160913D
:100760003A0470913B0480913C0490913D040E94B6
:10077000FDE987FF20C142E15CE165E27CE18FEFAA
:10078000F6DA6091380470913904072E000C880B5A
:10079000990B0E9403EA69837A838B839C8395E09B
:1007A000C92ED12C24E1E22EF12C0FEF9E012F5FF8
:1007B0003F4F4AE354E061EA7FE085EA9FE081DC55
:1007C000C0903A04D0903B04E0903C04F0903D048B
:1007D00020E030E040EA50E4C701B6010E94A0F0FA
:1007E00087FDE5C020E030E040EF52E4C701B601EC
:1007F0000E94FDE918160CF4DAC06091380470917B
:100800003904072E000C880B990B0E9403EAA701FC
:1008100096010E9479EE4B015C0120916C0F3091A2
:100820006D0F40916E0F50916F0F0E9462EA6987C1
:100830007A878B879C872091900F3091910F409100
:10084000920F5091930FC501B4010E947AEE6D830F
:100850007E838F8398876093900F7093910F80931E
:10086000920F9093930F2091680F3091690F4091F0
:100870006A0F50916B0F0E9462EA6D877E878F87A7
:10088000988B20ED3CEC4CE45DE36091640F70913B
:10089000650F8091660F9091670F0E9462EA2B01AD
:1008A0003C0120918C0F30918D0F40918E0F509113
:1008B0008F0FC701B6010E9479EE9B01AC01C30105
:1008C000B2010E9462EA2B013C0123E333E343E7D8
:1008D0005FE36091880F7091890F80918A0F9091EA
:1008E0008B0F0E9462EA9B01AC01C301B2010E941E
:1008F0007AEE2B013C016093880F7093890F8093EF
:100900008A0F90938B0FC0928C0FD0928D0FE09234
:100910008E0FF0928F0F2D853E854F855889698502
:100920007A858B859C850E947AEEA30192010E94B4
:1009300079EE6B017C0120E030E04FE753E40E9448
:10094000A0F020E030E0A9011816BCF5C501B40103
:100950000E94A0F0181684F4A50194016D817E8197
:100960008F8198850E9479EE6093900F7093910F1C
:100970008093920F9093930F6FE71AC020E030E0BE
:10098000A901C501B4010E94FDE987FF10C0A501BE
:1009900094016D817E818F8198850E9479EE6093AC
:1009A000900F7093910F8093920F9093930F60E04C
:1009B0006093850F07CDBED8E4CEC701B6010E9473
:1009C000FDE987FDDBCFC701B6010E94BEEF75953B
:1009D0006795EECF81E08093980F6FE753CE80E06C
:1009E0000E94FA7B81CE81E08093980F4ACE1092CC
:1009F000980F19861A861B861C86D9CDC301B201B1
:100A00000E94A0F018164CF7A301920169857A851F
:100A10008B859C850E9479EE6093940F7093950F5F
:100A20008093960F9093970F6FE72CCE0F931F93A1
:100A30008091630F813019F40E941F5908C06091A2
:100A40005F0F7091600F8091610F9091620F009124
:100A50005B0F10915C0F20915D0F30915E0F601B5A
:100A6000710B820B930B28EE33E040E050E00E94C4
:100A70001CEE8091570F9091580FA091590FB09193
:100A80005A0FBC01CD01620F731F841F951F1F9168
:100A90000F9108951092630F10925B0F10925C0FEC
:100AA00010925D0F10925E0F10925F0F1092600F08
:100AB0001092610F1092620F1092570F1092580F00
:100AC0001092590F10925A0F089590916F00292F8C
:100AD000227091FF05C090916F009D7F90936F00F1
:100AE00034E0839FC0011124FC01EF51F84E408196
:100AF000518162817381FC01E55BF04F408351833A
:100B00006283738381E080934A0F222329F08091CE
:100B10006F00826080936F000895BC012091480FA0
:100B20003091490F4091480F5091490F24173507D4
:100B300011F09A01F7CF81E02617370709F080E01E
:100B4000089590911E18E92FF0E0E75AFA4F80833C
:100B50009F5F943018F490931E1802C010921E18D4
:100B600080911F188F5F80931F180895CF93FC0109
:100B700020812B33A1F020911F18243080F4C62F40
:100B8000BC0180911E18F0E68F9FC0011124825A8B
:100B90009A4F0E94DEF18C2FD4DF81E001C080E00B
:100BA000CF9108952F923F924F925F926F927F92D2
:100BB0008F929F92AF92BF92CF92DF92EF92FF926D
:100BC0000F931F93CF93DF9300D000D0CDB7DEB744
:100BD0009A8389830E941F59E981FA81C680D78050
:100BE000E084F184C114D104E104F10409F0ACC241
:100BF0002485222309F469C332852150248721E00A
:100C0000230F22874585241301C01286E981FA81CA
:100C100024E0329FE00DF11D1124C684D784E088C2
:100C2000F188E981FA81C282D382E482F582DC0113
:100C3000CB018C0D9D1DA11DB11D86839783A087BF
:100C4000B18784819581892B09F43FC3FFB7FD8368
:100C5000F894E981FA81228033802101612C712C82
:100C600004811581809119028F3121F08F3F09F0A5
:100C700068C205C0E7E6F8E124912E83DAC08FE16F
:100C800080931902E7E6F8E184918E838F3F09F49F
:100C900058C2823009F469C030F5882309F44CC089
:100CA000813009F0C6C010928000109281008091BE
:100CB00081008860809381008091810081608093B1
:100CC0008100EAE3F8E2E491F0E0EE0FFF1FE95162
:100CD000F84D85919491E0E8F8E2E491E093D60F25
:100CE000E1E0EE8330C19E81943009F482C008F4C3
:100CF00060C0953009F09DC0109220011092210132
:100D0000809121018860809321018091210181607F
:100D100080932101EAE3F8E2E491F0E0EE0FFF1F97
:100D2000E951F84D85919491E0E8F8E2E491E0937F
:100D3000D30F95E09E8307C114BC15BC84B58260B7
:100D400084BD85B5816085BDEAE3F8E2E491F0E019
:100D5000EE0FFF1FE951F84D85919491E0E8F8E21C
:100D6000E491E093D70F1E82ABC21092B0001092B4
:100D7000B1008091B00082608093B0008091B1009A
:100D800081608093B100EAE3F8E2E491F0E0EE0FD5
:100D9000FF1FE951F84D8591949190932D05809313
:100DA0002C05E0E8F8E2E491E0932E05F2E0FE8302
:100DB00087C21092900010929100809191008860FB
:100DC0008093910080919100816080939100EAE38B
:100DD000F8E2E491F0E0EE0FFF1FE951F84D859144
:100DE0009491E0E8F8E2E491E093D50F23E02E83BC
:100DF000AAC01092A0001092A1008091A10088606A
:100E00008093A1008091A10081608093A100EAE31A
:100E1000F8E2E491F0E0EE0FFF1FE951F84D859103
:100E20009491E0E8F8E2E491E093D40F84E08E83BB
:100E30008AC0EE81E7FD85C161E08FE10E944AC66C
:100E40008E818D7F09F083C04801A12CB12C60E018
:100E500072E18AE790E0A50194010E943EEE2983A9
:100E60003A834B835C8369017A01F1E0CF1AD108A0
:100E7000E108F1082FEFC216D104E104F10409F0F2
:100E800008F44EC060E472E48FE090E0A5019401A4
:100E90000E943EEE69017A0181E0C81AD108E1089A
:100EA000F1089E81923009F5EFEFCE16D104E104EE
:100EB000F10409F008F4CBC160E970ED83E090E043
:100EC000A50194010E943EEE69017A01F1E0CF1A7A
:100ED000D108E108F1082FEFC216D104E104F104B2
:100EE00011F008F041C183E027C08FEFC816D1048C
:100EF000E104F104B9F0B0F068E478EE81E090E04C
:100F0000A50194010E943EEE69017A0191E0C91A9F
:100F1000D108E108F108EE81EE2309F49AC163C11A
:100F200081E001C082E09E81911106C095B5987F55
:100F3000892B85BD7AC085E09091B100987F892B7F
:100F40008093B10072C061E08FE10E944AC64801FF
:100F5000A12CB12C60E072E18AE790E0A501940138
:100F60000E943EEE69017A01E1E0CE1AD108E10863
:100F7000F108C114D104F1E0EF06F10488F068E44F
:100F800078EE81E090E0A50194010E943EEE6901B7
:100F90007A0181E0C81AD108E108F10883E001C0B4
:100FA00081E09E81913071F490918100987F892B2E
:100FB00080938100452846284728D9F52FEF3FEF39
:100FC000A90168C0EE81E33071F490919100987F9F
:100FD000892B8093910045284628472851F52FEF0B
:100FE0003FEFA90179C0FE81F43071F49091A10026
:100FF000987F892B8093A100452846284728C9F46B
:101000002FEF3FEFA9017AC02E81253071F4909126
:101010002101987F892B8093210145284628472864
:1010200041F42FEF3FEFA9017BC045284628472810
:1010300069F0D801AA0FBB1F91010E946AEE28EE49
:1010400033E040E050E00E941CEE03C02FEF3FEF82
:10105000A9018E81823081F12CF4882361F08130E6
:10106000C9F06FC09E81943009F448C0ACF195304E
:1010700009F456C066C0C7BC2093E80F3093E90F4F
:101080004093EA0F5093EB0F80916E008260809343
:101090006E0057C0D0928900C09288002093E40F60
:1010A0003093E50F4093E60F5093E70F80916F0068
:1010B000826080936F0045C0C092B30020932F05DB
:1010C0003093300540933105509332058091700084
:1010D00082608093700035C0D0929900C0929800D1
:1010E0002093E00F3093E10F4093E20F5093E30F12
:1010F0008091710082608093710023C0D092A9001A
:10110000C092A8002093DC0F3093DD0F4093DE0FD8
:101110005093DF0F8091720082608093720011C043
:10112000D0922901C09228012093D80F3093D90F73
:101130004093DA0F5093DB0F8091730082608093AD
:101140007300ED81EFBFC1C0DC01CB018C199D099B
:10115000AE09BF09B7FDB9C04698E981FA81168288
:10116000178210861186B1C068E478EE81E090E0C5
:10117000A50194010E943EEE69017A01F1E0CF1AC7
:10118000D108E108F1082FEFC216D104E104F104FF
:1011900041F138F164E274EF80E090E0A501940140
:1011A0000E943EEE69017A01F1E0CF1AD108E10810
:1011B000F1082FEFC216D104E104F10409F008F49C
:1011C000BACE62E17AE780E090E0A50194010E9446
:1011D0003EEE69017A0181E0C81AD108E108F10800
:1011E00019C084E0A9CE2FEFC216D104E104F104A6
:1011F00009F008F463C062E17AE780E090E0A501BD
:1012000094010E943EEE69017A01F1E0CF1AD10803
:10121000E108F1082FEFC216D104E104F104A9F0AE
:10122000A0F089819A81AB81BC812AE0B595A79510
:10123000979587952A95D1F76C017D01F1E0CF1A3A
:10124000D108E108F10887E077CE86E075CE82E02C
:1012500073CEEFEFCE16D104E104F10469F160F131
:1012600062E17AE780E090E0A50194010E943EEE01
:1012700069017A0181E0C81AD108E108F1089FEFFD
:10128000C916D104E104F104A9F0A0F089819A8182
:10129000AB81BC813AE0B595A795979587953A952E
:1012A000D1F76C017D01E1E0CE1AD108E108F10827
:1012B00085E03CCE84E03ACE83E038CE84E033CE85
:1012C00061E08FE10E944AC6BFCD26960FB6F89422
:1012D000DEBF0FBECDBFDF91CF911F910F91FF9069
:1012E000EF90DF90CF90BF90AF909F908F907F90C6
:1012F0006F905F904F903F902F9008950F931F93A2
:10130000CF93DF93CDB7DEB72C970FB6F894DEBF3F
:101310000FBECDBFE0E4F4E080859185A285B38562
:1013200044815581668177810081118122813381D9
:1013300009831A832B833C834D835E836F83788775
:1013400089879A87AB87BC87AE01475F5F4FBE0135
:101350006B5F7F4FCE0101960E9414BF2CE434E0F6
:10136000AE01475F5F4FBE016B5F7F4FCE010196BD
:101370000E9412B82C960FB6F894DEBF0FBECDBFF8
:10138000DF91CF911F910F9108952F923F924F922D
:101390005F926F927F928F929F92AF92BF92CF9205
:1013A000DF92EF92FF920F931F93CF93DF93EB01A6
:1013B000FC0180809180A280B380C501B40120E847
:1013C00031E541E050E00E941CEEC9016DE671E09C
:1013D0000E944FF16B017C01C501B40120E13EE0A8
:1013E00040E050E00E941CEECA01B90128E130E063
:1013F00040E050E00E941CEE362E272E062F172FBD
:101400008CE3482E512C612C712CC501B401A30131
:1014100092010E941CEEB62EA72ECA01B901A301AB
:1014200092010E941CEECB01C114D104D9F0AF92FD
:10143000BF927F936F932F923F92FF92EF92DF9232
:10144000CF9282E39EE19F938F93DF93CF930E948D
:10145000CFE98DB79EB70E960FB6F8949EBF0FBE1C
:101460008DBF5CC0E114F104C9F0AF92BF927F93CD
:101470006F932F923F92FF92EF9282E29EE19F93B1
:101480008F93DF93CF930E94CFE9EDB7FEB73C96E1
:101490000FB6F894FEBF0FBEEDBF40C0012BB9F0F0
:1014A000AF92BF927F936F932F923F9286E19EE11E
:1014B0009F938F93DF93CF930E94CFE98DB79EB711
:1014C0000A960FB6F8949EBF0FBE8DBF27C0892B1A
:1014D000A9F0AF92BF927F936F938EE09EE19F93AE
:1014E0008F93DF93CF930E94CFE9EDB7FEB7389685
:1014F0000FB6F894FEBF0FBEEDBF10C0AF92BF9203
:101500008AE09EE19F938F93DF93CF930E94CFE970
:101510000F900F900F900F900F900F90DF91CF9141
:101520001F910F91FF90EF90DF90CF90BF90AF9001
:101530009F908F907F906F905F904F903F902F90F3
:101540000895FC01238121110C94C7A20895909164
:10155000C00095FFFCCF8093C6000895EF92FF92E4
:101560001F93CF93DF937C0160E000DB182F88236B
:1015700099F0E1E8FAE18491EF012196882319F0CE
:10158000E6DFFE01F8CFB70186E49EE10E9497B442
:1015900082E2DDDF8AE0DBDF812FDF91CF911F91D7
:1015A000FF90EF900895DF92EF92FF920F931F93B9
:1015B000CF93DF93CDB7DEB76E970FB6F894DEBF4B
:1015C0000FBECDBF60912B0770912C07611571057F
:1015D00041F14DE150E0CE0101967C010E94A6E967
:1015E0001E8EF7018F010E191F09D190DD2019F011
:1015F0009AE0D912F7CFF701E00FF11F1082C7016F
:10160000ADDF882371F0DD20A9F00F5F1F4F8091BF
:101610002B0790912C07080F191F10932C0700938C
:101620002B0781E020912B0730912C07232B29F4E5
:1016300080E003C000E010E0F0CF6E960FB6F894A3
:10164000DEBF0FBECDBFDF91CF911F910F91FF90F5
:10165000EF90DF9008953F924F925F926F927F924A
:101660008F929F92AF92BF92CF92DF92EF92FF92B2
:101670000F931F93CF93DF931F92CDB7DEB793DF06
:10168000811175C280911F18843008F048C00E94F3
:10169000F34BAC0197FF7BC142C08E3409F0D8C137
:1016A0000115110509F4D4C169E77FE1C8010E9461
:1016B000B5E97C01892B09F48DC16EE470E0C801A5
:1016C00004960E94CAF1009709F484C14AE050E0F0
:1016D00060E070E001960E9451E76093EC0F709318
:1016E000ED0F8093EE0F9093EF0F8090F418909091
:1016F000F518A090F618B090F7182FEF821A920AFA
:10170000A20AB20A681579058A059B0509F464C125
:10171000EF2809F061C186E49FE10E94D2DA80914E
:10172000B909882309F423C280911F18811102C0CE
:1017300010925210EE24E3944091330C5091340CEB
:101740006091350C7091360C80912F0C9091300C7B
:10175000A091310CB091320C481759076A077B07EA
:1017600008F4E12C00E010E09924939480E6882EA0
:101770009EE7A92E9FE1B92E2DE8322E80911F18E9
:10178000843008F0F4C1E110F2C18091521081114F
:10179000EEC180918A0B90918B0BA0918C0BB09134
:1017A0008D0B8093330C9093340CA093350CB09335
:1017B000360C41E050E0BE016F5F7F4F82E89BE056
:1017C0000E9447A5019719F4898190E002C08FEF2C
:1017D0009FEFF82E4090330C5090340C6090350CF5
:1017E0007090360C40912F0C5091300C6091310C60
:1017F0007091320CEE24E394441655066606770683
:1018000008F4E12C4416550666067706B0F40196F6
:1018100009F469C08AE0F81609F488C09DE0F91659
:1018200009F484C023E2F21619F08AE3F81295C095
:1018300080915110811191C06EC00E94386A82E877
:101840009BE00E94C7A280919D0B882359F1815093
:1018500080939D0B389EC001112441E061E08E55BC
:10186000944F0E9432D9E0919D0B94E0E99FF001E2
:101870001124E256F44F408151816281738140937B
:10188000330C5093340C6093350C7093360C82E813
:101890009BE00E94DDA18091BA098823A1F090927B
:1018A000B90911C01092B9090E94F8B90E94F9B49F
:1018B000BDD86D3371058105910528F0B0922C07D4
:1018C000A0922B0770DE8091B909811128C0E1E94F
:1018D000FFE184916F012FEFC21AD20A8823D9F059
:1018E00036DEF601F6CFECE6FAE184916F019FEF68
:1018F000C91AD90A882319F02ADEF601F6CFE2E8E0
:10190000FFE184916F012FEFC21AD20A882319F0E8
:101910001EDEF601F6CF83E2F81208C005C023E20E
:10192000F21222C100E010E0909252101092511079
:101930000115110519F40E94C6810CC080911E1872
:10194000889E000D111D1124F801E25AFA4F1082F1
:1019500080E0F7D800E010E011CF0F35110508F056
:101960000DCF9BE3F91202C090925110809151105B
:10197000811104CF80911E18F801889EE00DF11DA1
:101980001124E25AFA4FF0820F5F1F4FF7CE982FC3
:101990002091F2183091F3188A3019F09D3009F037
:1019A000B1C0109250102115310519F40E94C68162
:1019B00069CEF901E051F04F10821092F3181092A5
:1019C000F21800EF1FE0F8018191803209F065CE36
:1019D0008F01F9CFC8017ACE6AE270E0C8010E9497
:1019E00002F29C01009701F1982F901BF12C992392
:1019F00039F09150F801E90FF11D8081F826F7CFF9
:101A00004AE050E060E070E0C90101960E9451E7B1
:101A1000CF2CD12CE12CF12C6C157D058E059F056A
:101A200031F087E29FE179CE8DEF9EE176CE809115
:101A3000EC0F9091ED0FA091EE0FB091EF0F80930E
:101A4000F4189093F518A093F618B093F7180EC0F9
:101A50008091B709882351F065EF73E0C8010E94B7
:101A6000D5F1892B19F083ED9EE157CE80912702A5
:101A7000811126C067E470E0C8010E94CAF1009796
:101A8000F9F04AE050E060E070E001960E9451E712
:101A900097FD16C064307105810591052CF0653005
:101AA00071058105910561F4ECE5FEE184917F010A
:101AB0009FEFE91AF90A882319F049DDF701F6CFFB
:101AC00069EF73E0C8010E94D5F1892B11F41092DF
:101AD00020026EEF73E0C8010E94D5F1892B21F43A
:101AE00083E59EE10E94A3AA63E074E0C8010E941E
:101AF000D5F1892B11F40E94AC9861E080EF9FE052
:101B000035D8C0CD2F3531050CF0BCCD9C35C1F496
:101B10000E94F34B97FDB6CD209150102111B2CD0C
:101B20002091F2183091F318A9014F5F5F4F509345
:101B3000F3184093F218F901E051F04F8083A2CDE1
:101B40009B3319F481E080935010809150108111E3
:101B500099CDC90101969093F3188093F218F90179
:101B6000E051F04F40838ECD10925110E4CE0F9093
:101B7000DF91CF911F910F91FF90EF90DF90CF9069
:101B8000BF90AF909F908F907F906F905F904F909D
:101B90003F9008958F929F92AF92BF92EF92FF92E3
:101BA0000F931F93CF93DF93CDB7DEB7A0970FB6F8
:101BB000F894DEBF0FBECDBF61157105810591059B
:101BC00089F100E0842E912CA12CB12C102FEE2451
:101BD000E394F12CEC0EFD1EE00EF11C07FDFA94CF
:101BE000A50194010E941CEEF7016083B901CA01AE
:101BF0000F5F611571058105910541F71F3F21F1C7
:101C0000E1E0F0E0EC0FFD1FE10FF11D17FDFA958B
